:100000000C948A020C94A91A0C94F21C0C941B1FD9
:100010000C94F3200C94CE220C943B130C94911569
:100020000C9468170C94AA1B0C94D61D0C945123A5
:100030000C94BE130C9414160C9459190C949E1F16
:100040000C9476210C94271B0C94D6190C944C1EFE
:100050000C94261C0C9471120C94D6180C94C31496
:100060000C94F2170C9424200C9400220C94DB23A3
:100070000C9448140C949E160C9404030C940403E2
:100080000C9404030C947C180C94531DDF42E94239
:10009000F042F64200430E43DC42DC42DC42DC42EA
:1000A0001D432343264338433B434643DC424943F5
:1000B0004F43524358435B43614364436C432320A3
:1000C00070726F6772616D2076657273696F6E3AD8
:1000D0002025730A00414C41524D3A20496C6C7501
:1000E0006D696E616E6365203D202564206C780A21
:1000F000004552524F523A207374616E6462792007
:10010000666F72207265626F6F740A004552524FBB
:10011000523A2073797374656D206572726F720A3A
:10012000004552524F523A20636F756C64206E6FD7
:10013000742072656164206C696768742073656EF1
:10014000736F720A00414C41524D3A204D696372FF
:100150006F70686F6E65203D2025640A004552521D
:100160004F523A206E6F206C696768742073656E19
:10017000736F7220666F756E640A003A4D562025C3
:10018000730A000A25730A000A25730A00455252B1
:100190004F523A206E6F2062745F737461636B20FC
:1001A0007370656369666965642E0A00726567200D
:1001B00061646472203078253032783A20307825B6
:1001C0003032780A002020202020202020202020EB
:1001D000206D6F6E207665720A002020202020207E
:1001E0002020202020206D6F6E2074696D65727351
:1001F0000A002020202020202020202020206D6F99
:100200006E20726567203C7265672F706F72742F65
:100210006D656D2D616464723E0A002020202020EF
:10022000202020202020206D6F6E206E65740A0033
:100230002020202020202020202020206D6F6E20D4
:10024000697271205B3C6E723E5D0A0020202020A6
:1002500020202020202020206D6F6E206865617096
:100260000A002020202020202020202020206D6F28
:100270006E20636D64203C636D643E0A006D6F6E9A
:100280003A2075736167653A206D6F6E2062617404
:100290000A004261747465727920566F6C746167EC
:1002A000653A2025642E256420560A004261747444
:1002B00065727920566F6C746167653A2065787451
:1002C00065726E616C0A006972712025753A20258D
:1002D0006C750A006972712025753A20256C750AC3
:1002E00000257520627974657320667265650A0061
:1002F000257520636F756E7465642C20627574209B
:100300002575207265706F727465640A002530343B
:1003100078202535640A002825303458290A00251C
:1003200030356C58002530345825366C7525366CC0
:1003300075200041646472205469636B7320204C03
:100340006566742043616C6C6261636B0A004E7574
:10035000744576656E7454696D656F7574004E757D
:100360007454687265616457616B65000A486E6415
:100370006C204E616D6520202020205072696F2016
:1003800053746120515545202054696D7220537477
:100390006B5020467265654D656D0A00202530342E
:1003A00058002530345820252D38732025347520E9
:1003B00025732025303458202530345820253034FA
:1003C0005820253575202573002530345820252DDB
:1003D0003873202534752025732025303458202586
:1003E0003034582025303458202535752025730A9F
:1003F000005445524D494E414C204552524F523ABD
:100400002063616E6E6F7420616C6C6F63206D652C
:100410006D6F72790A0025630021214C494E4520F9
:10042000544F4F204C4F4E4721210A002563202571
:10043000630025733A20636F6D6D616E64206E6F8B
:100440007420666F756E640A000A002563202563B8
:10045000000A207561727420726561642065727291
:100460003A2025640A0042544E5F5445524D494E8D
:10047000414C3A204552524F523A207768696C6598
:100480002072656164696E672066726F6D207561A8
:1004900072740A006661696C65642120636D64731F
:1004A000206275666665722066756C6C210A007242
:1004B00065676973746572696E6720636D643A2558
:1004C0007320006661696C656421206E616D652032
:1004D000746F6F206C6F6E67210A007265676973B5
:1004E000746572696E6720636D643A257320000A33
:1004F0000009000A000A000A0072252E32787C00EA
:100500000A0077252E327820000A007C0072252E02
:100510003278200085B7806885BFECE6F0E0808106
:1005200080688083BF9ABE9AC798C69880EC85BFC2
:10053000AF9AA79AAE9AA69A81EE8093008380E440
:100540008093018385B78F7785BF80E090E09D9B86
:1005500005C0019641F09D9BF8CFFBCF019619F0A5
:100560009D99F3CFFBCF85B7806885BFAF98A798DB
:10057000AE98A69887E089B98093990011241FBE90
:10058000CFEFD0E1DEBFCDBF17E0A0E0B1E0EEE5F8
:10059000F6EF00E00BBF02C007900D92A03DB1073F
:1005A000D9F718E0A0EDB7E001C01D92AC38B10753
:1005B000E1F78FEF9FEF9EBF8DBF2CE838E0C901B8
:1005C000809590958158914038F06FEF7EEF621BD7
:1005D000730BC9010E94E00C0E943F0F892B41F070
:1005E0006FEA73E082E598E00E94367A0E94260F57
:1005F00020E831E040E050E06FE777E088EB93E0FF
:100600000E9404110C9400000C940000FF920F93C0
:100610001F93CF93DF93CDB7DEB722970FB6F89431
:10062000DEBF0FBECDBF84EB0E94640B84E10E944D
:10063000282D0E944F06882341F08DE591E09F937D
:100640008F930E94623A0F900F900E9491290E940E
:10065000F406FF240E94EB068C010E94FF0683E053
:10066000073F180760F01F930F9385E491E09F9375
:100670008F930E94623A0F900F900F900F9064E654
:1006800070E080E090E00E94260AF3949AE0F91668
:1006900009F7BE016E5F7F4FCE0101960E948B0667
:1006A000882381F181E291E09F938F930E94623AC7
:1006B0002FEF41E069E084E00E9452368CE091E047
:1006C0009F938F930E94623A81EF90E09F938F9364
:1006D0000E94623A67EF73E080E090E00E94260A91
:1006E00088E190E02DE00FB6F894A89581BD0FBE8B
:1006F00021BD8DB79EB706960FB6F8949EBF0FBE6C
:100700008DBFA7CF6A8189810E9404068C3D910527
:1007100008F49FCF9F938F9385ED90E09F938F93E5
:100720000E94623A0F900F900F900F9092CF0F930C
:100730001F93CF93DF93CDB7DEB724970FB6F8940E
:10074000DEBF0FBECDBF0E94D43581E00E94FE36D1
:1007500081E00E94B6350CE215E040E060E070E018
:10076000C8010E94C4074091AB055091AC0560E000
:1007700071E0C80102960E94652F80E09BE4A0E032
:10078000B0E089839A83AB83BC838091AB05909161
:10079000AC050E94CC2EAE014F5F5F4F61E071E06F
:1007A0000E94D02F63E071E08091AB059091AC0581
:1007B0000E942B3B8CE091E00E94A03A88E391E0FC
:1007C0000E94A03A05E611E01F930F938EEB90E094
:1007D0009F938F930E94623A83E791E00E94A03A30
:1007E00068EC70E080E090E00E94260A0E94B83F2A
:1007F000B80180E090E00E9417040E94200460E0AD
:1008000074E080E00E94A43F0E9406030F900F90C6
:100810000F900F9081E090E024960FB6F894DEBF21
:100820000FBECDBFDF91CF911F910F91089590938F
:10083000D1078093D0077093D3076093D2070895B0
:100840006CE375E08FE991E00E94133C08958DE719
:1008500092E09F938F930E94623A82E692E09F9388
:100860008F930E94623A8CE492E09F938F930E9450
:10087000623A80E392E09F938F930E94623A8BE109
:1008800092E09F938F930E94623A82EF91E09F9350
:100890008F930E94623A8AED91E09F938F930E941A
:1008A000623A85EC91E09F938F930E94623A8DB7F4
:1008B0009EB740960FB6F8949EBF0FBE8DBF0895A9
:1008C000CF93DF93CDB7DEB722970FB6F894DEBF94
:1008D0000FBECDBF9A83898340E050E0BE016F5FB9
:1008E0007F4F0E94B1789B01AC01FB01672BA9F0FF
:1008F000808199279F938F933F932F938CEA91E068
:100900009F938F930E94623A8DB79EB706960FB65B
:10091000F8949EBF0FBE8DBF02C00E94270422968E
:100920000FB6F894DEBF0FBECDBFDF91CF91089513
:10093000DF92EF92FF920F931F93CF93DF93CDB788
:10094000DEB722970FB6F894DEBF0FBECDBF40E0F2
:1009500050E0BE016F5F7F4F0E94B1787B018C0138
:100960000E94C839EE2019F12E2D3327F901EE0F20
:10097000FF1FEE51FE4F0190F081E02D80819181AB
:10098000A281B381BF93AF939F938F933F932F9394
:1009900084ED92E09F938F930E94623A8DB79EB749
:1009A00008960FB6F8949EBF0FBE8DBF27C000E01B
:1009B00010E082EEE82E81E0F82ED701ED91FD9156
:1009C0007D0180819181A281B381BF93AF939F9379
:1009D0008F931F930F9387EC92E09F938F930E94C6
:1009E000623A0F5F1F4F8DB79EB708960FB6F89407
:1009F0009EBF0FBE8DBF02321105F9F60E94BF39AE
:100A000022960FB6F894DEBF0FBECDBFDF91CF9117
:100A10001F910F91FF90EF90DF9008950E9489340D
:100A2000882349F08CEA92E09F938F930E94623A68
:100A30000F900F90089580E090E00E942E359C0169
:100A400068EE73E00E94997A9F938F93C90168EED4
:100A500073E00E94997A7F936F9382E992E09F936B
:100A60008F930E94623A8DB79EB706960FB6F894A0
:100A70009EBF0FBE8DBF0895CF93DF93EC0144E07E
:100A800050E063EA71E00E943D7A892B49F40E94AC
:100A9000C83980918508909186080E94270D11C061
:100AA00047E050E068EA71E0CE010E943D7A892B70
:100AB00059F40E94C83980918508909186080E9457
:100AC000140E0E94BF399DC046E050E060EB71E01B
:100AD000CE010E943D7A892B49F40E94C839809149
:100AE0008508909186080E94920DEBCF43E050E07C
:100AF00067EB71E0CE010E943D7A892B19F40E94C8
:100B00000E057FC043E050E06BEB71E0CE010E9428
:100B10003D7A892B29F4CE0103960E94980471C076
:100B200043E050E06FEB71E0CE010E943D7A892BEB
:100B300029F4CE0103960E94600463C043E050E0B4
:100B400063EC71E0CE010E943D7A892B81F48091A3
:100B5000D0079091D107892B09F053C08DE891E01F
:100B60009F938F930E94623A0F900F904AC044E087
:100B700050E067EC71E0CE010E943D7A892B29F5A7
:100B80000E94C83980ED91E09F938F9388E891E0AF
:100B90009F938F930E94623ACE0104960E94733B0A
:100BA0008AED91E09F938F9383E891E09F938F93D9
:100BB0000E94623A0E94BF398DB79EB708960FB661
:100BC000F8949EBF0FBE8DBF1CC043E050E06CEC9C
:100BD00071E0CE010E943D7A892B89F48091D20781
:100BE0009091D3079F938F938BE791E09F938F937F
:100BF0000E94623A0F900F900F900F9002C00E94D7
:100C00002704DF91CF910895962F87FF45C067FF96
:100C100043C0E82FFF27EF77F070EE0FFF1FEA5D6C
:100C2000FD4F60817181E92FFF27EF77F070EE0FA4
:100C3000FF1FEA5DFD4F808191816115710561F1B2
:100C40006817790748F19B01281B390B9695982F57
:100C50008827979587950E94857AFB01FF27EA5D93
:100C6000FC4F80819927AC01249FC001259F900DE6
:100C7000349F900D1124892F9927AA27BB278733EA
:100C800057E0950750E0A50750E0B50738F086E338
:100C900097E0A0E0B0E008958FEF9FEF0895CF9226
:100CA000DF92EF92FF920F931F93CF93DF93CDB715
:100CB000DEB722970FB6F894DEBF0FBECDBF83E03C
:100CC000898378EEC72E73E0D72EE12CF12C01E05A
:100CD00010E09E012E5F3F4F41E050E0BE016F5F8C
:100CE0007F4F89E30E942C2E20E030E08A81833000
:100CF00011F021E030E0C90122960FB6F894DEBF72
:100D00000FBECDBFDF91CF911F910F91FF90EF905C
:100D1000DF90CF900895AF92BF92CF92DF92EF9283
:100D2000FF920F931F93CF93DF93CDB7DEB7219739
:100D30000FB6F894DEBF0FBECDBF9C015B01892BBF
:100D4000C1F083E48983F8EECF2EF3E0DF2EE12CAF
:100D5000F12C01E010E041E050E0BE016F5F7F4FF9
:100D600089E30E942C2E8F5F9F4F19F481E090E061
:100D700021C0A114B10419F480E090E01BC083E805
:100D80008983E8EECE2EE3E0DE2EE12CF12C01E0AB
:100D900010E0950141E050E0BE016F5F7F4F89E3B5
:100DA0000E942C2E20E030E08F5F9F4F11F421E055
:100DB00030E0C90121960FB6F894DEBF0FBECDBF5B
:100DC000DF91CF911F910F91FF90EF90DF90CF9027
:100DD000BF90AF9008958091DE079091DF07109249
:100DE000DF071092DE07089520E032E040E050E097
:100DF00061E477E087EA93E00E940411089523E01C
:100E00008833920720F480E00E947E3607C023E0FA
:100E10008E3C920738F480E00E94963681E00E9472
:100E20007E360AC023E0873E920750F480E00E949D
:100E3000963681E00E94963682E00E947E360DC092
:100E400023E0863F920768F480E00E94963681E0B6
:100E50000E94963682E00E94963683E00E947E369B
:100E600008958050944060F480E00E94963681E0BE
:100E70000E94963682E00E94963683E00E94963663
:100E80000895CF93DF93CDB7DEB722970FB6F894CE
:100E9000DEBF0FBECDBF8DEF0E94640B81E090E0FE
:100EA0000E94622987E00E94022981E090E00E946E
:100EB000342980E090E00E94F1280E94F62802C0C8
:100EC0000E94E80BCE0101960E947A298823C1F77F
:100ED0002FEF33E089819A81281B390B3A832983CC
:100EE0008091DE079091DF078217930758F73093C0
:100EF000DF072093DE07E6CF8093C20308950E94A8
:100F0000850820E033E040E050E067E973E08DEBD6
:100F100093E00E9404118EEF0E94640B0E94E80B84
:100F20000E942F0B2091C2032F3FC1F395B785B7C5
:100F3000837E822B85BF85B7806285BF889585B704
:100F40008F7D85BF85B7837E9C71892B85BFE6CF5A
:100F50000F931F93CF93DF938C01C091E107D09142
:100F6000E2070AC0B801CE0102960E942C7A892BB2
:100F700029F00990D881C02D2097A1F7CE01DF91EB
:100F8000CF911F910F910895CF93DF93EC01892B9F
:100F900011F16115710511F07D876C8741114E8744
:100FA000CE0102960E94A807892BA9F4EB89FC893F
:100FB000309721F0CE010995892B69F48091E107E2
:100FC0009091E20799838883D093E207C093E10769
:100FD00080E090E002C08FEF9FEFDF91CF91089506
:100FE00080913B0890913C08A0913D08B0913E084B
:100FF0000196A11DB11D80933B0890933C08A093DE
:101000003D08B0933E080895CF93DF93EC011B8217
:101010001A82E0913908F0913A081AC0288539857A
:101020004A855B8580859185A285B3852817390718
:101030004A075B0780F0281B390B4A0B5B0B28879C
:1010400039874A875B87FB83EA830190F081E02D33
:10105000309721F718C0821B930BA40BB50B808728
:101060009187A287B387F983E883D383C283EA8118
:10107000FB81309719F0D183C08308C0D0933A0820
:10108000C093390803C019821882F1CFDF91CF9144
:1010900008950FB6F8940F9260913B0870913C0848
:1010A00080913D0890913E080F900FBE0895CF9318
:1010B000DF93EC01EA81FB8188819981309719F0F7
:1010C0009183808304C090933A0880933908E88123
:1010D000F9813097A1F08A819B81938382838085F7
:1010E0009185A285B385288539854A855B85820FE0
:1010F000931FA41FB51F80879187A287B387CE0156
:101100000E94730CDF91CF91089580EF97E00E94C9
:10111000BE1187B7826087BF0895EF92FF920F9349
:101120001F93CF93DF930FB6F8940F9220913B0853
:1011300030913C0840913D0850913E080F900FBE01
:101140008091E3079091E407A091E507B091E6074D
:1011500079018A01E81AF90A0A0B1B0B2093E307AD
:101160003093E4074093E5075093E6074FC0888526
:101170009985AA85BB85E816F9060A071B07A0F41E
:101180008E199F09A00BB10B88879987AA87BB8707
:101190000097A105B10521F0EE24FF24870136C098
:1011A000EE24FF24870108C0E81AF90A0A0B1B0B7A
:1011B000188619861A861B86EC85FD85309721F0E6
:1011C0006E857F85CE0109958C819D81AE81BF8121
:1011D00088879987AA87BB870097A105B10521F465
:1011E000CE010E94570812C0E0913908F0913A08E8
:1011F0000190F081E02DF0933A08E09339083097A0
:1012000011F013821282CE010E940408C0913908A5
:10121000D0913A08209731F0E114F104010511054D
:1012200009F0A5CFDF91CF911F910F91FF90EF9023
:1012300008952F923F924F925F926F927F928F927A
:101240009F92AF92BF92CF92DF92EF92FF920F9355
:101250001F93CF93DF93CDB7DEB724970FB6F894E3
:10126000DEBF0FBECDBF0FB6F8940F92A0903B0823
:10127000B0903C08C0903D08D0903E080F900FBE43
:101280000E94B9119B01AC01C601B5010E94AC7A64
:1012900039014A010E94B9111B012C010E94B911A8
:1012A00069837A838B839C83C401B30128EE33E086
:1012B00040E050E00E945A7A7B018C01C401B301E6
:1012C000A20191010E945A7AA61AB70AC80AD90A3D
:1012D000C601B50128EE33E040E050E00E945A7AA2
:1012E00029813A814B815C810E94AC7AE20EF31E27
:1012F000041F151FC801B70124960FB6F894DEBF6E
:101300000FBECDBFDF91CF911F910F91FF90EF9056
:10131000DF90CF90BF90AF909F908F907F906F9015
:101320005F904F903F902F900895EF92FF920F9310
:101330001F930FB6F8940F92E0903B08F0903C0892
:1013400000913D0810913E080F900FBE0E94B91108
:101350009B01AC01C801B7010E94AC7ACA01B90176
:101360001F910F91FF90EF900895AF92BF92CF928F
:10137000DF92EF92FF920F93CF93DF936B017C018B
:10138000EA01590180E190E00E94000CFC01892BE8
:1013900081F10FB6F8940F9280913B0890913C0830
:1013A000A0913D08B0913E080F900FBE8C0D9D1D81
:1013B000AE1DBF1D2091E3073091E4074091E50782
:1013C0005091E607821B930BA40BB50B8087918786
:1013D000A287B38700FF05C0148215821682178288
:1013E00004C0C482D582E682F782D587C487B786D7
:1013F000A686CF01DF91CF910F91FF90EF90DF9004
:10140000CF90BF90AF9008950F93CF93DF930E943A
:10141000B509EC01009711F00E940408CE01DF919C
:10142000CF910F910895CF92DF92EF92FF920F9399
:101430006A0179010E940E129701A6010E94040A16
:101440000F91FF90EF90DF90CF900895AF92BF92F1
:10145000CF92DF92EF92FF920F93CF93DF935B01D6
:101460006C016115710581059105D1F1C1E4D8E0E8
:10147000BE0180914308909144080E94CA0AE091FD
:101480004308F091440883E08787E0904308F09098
:10149000440801E0970145E05BE0C601B5010E9408
:1014A000130AF701968B858B892B19F00E94A30BE9
:1014B00019C0E0914308F0914408D08FC78B809108
:1014C0004108909142089383828381E087878091CD
:1014D000430890914408909342088093410802C0C9
:1014E0000E94E80BDF91CF910F91FF90EF90DF907A
:1014F000CF90BF90AF900895CF93DF93DC019B0115
:10150000EC01788F6F8B1D821C820FB6F8940F92BE
:10151000EB01E881F9818FEFEF3FF80749F4ED0126
:101520008C819D8101969D838C83E0E0F0E015C065
:10153000309799F00F900FBEED019A8908C09F0176
:101540002E5F3F4F0280F381E02D309719F08289A2
:101550009817A8F70FB6F8940F92ED01FB83EA8372
:10156000F901B183A083EA81FB81309771F0848116
:101570009581892B51F08C819D8124813581820F49
:10158000931F9D838C83158214820F900FBEDF9171
:10159000CF910895CF93DF939C01DB010FB6F894B0
:1015A0000F92ED91FC9111970F900FBE8FEFEF3FCF
:1015B000F80731F527C082819381E217F307E9F438
:1015C0000FB6F8940F9211969C938E938481958117
:1015D000892B59F0A281B381109729F084819581DC
:1015E000ED019D838C83158214820F900FBEF9014B
:1015F00013821282108E178A05C0DF011296FC0139
:101600003097C9F6DF91CF910895FB01168A158AAC
:1016100082E0878761E478E0CF010E947C0A089528
:101620000F931F93CF93DF938C01C0913F08D0910C
:1016300040080CC0B801CE0106960E942C7A892B76
:1016400011F4CE0107C00990D881C02D209791F7E1
:1016500080E090E0DF91CF911F910F910895E0918C
:101660004508F0914608309741F0838994890E949B
:10167000730C10924608109245080895CF93DF939B
:10168000C0913F08D09140080E942F0B2091430841
:1016900030914408EFE3F8E00AC088819981C217CD
:1016A000D30719F49183808304C0FE01EC012097D5
:1016B000A1F7809143089091440890934608809345
:1016C0004508DF91CF9108950F931F93182FE09154
:1016D0004308F0914408028961E478E0CF010E9458
:1016E000CA0AE0914308F0914408128B1F3F49F069
:1016F00061E478E080914308909144080E947C0A5C
:1017000002C00E943E0BE0914308F0914408809192
:10171000410890914208E817F90719F481E087879A
:1017200009C082E087870FB6F8940F920E94C51017
:101730000F900FBE802F99271F910F9108958FEF63
:101740000E94640B0895CF93DF93C0913F08D0911E
:10175000400820C00FB6F8940F928C819D810F90A5
:101760000FBE892BA1F0EF89F88D0FB6F8940F9278
:101770008C819D8101979D838C830F900FBE80810A
:1017800091818F5F9F4F19F0CF010E945B0F0990ED
:10179000D881C02D2097F1F60E948D08E091430872
:1017A000F09144088091410890914208E817F907A8
:1017B00061F08785813011F482E087870FB6F89455
:1017C0000F920E94C5100F900FBEDF91CF91089528
:1017D000E0914308F091440882819381892B69F05C
:1017E00061E478E0CF010E94CA0A61E478E0809168
:1017F0004308909144080E947C0A0E94A30B08951C
:101800000F931F93CF93DF930091E7071091E807A1
:101810008017910730F080E090E060C0EF01DB01BD
:101820002FC0AC014A5F5F4F4430510510F444E0D3
:1018300050E0E0914708F091480867E478E0C0E0A4
:10184000D0E0A0E0B0E017C0208131812417350737
:1018500060F02417350711F3209729F088819981CA
:101860002817390710F4EF01DB01BF016E5F7F4FCE
:101870000280F381E02D309739F7CE01209771F186
:1018800028813981CA010A966A817B818217930770
:1018900070F4FE01E40FF51F241B350B3183208308
:1018A0007383628359834883ED93FC9302C06D93E5
:1018B0007C93E881F9810E1B1F0B1093E8070093BE
:1018C000E707EC0FFD1F34978FEE9EEBADEABEED00
:1018D00080839183A283B383CE010296DF91CF915F
:1018E0001F910F910895CF93DF93DC0112976D91B3
:1018F0007C911197E0914708F0914808C7E4D8E03F
:101900003AC040815181CF01840F951F8A179B07F0
:10191000C1F49A01260F371F31832083828193817E
:10192000DF01A20FB31FA817B90791F58D919C9104
:101930001197280F391F31832083ED018A819B8104
:1019400025C0AE17BF0778F4B983A8832D913C91C9
:101950001197CD01820F931F8E179F0779F0ED012C
:10196000FB83EA8315C0A817B90728F1EF01229677
:101970000280F381E02D309721F617C0240F351F28
:1019800011963C932E9382819381FD0193838283F0
:101990008091E7079091E807860F971F9093E807DB
:1019A0008093E70780E090E008C0FD011382128277
:1019B000B983A883EDCF8FEF9FEFDF91CF9108958B
:1019C000FC0161937193CF010E94730C0895809183
:1019D000E7079091E80708950F931F93CF93DF9344
:1019E0008C010E94000CEC01009729F0A80160E036
:1019F00070E00E94227ACE01DF91CF911F910F916A
:101A00000895009729F090934A088093490806C0EA
:101A10008091490890914A08892B19F060934D08EC
:101A2000089510924D080895009729F090934C085E
:101A300080934B0806C080914B0890914C08892BED
:101A400019F060934E08089510924E080895EF9291
:101A5000FF920F931F93CF93DF938C01BC018AE019
:101A600090E00E942C2FC0914708D0914808EE24A6
:101A7000FF2422C088819981E80EF91E9F938F93DD
:101A8000DF93CF938DE093E09F938F931F930F93FA
:101A90000E945D30CE01805690402DB73EB7285F42
:101AA0003F4F0FB6F8943EBF0FBE2DBF805A9F47E1
:101AB00028F40A80DB81C02D2097E1F60E94E70C14
:101AC0008E159F05A9F09F938F93FF92EF9280EF61
:101AD00092E09F938F931F930F930E945D308DB779
:101AE0009EB708960FB6F8949EBF0FBE8DBF13C069
:101AF0009F938F9381EE92E09F938F931F930F9309
:101B00000E945D302DB73EB72A5F3F4F0FB6F89465
:101B10003EBF0FBE2DBFDF91CF911F910F91FF9060
:101B2000EF9008950F931F93CF93DF938C01C09193
:101B30003908D0913A08209709F471C0BC0183E3B9
:101B400093E00E947B3088859985AA85BB85BF93E9
:101B5000AF939F938F938C819D81AE81BF81BF9303
:101B6000AF939F938F93DF93CF9385E293E09F93FF
:101B70008F931F930F930E945D308C859D852DB7A9
:101B80003EB7225F3F4F0FB6F8943EBF0FBE2DBF4A
:101B90003BE08530930721F4B8018EE593E007C060
:101BA0002FE0853F920731F4B8018EE493E00E9464
:101BB0007B301AC0AA27BB27880F991FAA1FBB1FFB
:101BC000BF93AF939F938F938FE193E09F938F93F6
:101BD0001F930F930E945D308DB79EB708960FB686
:101BE000F8949EBF0FBE8DBF8E859F859F938F9368
:101BF00087E193E09F938F931F930F930E945D3033
:101C00000990D881C02D2DB73EB72A5F3F4F0FB640
:101C1000F8943EBF0FBE2DBF209709F094CFDF91FF
:101C2000CF911F910F910895EF92FF920F931F9301
:101C3000CF93DF937C01BC018CE693E00E947B3064
:101C4000C0913F08D09140087AC0EB89FC8980811F
:101C50009181A281B3818F5E9E4BAD4ABE4D19F03A
:101C600083EC93E002C088EC93E0288939894F899E
:101C7000588D9F938F93C9018E1B9F0B9F938F93BA
:101C80003F932F938D899E899F938F935F934F935B
:101C9000EF85FF27EE0FFF1FE251FC4F80819181FE
:101CA0009F938F938A8999279F938F932696DF938B
:101CB000CF932697DF93CF9382EA93E09F938F93FE
:101CC000FF92EF920E945D308F89988DEDB7FEB73D
:101CD00076960FB6F894FEBF0FBEEDBF892B39F193
:101CE000EF89F88D00811181FFEF0F3F1F07E1F4AD
:101CF000B7018BEC93E00E94542F19C01F930F93F0
:101D00008CE993E09F938F93FF92EF920E945D3056
:101D1000F801028113812DB73EB72A5F3F4F0FB6FE
:101D2000F8943EBF0FBE2DBF0115110539F7B7015D
:101D30008AE090E00E942C2F0990D881C02D209736
:101D400009F083CFDF91CF911F910F91FF90EF901A
:101D500008950F931F93CF93DF938C01EB016F5F77
:101D60007F4F09F06BC0BC0184ED93E00E94542FBB
:101D700068C0EB89FC8980819181A281B3818F5EEB
:101D80009E4BAD4ABE4DF1F084819581A681B7810D
:101D90008F5E9E4BAD4ABE4DA9F080859185A28590
:101DA000B3858F5E9E4BAD4ABE4D61F084859585AF
:101DB000A685B7858F5E9E4BAD4ABE4D19F083EC6C
:101DC00093E002C088EC93E0288939894F89588DC7
:101DD0009F938F93C9018E1B9F0B9F938F933F936C
:101DE0002F938D899E899F938F935F934F93EF8558
:101DF000FF27EE0FFF1FE251FC4F808191819F93DF
:101E00008F938A8999279F938F932696DF93CF93F9
:101E10002697DF93CF9389EC93E09F938F931F9343
:101E20000F930E945D300A80DB81C02D8DB79EB775
:101E300046960FB6F8949EBF0FBE8DBF209709F04F
:101E400098CFDF91CF911F910F91089583E18093F7
:101E50004F088FE48093500883E58093510843E155
:101E600050E06FE478E080E090E00E94B710892BAA
:101E700019F08FEF9FEF089580E090E0089543E11F
:101E800050E06FE478E080E090E00E94BA10892B87
:101E900079F480914F08833159F4809150088F3440
:101EA00039F480915108833519F480E090E0089569
:101EB0008FEF9FEF0895CF93DF93DC010FB6F89477
:101EC0000F92CD91DC9111970F900FBE8FEFCF3F06
:101ED000D80709F43AC0209771F10FB6F8940F9221
:101EE000EA81FB811196FC93EE938C819D81892B75
:101EF00071F0309729F08C819D819583848305C092
:101F00008FEF9FEF11969C938E931D821C820F90F2
:101F10000FBE8D899E89009721F00E9457081E8A66
:101F20001D8A82E08F8761E478E0CE010E947C0AFE
:101F300081E090E00CC00FB6F8940F928FEF9FEF06
:101F400011969C938E930F900FBE80E090E0DF91EE
:101F5000CF9108950F931F93CF93DF93EC010FB6AA
:101F6000F8940F92888199810F900FBE2FEF8F3FC9
:101F7000920741F40FB6F8940F92198218820F90CD
:101F80000FBE02C0892B19F400E010E012C000E07F
:101F900010E0CE010E945B0F080F191F0FB6F894D6
:101FA0000F92888199810F900FBE01978E5F9F4F8E
:101FB00080F3C801DF91CF911F910F9108950F9386
:101FC0001F930E94AA0F8C010E94E80BC8011F9169
:101FD0000F9108950F931F930E945B0F8C010E9435
:101FE000E80BC8011F910F910895CF93DF93AC01C7
:101FF000DB010FB6F8940F92CD91DC9111970F9001
:102000000FBE8FEFCF3FD80799F534C08D899E89D9
:102010002A813B818417950741F50FB6F8940F92FA
:1020200011963C932E938C819D81892B81F0EA81BE
:10203000FB81309729F08C819D819583848305C035
:102040008FEF9FEF11969C938E931D821C820F90B1
:102050000FBE82E08F8761E478E0CE010E947C0AA7
:102060008FEF9FEF9E8B8D8B05C0DE011296E901ED
:10207000209761F6DF91CF910895AF92BF92CF92F2
:10208000DF92EF92FF920F93CF93DF93EC015A010F
:102090006B010FB6F8940F92888199810F900FBE53
:1020A0008F5F9F4F51F40FB6F8940F9219821882E8
:1020B0000F900FBE0E94E80B38C061E478E0809179
:1020C0004308909144080E94CA0ABE0180914308C7
:1020D000909144080E947C0AE0914308F0914408E2
:1020E00083E08787E0904308F0904408A114B1048E
:1020F000C104D10461F001E09E0145EF5FE0C6013B
:10210000B5010E94130AF701968B858B03C0F70176
:10211000168A158A0E94A30BE0914308F0914408A7
:10212000858996898F5F9F4F19F080E090E004C009
:10213000168A158A8FEF9FEFDF91CF910F91FF9055
:10214000EF90DF90CF90BF90AF900895FC010FB655
:10215000F8940F92808191818F5F9F4F11F41182CB
:1021600010820F900FBECF010E943D1008950E9473
:10217000BF2908950E94DF2908959F918F910F90A4
:102180000BBE0F900FBE1F9018952F923F924F924B
:102190005F926F927F928F929F92AF92BF92CF92F7
:1021A000DF92EF92FF920F931F93CF93DF938DB740
:1021B0009EB7E0914308F0914408918B808BE091A9
:1021C0004108F0914208F0934408E093430881E00D
:1021D0008787E0914308F0914408808991898DBFF9
:1021E0009EBFDF91CF911F910F91FF90EF90DF90F5
:1021F000CF90BF90AF909F908F907F906F905F90A7
:102200004F903F902F900895CF92DF92EF92FF92E0
:102210000F931F93CF93DF938C017B016A01E90138
:10222000C90149960E94000CFC01009719F480E056
:1022300090E075C0C80FD91F9E0127503040AE01F5
:102240004B515040CE01069668E0D8010D908D01AB
:10225000DC010D92CD016150C1F71E864150504006
:10226000598B488B4F5F5F4FFC8BEB8B8FEE9EEB58
:10227000ADEABEED80839183A283B383848395838B
:10228000A683B78380879187A287B3878487958742
:10229000A687B78780E48A8B8F2D9927F9018583DC
:1022A000E68280E8838312821482C1828D2D992771
:1022B00080832DEB30E1832F9927FA01828B238BCA
:1022C00080913F089091400899838883D09340087B
:1022D000C0933F0812E01F871E8A1D8A188E1F8A2E
:1022E00061E478E0CE010E947C0AE0914308F0911D
:1022F0004408309721F40FB6F8940F9260CF809184
:10230000410890914208E817F90741F017870FB686
:10231000F8940F920E94C5100F900FBECE01DF916E
:10232000CF911F910F91FF90EF90DF90CF90089584
:102330001F93182F6091E9077091EA078091EB07CE
:102340009091EC0720EA3FE040E050E00E94AC7A38
:10235000822F932F0197F1F71A95D1F71F910895C6
:102360006091E9077091EA078091EB079091EC0783
:10237000089560E074E080E090E00895BC0187B7C4
:102380008D7F87BF80B7886080BF12BE82E083BF29
:1023900080B7992787709070892BD1F781E086BF2D
:1023A0000FB6F8940F9281E090E0A0E0B0E0B6B7ED
:1023B000B170E9F3B6BF0894811D911DA11DB6B798
:1023C000B170C9F3BB270F900FBE27E0880F991F8C
:1023D000AA1FBB1F2A95D1F78093E9079093EA07BC
:1023E000A093EB07B093EC0787B78D7F87BF80B7CB
:1023F000886080BF12BE89E083BF8FE181BF80B754
:10240000992787709070892BD1F782E086BF40E0D2
:1024100050E08CED94E00E941B46089528EE33E0D6
:1024200040E050E00E945A7A3AE096958795779579
:1024300067953A95D1F708959C01FB0186B1482F25
:1024400055274870507033982131310569F1223198
:1024500031054CF421303105A1F020313105A1F0D6
:10246000232B69F009C02032310509F120363105EE
:1024700009F12231310591F18FEF9FEF2BC040E040
:1024800050E080E186B924C0349B05C081E090E033
:102490009183808302C011821082452BF9F08081E4
:1024A000918180689183808380E090E015C01182E3
:1024B00010820EC08091F6039091F7039183808380
:1024C0001092F6031092F7031092F8031092F9039A
:1024D00080E090E0452B21F0339A089580E090E071
:1024E00008951F920F920FB60F9211242F933F93CE
:1024F0004F935F936F937F938F939F93AF93BF930C
:10250000EF93FF9386EF93E00E940546FF91EF91D2
:10251000BF91AF919F918F917F916F915F914F91FB
:102520003F912F910F900FBE0F901F9018959C0117
:10253000FB0189B7482F55274072507089B78F7DAE
:1025400089BF2231310509F492C0233131058CF461
:102550002130310541F1223031051CF4232BE9F003
:102560007EC02031310511F12131310509F077C0EC
:102570002FC02931310509F442C02A3131052CF42C
:102580002831310509F06BC026C02032310541F1F8
:102590002036310509F063C053C08AB78B7F8ABFEC
:1025A0008AB7877F8ABF80E288BF1EC008B605FE53
:1025B00005C081E090E09183808302C01182108287
:1025C000452B09F454C08081918180689183808378
:1025D00020E030E048C08AB7982F987083FF07C08A
:1025E00085E090E09183808320E030E03AC0943031
:1025F00019F487E090E0F6CF81E090E0F3CF6081BE
:1026000071816130710519F48AB78B7F05C067301D
:10261000710531F48AB784608ABF8AB7877F0EC09C
:102620006530710519F48AB78B7F05C06630710576
:10263000B1F48AB784608ABF8AB788608ABFD4CF72
:102640008091000490910104918380831092000492
:10265000109201041092020410920304C5CF2FEFD0
:102660003FEF452B31F089B7806289BF02C020E07F
:1026700030E0C90108951F920F920FB60F921124F6
:102680002F933F934F935F936F937F938F939F937A
:10269000AF93BF93EF93FF9380E094E00E940546D1
:1026A000FF91EF91BF91AF919F918F917F916F912A
:1026B0005F914F913F912F910F900FBE0F901F9000
:1026C00018959C01FB0187B7482F55274071507022
:1026D00087B78F7E87BF2131310571F122313105F6
:1026E0004CF421303105A1F020313105A1F0232B2C
:1026F00069F009C02032310511F12036310521F190
:1027000022313105B9F12FEF3FEF2EC040E050E00C
:1027100080E186BF27C006B604FE05C081E090E0D8
:102720009183808302C011821082452B19F1808130
:10273000918180689183808320E030E017C08BE036
:1027400090E0918380830EC080910A0490910B04E5
:102750009183808310920A0410920B0410920C044F
:1027600010920D0420E030E0452B31F087B78061F6
:1027700087BF02C020E030E0C90108951F920F9288
:102780000FB60F9211242F933F934F935F936F9344
:102790007F938F939F93AF93BF93EF93FF938AE0C1
:1027A00094E00E940546FF91EF91BF91AF919F91F8
:1027B0008F917F916F915F914F913F912F910F90EA
:1027C0000FBE0F901F9018959C01FB0180917D001A
:1027D000482F55274270507080917D008D7F8093E7
:1027E0007D002131310581F1223131054CF4213058
:1027F0003105A1F020313105A9F0232B69F009C082
:102800002032310521F12036310531F122313105F7
:10281000D9F12FEF3FEF30C040E050E082E08093ED
:102820007C0028C080917C0081FF05C081E090E0A1
:102830009183808302C011821082452B29F180810F
:10284000918180689183808320E030E017C08BE025
:1028500090E0918380830EC08091140490911504C0
:102860009183808310921404109215041092160420
:102870001092170420E030E0452B41F080917D005C
:10288000826080937D0002C020E030E0C90108959D
:102890001F920F920FB60F9211242F933F934F93D5
:1028A0005F936F937F938F939F93AF93BF93EF93B8
:1028B000FF9384E194E00E940546FF91EF91BF9160
:1028C000AF919F918F917F916F915F914F913F91C8
:1028D0002F910F900FBE0F901F9018959C01FB0138
:1028E00088B1482F552748705070439821313105E1
:1028F00069F1223131054CF421303105A1F020314C
:102900003105A1F0232B69F009C02032310509F10E
:102910002036310509F12231310591F18FEF9FEF1A
:102920002BC040E050E080E186B924C0449B05C044
:1029300081E090E09183808302C011821082452B58
:10294000F9F08081918180689183808380E090E0BC
:1029500015C0118210820EC080911E0490911F0438
:102960009183808310921E0410921F041092200401
:102970001092210480E090E0452B21F0439A0895C5
:1029800080E090E008951F920F920FB60F921124ED
:102990002F933F934F935F936F937F938F939F9367
:1029A000AF93BF93EF93FF938EE194E00E940546AF
:1029B000FF91EF91BF91AF919F918F917F916F9117
:1029C0005F914F913F912F910F900FBE0F901F90ED
:1029D00018959C01FB0189B7482F5527407450700A
:1029E00089B78F7B89BF2231310509F496C0233125
:1029F00031058CF42130310549F1223031051CF4C8
:102A0000232BF1F082C02031310519F1213131053C
:102A100009F07BC030C02931310509F443C02A31A7
:102A200031052CF42831310509F06FC027C0203260
:102A3000310509F458C02036310509F066C056C08A
:102A40008AB78F7E8ABF8AB78F7D8ABF80E488BFAE
:102A50001EC008B606FE05C081E090E09183808329
:102A600002C011821082452B09F457C080819181E8
:102A700080689183808320E030E04BC08AB7982F34
:102A8000907285FF07C085E090E09183808320E00D
:102A900030E03DC0903119F487E090E0F6CF81E05E
:102AA00090E0F3CF608171816130710519F48AB7CC
:102AB0008F7E05C06730710531F48AB780618ABFA7
:102AC0008AB78F7D0EC06530710519F48AB78F7E85
:102AD00005C066307105C9F48AB780618ABF8AB7BC
:102AE00080628ABFD4CF86E090E0CFCF8091280467
:102AF00090912904918380831092280410922904D4
:102B000010922A0410922B04C2CF2FEF3FEF452BD7
:102B100031F089B7806489BF02C020E030E0C9018C
:102B200008951F920F920FB60F9211242F933F9387
:102B30004F935F936F937F938F939F93AF93BF93C5
:102B4000EF93FF9388E294E00E940546FF91EF9196
:102B5000BF91AF919F918F917F916F915F914F91B5
:102B60003F912F910F900FBE0F901F9018959C01D1
:102B7000FB0187B7482F55274870507087B7877F6C
:102B800087BF2131310571F1223131054CF42130FB
:102B90003105A1F020313105A1F0232B69F009C0E6
:102BA0002032310511F12036310521F12231310574
:102BB000B9F12FEF3FEF2EC040E050E088E086BF34
:102BC00027C006B603FE05C081E090E091838083B4
:102BD00002C011821082452B19F180819181806899
:102BE0009183808320E030E017C08CE090E09183F7
:102BF00080830EC08091320490913304918380834E
:102C0000109232041092330410923404109235045E
:102C100020E030E0452B31F087B7886087BF02C0E5
:102C200020E030E0C90108951F920F920FB60F9275
:102C300011242F933F934F935F936F937F938F93C1
:102C40009F93AF93BF93EF93FF9382E394E00E942F
:102C50000546FF91EF91BF91AF919F918F917F9129
:102C60006F915F914F913F912F910F900FBE0F90F9
:102C70001F9018959C01FB0180917D00482F5527DE
:102C80004470507080917D008B7F80937D00213156
:102C9000310581F1223131054CF421303105A1F0AB
:102CA00020313105A9F0232B69F009C0203231050C
:102CB00021F12036310531F122313105D9F12FEFE3
:102CC0003FEF30C040E050E084E080937C0028C0BB
:102CD00080917C0082FF05C081E090E09183808339
:102CE00002C011821082452B29F180819181806878
:102CF0009183808320E030E017C08CE190E09183E5
:102D000080830EC080913C0490913D049183808328
:102D100010923C0410923D0410923E0410923F0425
:102D200020E030E0452B41F080917D00846080936D
:102D30007D0002C020E030E0C90108951F920F928B
:102D40000FB60F9211242F933F934F935F936F937E
:102D50007F938F939F93AF93BF93EF93FF938CE3F6
:102D600094E00E940546FF91EF91BF91AF919F9132
:102D70008F917F916F915F914F913F912F910F9024
:102D80000FBE0F901F9018959C01FB0189B7482F2B
:102D900055274078507089B78F7789BF2231310528
:102DA00009F492C0233131058CF42130310549F109
:102DB000223031051CF4232BF1F07EC02031310587
:102DC00019F12131310509F077C030C029313105C1
:102DD00009F43FC02A3131052CF42831310509F0BE
:102DE0006BC027C02032310509F454C020363105AC
:102DF00009F062C052C08AB78F7B8ABF8AB78F77CB
:102E00008ABF80E888BF1DC008B607FE05C081E004
:102E100090E09183808302C011821082452B09F4D7
:102E200053C08081918180689183808320E030E06D
:102E300047C08AB78078803839F485E090E0918384
:102E4000808320E030E03AC0803421F181E090E0DE
:102E5000F6CF608171816130710519F48AB78F7B7B
:102E600005C06730710531F48AB780648ABF8AB7BC
:102E70008F770EC06530710519F48AB78F7B05C056
:102E800066307105C9F48AB780648ABF8AB78068E2
:102E90008ABFD7CF87E090E0D2CF8091460490914F
:102EA0004704918380831092460410924704109245
:102EB000480410924904C5CF2FEF3FEF452B31F066
:102EC00089B7806889BF02C020E030E0C901089559
:102ED0001F920F920FB60F9211242F933F934F938F
:102EE0005F936F937F938F939F93AF93BF93EF9372
:102EF000FF9386E494E00E940546FF91EF91BF9115
:102F0000AF919F918F917F916F915F914F913F9181
:102F10002F910F900FBE0F901F9018959C01FB01F1
:102F200080917D00482F55274170507080917D0021
:102F30008E7F80937D002131310581F12231310571
:102F40004CF421303105A1F020313105A9F0232BBB
:102F500069F009C02032310521F12036310531F107
:102F600022313105D9F12FEF3FEF30C040E050E082
:102F700081E080937C0028C080917C0080FF05C0A8
:102F800081E090E09183808302C011821082452B02
:102F900029F18081918180689183808320E030E0F5
:102FA00017C087E190E0918380830EC08091500428
:102FB0009091510491838083109250041092510497
:102FC000109252041092530420E030E0452B41F05F
:102FD00080917D00816080937D0002C020E030E020
:102FE000C90108951F920F920FB60F9211242F93CB
:102FF0003F934F935F936F937F938F939F93AF9381
:10300000BF93EF93FF9380E594E00E940546FF9104
:10301000EF91BF91AF919F918F917F916F915F9150
:103020004F913F912F910F900FBE0F901F901895C9
:103030009C01FB0180917400482F5527417050700E
:10304000809174008E7F809374002131310581F16D
:10305000223131054CF421303105A1F02031310508
:10306000A9F0232B69F009C02032310521F1203667
:10307000310531F122313105D9F12FEF3FEF30C069
:1030800040E050E0779B2AC08FB128C08091740047
:1030900087FF05C081E090E09183808302C01182A8
:1030A0001082452B29F180819181806891838083F2
:1030B00020E030E017C080E190E0918380830EC073
:1030C00080915A0490915B049183808310925A04FA
:1030D00010925B0410925C0410925D0420E030E0DA
:1030E000452B41F08091740081608093740002C090
:1030F00020E030E0C90108951F920F920FB60F92A1
:1031000011242F933F934F935F936F937F938F93EC
:103110009F93AF93BF93EF93FF938AE594E00E9450
:103120000546FF91EF91BF91AF919F918F917F9154
:103130006F915F914F913F912F910F900FBE0F9024
:103140001F901895FB012CB3E3988231910579F01B
:10315000833191052CF4009751F0419771F40AC026
:103160008032910569F08036910539F40CC080E019
:1031700090E0089580E090E017C08FEF9FEF13C0BC
:10318000118210820EC08091640490916504918335
:103190008083109264041092650410926604109269
:1031A000670480E090E023FDE39A08951F920F9258
:1031B0000FB60F9211242F933F934F935F936F930A
:1031C0007F938F939F93AF93BF93EF93FF9384E687
:1031D00094E00E940546FF91EF91BF91AF919F91BE
:1031E0008F917F916F915F914F913F912F910F90B0
:1031F0000FBE0F901F9018959C01FB0187B7482FB9
:1032000055274470507087B78B7F87BF21313105B8
:1032100071F1223131054CF421303105A1F020311A
:103220003105A1F0232B69F009C02032310511F1DD
:103230002036310521F122313105B9F12FEF3FEF71
:103240002EC040E050E084E086BF27C006B602FEF4
:1032500005C081E090E09183808302C011821082DA
:10326000452B19F18081918180689183808320E0D2
:1032700030E017C08DE090E0918380830EC0809194
:103280006E0490916F049183808310926E0410926B
:103290006F04109270041092710420E030E0452B0E
:1032A00031F087B7846087BF02C020E030E0C901F9
:1032B00008951F920F920FB60F9211242F933F93F0
:1032C0004F935F936F937F938F939F93AF93BF932E
:1032D000EF93FF938EE694E00E940546FF91EF91F5
:1032E000BF91AF919F918F917F916F915F914F911E
:1032F0003F912F910F900FBE0F901F9018959C013A
:10330000FB018AB1482F55274078507057982131DA
:10331000310569F1223131054CF421303105A1F03C
:1033200020313105A1F0232B69F009C0203231058D
:1033300009F12036310519F122313105A1F18FEF64
:103340009FEF2DC040E050E08CB18CB126C05F9B58
:1033500005C081E090E09183808302C011821082D9
:10336000452B09F18081918180689183808380E081
:1033700090E017C080E190E0918380830EC080913F
:10338000780490917904918380831092780410924C
:10339000790410927A0410927B0480E090E0452B2F
:1033A00021F0579A089580E090E008951F920F92BF
:1033B0000FB60F9211242F933F934F935F936F9308
:1033C0007F938F939F93AF93BF93EF93FF9388E780
:1033D00094E00E940546FF91EF91BF91AF919F91BC
:1033E0008F917F916F915F914F913F912F910F90AE
:1033F0000FBE0F901F9018959C01FB0189B7482FB5
:1034000055274170507089B78E7F89BF22313105B1
:1034100009F49BC0233131058CF42130310569F169
:10342000223031051CF4232BF1F087C02031310507
:1034300039F12131310509F080C034C0293131051D
:1034400009F446C02A3131052CF42831310509F040
:1034500074C02BC02032310509F45DC0203631051F
:1034600009F06BC05BC080916A008E7F80936A0018
:1034700080916A008D7F80936A0081E088BF1DC0C3
:1034800008B600FE05C081E090E09183808302C011
:1034900011821082452B09F458C080819181806887
:1034A0009183808320E030E04CC080916A0083707B
:1034B00039F481E090E09183808320E030E03FC0E8
:1034C000833019F486E090E0F6CF85E090E0F3CF0A
:1034D000608171816130710549F480916A008E7F4D
:1034E00080936A0080916A008D7F12C065307105FB
:1034F00021F480916A008E7F06C066307105E9F480
:1035000080916A00816080936A0080916A00826085
:1035100080936A00D2CF11821082CFCF8091820433
:10352000909183049183808310928204109283048B
:103530001092840410928504C0CF2FEF3FEF452BEB
:1035400031F089B7816089BF02C020E030E0C90155
:1035500008951F920F920FB60F9211242F933F934D
:103560004F935F936F937F938F939F93AF93BF938B
:10357000EF93FF9382E894E00E940546FF91EF915C
:10358000BF91AF919F918F917F916F915F914F917B
:103590003F912F910F900FBE0F901F9018959C0197
:1035A000FB018DB1482F5527407850706F9821311D
:1035B000310571F1223131054CF421303105A1F092
:1035C00020313105A9F0232B69F009C020323105E3
:1035D00011F12036310521F122313105A9F18FEFAA
:1035E0009FEF2EC040E050E0779B28C08FB126C0EF
:1035F000779B05C081E090E09183808302C01182B7
:103600001082452B09F180819181806891838083AC
:1036100080E090E017C080E190E0918380830EC04D
:1036200080918C0490918D049183808310928C04FE
:1036300010928D0410928E0410928F0480E090E01E
:10364000452B21F06F9A089580E090E008951F9235
:103650000F920FB60F9211242F933F934F935F93C6
:103660006F937F938F939F93AF93BF93EF93FF934A
:103670008CE894E00E940546FF91EF91BF91AF91D5
:103680009F918F917F916F915F914F913F912F917A
:103690000F900FBE0F901F9018959C01FB0187B7EC
:1036A000482F55274078507087B78F7787BF2131D3
:1036B000310571F1223131054CF421303105A1F091
:1036C00020313105A1F0232B69F009C020323105EA
:1036D00011F12036310521F122313105B9F12FEFF9
:1036E0003FEF2EC040E050E080E886BF27C006B61E
:1036F00007FE05C081E090E09183808302C01182C3
:103700001082452B19F1808191818068918380839B
:1037100020E030E017C088E090E0918380830EC005
:1037200080919604909197049183808310929604DF
:1037300010929704109298041092990420E030E0BF
:10374000452B31F087B7806887BF02C020E030E0AA
:10375000C90108951F920F920FB60F9211242F9353
:103760003F934F935F936F937F938F939F93AF9309
:10377000BF93EF93FF9386E994E00E940546FF9183
:10378000EF91BF91AF919F918F917F916F915F91D9
:103790004F913F912F910F900FBE0F901F90189552
:1037A0009C01FB018AB1482F5527407450705698F0
:1037B0002131310561F1223131054CF421303105DF
:1037C000A1F02031310599F0232B69F009C0203296
:1037D000310501F12036310511F12231310599F120
:1037E0008FEF9FEF2CC040E050E05E9A26C05E9BBA
:1037F00005C081E090E09183808302C01182108235
:10380000452B09F18081918180689183808380E0DC
:1038100090E017C080E190E0918380830EC080919A
:10382000A0049091A104918380831092A00410922F
:10383000A1041092A2041092A30480E090E0452B12
:1038400021F0569A089580E090E008951F920F921B
:103850000FB60F9211242F933F934F935F936F9363
:103860007F938F939F93AF93BF93EF93FF9380EAE0
:1038700094E00E940546FF91EF91BF91AF919F9117
:103880008F917F916F915F914F913F912F910F9009
:103890000FBE0F901F9018959C01FB0189B7482F10
:1038A00055274270507089B78D7F89BF223131050D
:1038B00009F494C0233131058CF42130310569F1CC
:1038C000223031051CF4232BF1F080C0203131056A
:1038D00039F12131310509F079C034C02931310580
:1038E00009F43FC02A3131052CF42831310509F0A3
:1038F0006DC02BC02032310509F456C02036310589
:1039000009F064C054C080916A008B7F80936A0084
:1039100080916A00877F80936A0082E088BF1EC022
:1039200008B601FE05C081E090E09183808302C06B
:1039300011821082452B09F451C0808191818068E9
:103940009183808320E030E045C080916A008C70D4
:10395000883051F585E090E09183808320E030E06D
:1039600037C0608171816130710549F480916A00CE
:103970008B7F80936A0080916A00877F12C06530D8
:10398000710521F480916A008B7F06C06630710555
:10399000E9F480916A00846080936A0080916A00F3
:1039A000886080936A00DACF81E090E0D5CF809183
:1039B000AA049091AB04918380831092AA04109280
:1039C000AB041092AC041092AD04C8CF2FEF3FEFC0
:1039D000452B31F089B7826089BF02C020E030E01A
:1039E000C90108951F920F920FB60F9211242F93C1
:1039F0003F934F935F936F937F938F939F93AF9377
:103A0000BF93EF93FF938AEA94E00E940546FF91EB
:103A1000EF91BF91AF919F918F917F916F915F9146
:103A20004F913F912F910F900FBE0F901F901895BF
:103A3000FB0140916800E3988231910579F0833170
:103A400091052CF4009751F0419771F40AC080322F
:103A5000910569F08036910539F40CC020E030E022
:103A600020C020E030E018C02FEF3FEF13C01182DC
:103A700010820EC08091B4049091B504918380832C
:103A80001092B4041092B5041092B6041092B704C8
:103A900020E030E047FF05C0809168008068809397
:103AA0006800C90108951F920F920FB60F9211245A
:103AB0002F933F934F935F936F937F938F939F9336
:103AC000AF93BF93EF93FF9384EB94E00E9405467E
:103AD000FF91EF91BF91AF919F918F917F916F91E6
:103AE0005F914F913F912F910F900FBE0F901F90BC
:103AF00018959C01FB0187B7482F552740745070DB
:103B000087B78F7B87BF2131310571F122313105B4
:103B10004CF421303105A1F020313105A1F0232BE7
:103B200069F009C02032310511F12036310521F14B
:103B300022313105B9F12FEF3FEF2EC040E050E0C8
:103B400080E486BF27C006B606FE05C081E090E08F
:103B50009183808302C011821082452B19F18081EC
:103B6000918180689183808320E030E017C089E0F4
:103B700090E0918380830EC08091BE049091BF0439
:103B8000918380831092BE041092BF041092C004EF
:103B90001092C10420E030E0452B31F087B78064FB
:103BA00087BF02C020E030E0C90108951F920F9244
:103BB0000FB60F9211242F933F934F935F936F9300
:103BC0007F938F939F93AF93BF93EF93FF938EEB6E
:103BD00094E00E940546FF91EF91BF91AF919F91B4
:103BE0008F917F916F915F914F913F912F910F90A6
:103BF0000FBE0F901F9018959C01FB018AB1482FB2
:103C000055274072507055982131310531F12231DC
:103C100031053CF421153105E1F12031310551F434
:103C20000CC020323105E1F020363105F1F02231AF
:103C3000310579F18FEF9FEF28C05D9B05C081E0D2
:103C400090E09183808302C011821082452B09F19C
:103C50008081918180689183808380E090E017C0AB
:103C600080E190E0918380830EC08091C8049091A0
:103C7000C904918380831092C8041092C9041092E1
:103C8000CA041092CB0480E090E0452B21F0559AB5
:103C9000089580E090E008951F920F920FB60F9262
:103CA00011242F933F934F935F936F937F938F9341
:103CB0009F93AF93BF93EF93FF9388EC94E00E94A0
:103CC0000546FF91EF91BF91AF919F918F917F91A9
:103CD0006F915F914F913F912F910F900FBE0F9079
:103CE0001F9018959C01FB0189B7482F55274470F8
:103CF000507089B78B7F89BF2231310509F497C095
:103D0000233131058CF42130310569F12230310540
:103D10001CF4232BF1F083C02031310539F121311E
:103D2000310509F07CC034C02931310509F442C0A5
:103D30002A3131052CF42831310509F070C02BC02F
:103D40002032310509F459C02036310509F067C029
:103D500057C080916A008F7E80936A0080916A00CC
:103D60008F7D80936A0084E088BF1EC008B602FE83
:103D700005C081E090E09183808302C011821082AF
:103D8000452B09F454C080819181806891838083A0
:103D900020E030E048C080916A008073803239F4BE
:103DA00085E090E09183808320E030E03AC081E0BC
:103DB00090E0F8CF608171816130710549F48091A4
:103DC0006A008F7E80936A0080916A008F7D12C0A6
:103DD0006530710521F480916A008F7E06C06630DF
:103DE0007105E9F480916A00806180936A00809196
:103DF0006A00806280936A00D7CF82E090E0D2CFE1
:103E00008091D2049091D304918380831092D20444
:103E10001092D3041092D4041092D504C5CF2FEF82
:103E20003FEF452B31F089B7846089BF02C020E0A5
:103E300030E0C90108951F920F920FB60F9211241E
:103E40002F933F934F935F936F937F938F939F93A2
:103E5000AF93BF93EF93FF9382ED94E00E940546EA
:103E6000FF91EF91BF91AF919F918F917F916F9152
:103E70005F914F913F912F910F900FBE0F901F9028
:103E800018959C01FB0187B7482F55274270507049
:103E900087B78D7F87BF2131310571F1223131051F
:103EA0004CF421303105A1F020313105A1F0232B54
:103EB00069F009C02032310511F12036310521F1B8
:103EC00022313105B9F12FEF3FEF2EC040E050E035
:103ED00082E086BF27C006B601FE05C081E090E003
:103EE0009183808302C011821082452B19F1808159
:103EF000918180689183808320E030E017C08EE05C
:103F000090E0918380830EC08091DC049091DD0469
:103F1000918380831092DC041092DD041092DE0401
:103F20001092DF0420E030E0452B31F087B782604B
:103F300087BF02C020E030E0C90108951F920F92B0
:103F40000FB60F9211242F933F934F935F936F936C
:103F50007F938F939F93AF93BF93EF93FF938CEDDA
:103F600094E00E940546FF91EF91BF91AF919F9120
:103F70008F917F916F915F914F913F912F910F9012
:103F80000FBE0F901F9018959C01FB0180917D0042
:103F9000482F55274072507080917D008F7D80930F
:103FA0007D002131310571F1223131054CF437FDAD
:103FB00010C02230310584F02031310551F410C099
:103FC0002032310511F12036310511F12231310550
:103FD000B9F12FEF3FEF2CC080E280937C0026C028
:103FE00080917C0085FF05C081E090E09183808313
:103FF00002C011821082452B19F180819181806865
:104000009183808320E030E015C0118210820EC0C1
:104010008091E6049091E704918380831092E604F6
:104020001092E7041092E8041092E90420E030E0D6
:10403000452B41F080917D00806280937D0002C01D
:1040400020E030E0C90108951F920F920FB60F9241
:1040500011242F933F934F935F936F937F938F938D
:104060009F93AF93BF93EF93FF9386EE94E00E94EC
:104070000546FF91EF91BF91AF919F918F917F91F5
:104080006F915F914F913F912F910F900FBE0F90C5
:104090001F9018959C01FB0189B7482F5527487040
:1040A000507089B7877F89BF2231310509F497C0E5
:1040B000233131058CF42130310569F1223031058D
:1040C0001CF4232BF1F083C02031310539F121316B
:1040D000310509F07CC034C02931310509F442C0F2
:1040E0002A3131052CF42831310509F070C02BC07C
:1040F0002032310509F459C02036310509F067C076
:1041000057C080916A008F7B80936A0080916A001B
:104110008F7780936A0088E088BF1EC008B603FED0
:1041200005C081E090E09183808302C011821082FB
:10413000452B09F454C080819181806891838083EC
:1041400020E030E048C080916A00807C803839F4FB
:1041500085E090E09183808320E030E03AC081E008
:1041600090E0F8CF608171816130710549F48091F0
:104170006A008F7B80936A0080916A008F7712C0FB
:104180006530710521F480916A008F7B06C066302E
:104190007105E9F480916A00806480936A008091DF
:1041A0006A00806880936A00D7CF83E090E0D2CF26
:1041B0008091F0049091F104918380831092F00437
:1041C0001092F1041092F2041092F304C5CF2FEF75
:1041D0003FEF452B31F089B7886089BF02C020E0EE
:1041E00030E0C90108951F920F920FB60F9211246B
:1041F0002F933F934F935F936F937F938F939F93EF
:10420000AF93BF93EF93FF9380EF94E00E94054636
:10421000FF91EF91BF91AF919F918F917F916F919E
:104220005F914F913F912F910F900FBE0F901F9074
:1042300018959C01FB0187B7482F55274170507096
:1042400087B78E7F87BF2131310571F1223131056A
:104250004CF421303105A1F020313105A1F0232BA0
:1042600069F009C02032310511F12036310521F104
:1042700022313105B9F12FEF3FEF2EC040E050E081
:1042800081E086BF27C006B600FE05C081E090E051
:104290009183808302C011821082452B19F18081A5
:1042A000918180689183808320E030E017C08FE0A7
:1042B00090E0918380830EC08091FA049091FB047A
:1042C000918380831092FA041092FB041092FC04F4
:1042D0001092FD0420E030E0452B31F087B781607B
:1042E00087BF02C020E030E0C90108951F920F92FD
:1042F0000FB60F9211242F933F934F935F936F93B9
:104300007F938F939F93AF93BF93EF93FF938AEF26
:1043100094E00E940546FF91EF91BF91AF919F916C
:104320008F917F916F915F914F913F912F910F905E
:104330000FBE0F901F9018959C01FB0180917D008E
:10434000482F55274071507080917D008F7E80935B
:104350007D002131310581F1223131054CF42130CC
:104360003105A1F020313105A9F0232B69F009C0F6
:104370002032310521F12036310531F1223131056C
:10438000D9F12FEF3FEF30C040E050E080E1809363
:104390007C0028C080917C0084FF05C081E090E013
:1043A0009183808302C011821082452B29F1808184
:1043B000918180689183808320E030E017C089E19B
:1043C00090E0918380830EC0809104059091050553
:1043D00091838083109204051092050510920605C2
:1043E0001092070520E030E0452B41F080917D00E0
:1043F000806180937D0002C020E030E0C901089513
:104400001F920F920FB60F9211242F933F934F9349
:104410005F936F937F938F939F93AF93BF93EF932C
:10442000FF9384E095E00E940546FF91EF91BF91D4
:10443000AF919F918F917F916F915F914F913F913C
:104440002F910F900FBE0F901F9018959C01FB01AC
:1044500089B7482F55274071507089B78F7E89BF23
:104460002231310509F496C0233131058CF4213015
:10447000310549F1223031051CF4232BF1F082C0C3
:104480002031310519F12131310509F07BC030C0EF
:104490002931310509F443C02A3131052CF4283182
:1044A000310509F06FC027C02032310509F458C02A
:1044B0002036310509F066C056C08AB78E7F8ABFA4
:1044C0008AB78D7F8ABF80E188BF1EC008B604FE10
:1044D00005C081E090E09183808302C01182108248
:1044E000452B09F457C08081918180689183808336
:1044F00020E030E04BC08AB7982F927081FF07C050
:1045000085E090E09183808320E030E03DC09130F1
:1045100019F487E090E0F6CF81E090E0F3CF60817E
:1045200071816130710519F48AB78E7F05C06730DB
:10453000710531F48AB781608ABF8AB78D7F0EC05A
:104540006530710519F48AB78E7F05C06630710534
:10455000C9F48AB781608ABF8AB782608ABFD4CF24
:1045600084E090E0CFCF80910E0590910F0591836C
:10457000808310920E0510920F0510921005109274
:104580001105C2CF2FEF3FEF452B31F089B7806186
:1045900089BF02C020E030E0C90108951F920F9248
:1045A0000FB60F9211242F933F934F935F936F9306
:1045B0007F938F939F93AF93BF93EF93FF938EE07F
:1045C00095E00E940546FF91EF91BF91AF919F91B9
:1045D0008F917F916F915F914F913F912F910F90AC
:1045E0000FBE0F901F9018959C01FB0187B7482FB5
:1045F00055274072507087B78F7D87BF21313105B5
:1046000071F1223131054CF421303105A1F0203116
:104610003105A1F0232B69F009C02032310511F1D9
:104620002036310521F122313105B9F12FEF3FEF6D
:104630002EC040E050E080E286BF27C006B605FEEF
:1046400005C081E090E09183808302C011821082D6
:10465000452B19F18081918180689183808320E0CE
:1046600030E017C08AE090E0918380830EC0809193
:104670001805909119059183808310921805109266
:10468000190510921A0510921B0520E030E0452B09
:1046900031F087B7806287BF02C020E030E0C901F7
:1046A00008951F920F920FB60F9211242F933F93EC
:1046B0004F935F936F937F938F939F93AF93BF932A
:1046C000EF93FF9388E195E00E940546FF91EF91FB
:1046D000BF91AF919F918F917F916F915F914F911A
:1046E0003F912F910F900FBE0F901F9018959C0136
:1046F000FB0180917D00482F5527487050708091B4
:104700007D00877F80937D002131310581F1223149
:1047100031054CF421303105A1F020313105A9F0EB
:10472000232B69F009C02032310521F120363105F3
:1047300031F122313105D9F12FEF3FEF30C040E0A8
:1047400050E088E080937C0028C080917C0083FF4B
:1047500005C081E090E09183808302C011821082C5
:10476000452B29F18081918180689183808320E0AD
:1047700030E017C08BE090E0918380830EC0809181
:104780002205909123059183808310922205109237
:104790002305109224051092250520E030E0452BDA
:1047A00041F080917D00886080937D0002C020E010
:1047B00030E0C90108951F920F920FB60F92112495
:1047C0002F933F934F935F936F937F938F939F9319
:1047D000AF93BF93EF93FF9382E295E00E9405466B
:1047E000FF91EF91BF91AF919F918F917F916F91C9
:1047F0005F914F913F912F910F900FBE0F901F909F
:104800001895559A89B78F7E89BF0895CF93DF9306
:10481000DC01EC01EA81FB812091EE07422F552754
:10482000CA0180739070892B89F044FF04C083E132
:104830008CB9206403C081E18CB92F7B2093EE07F3
:104840008091EE078F7C8093EE0755C027FF02C052
:10485000559851C0ED018A859B85892BB1F18091D6
:10486000F107882339F00C9B05C0559889B7806102
:1048700089BF41C0ED018A859B8501979B878A8707
:104880008091EF07882311F0509A01C050988191D0
:104890008CB99F01FD01868197812817390711F492
:1048A00024813581ED013B832A832A853B858C85D4
:1048B0009D8528173907F9F4E889F989309769F057
:1048C0008FEFEF3FF807B9F011C05598ED011B8647
:1048D0001A86E889F989309729F48FEF9FEF998B31
:1048E000888B09C08FEFEF3FF80729F0848195810D
:1048F000019695838483DF91CF910895CF93DF93C1
:10490000DC013BB18091ED07382B3093ED076CB1A2
:104910002091EE07222361F0633119F45598206845
:1049200004C0613129F4559A2F772093EE075DC0BA
:10493000ED014A855B85888599854817590720F0E0
:1049400038603093ED0751C04F5F5F4F41305105E4
:10495000A1F4ED01E889F989309729F48FEF9FEFF1
:10496000998B888B2AC08FEFEF3FF80731F1848154
:10497000958101969583848320C0222399F0ED01CF
:104980008E859F8548175907C0F026FD16C05D9B90
:1049900005C083E18CB920642F7D01C02062209383
:1049A000EE070BC08091F007882339F0FD01868562
:1049B00097854817590708F01A9AED91FC911197BD
:1049C00061931196FC93EE932D913C911197ED011B
:1049D0008E819F812817390729F48C819D8111963A
:1049E0009C938E93FD0153874287DF91CF91089569
:1049F000529B03C089E090E008958091950082FF6A
:104A00000AC08091950081FF03C088E090E008957E
:104A100087E090E008958091950081FF03C086E0D3
:104A200090E0089585E090E008958091950085FDDF
:104A300003C080E090E008958091950084FF03C05A
:104A400081E090E0089582E090E0089580919500E3
:104A500083FF03C082E090E0089581E090E0089534
:104A6000EF92FF920F931F938091ED07682F7727A6
:104A7000CB0174E0969587957A95E1F79C014427E0
:104A80005527217030704070507063FD226062FDC8
:104A900024608091EE07882321F086FD426087FD27
:104AA00048601A9B14C0E12C62E0F62E012D112DF6
:104AB000E22AF32A042B152B8091F007882381F03A
:104AC000E12C92E0F92E92E0092F112D05C0E12C86
:104AD00081E0F82E012D112DE22AF32A042B152B4B
:104AE0000C9B0CC0A801970138608091F1078823C6
:104AF00041F0A80197013860426003C0A801970106
:104B0000346041FF416043FF44608091EF07882398
:104B100021F0CA01B901806403C0CA01B9018068EB
:104B2000589B02C0806101C080621F910F91FF906D
:104B3000EF900895EF92FF920F931F937B018C01EA
:104B40008091EE078823D9F00FB6F8940F9200FFFA
:104B500002C08F7B03C001FF03C080648093EE0717
:104B600002FF04C08091EE078F7705C003FF05C0E8
:104B70008091EE0780688093EE070F900FBE8091C2
:104B8000F007882321F001FD1A9A00FD1A98F1FC24
:104B90001A9AF0FC1A9806FF03C081E08093EF0791
:104BA00007FF02C01092EF0704FD589A05FD5898C0
:104BB000E0FE05C08091ED078F7E8093ED07E1FE5A
:104BC00005C08091ED07877F8093ED07E2FE05C069
:104BD0008091ED078B7F8093ED070E943025687FE1
:104BE0006E157F058007910719F08FEF9FEF02C0C8
:104BF00080E090E01F910F91FF90EF9008958091D9
:104C0000950086FF0BC0129B02C093E001C091E0AB
:104C10008091950080FF07C0946005C0599B02C039
:104C200090E201C090E0892F992708958091EE07C6
:104C3000882329F020E230E040E050E004C020E08A
:104C400030E040E050E08091F007882311F02160CF
:104C500001C02E7F8091F107882321F0CA01B9019C
:104C600062600895CA01B9016D7F0895559A08954B
:104C70009091EE079923A9F096FF13C00FB6F89410
:104C80000F925D9B04C081E18CB99F7E01C0906151
:104C90009093EE078091EE078F798093EE070F9047
:104CA0000FBE8091F00781111A9808950FB6F894FD
:104CB0000F925798569855980F900FBE8AE00E9411
:104CC00098115498539808951F93182F0E945626B0
:104CD0005298809195008D7F8093950080919500EA
:104CE0008B7F809395001730A1F0183018F41630A0
:104CF000A9F405C0183041F0193081F404C0809146
:104D00009500826009C0529A8091950082608093DC
:104D10009500809195008460809395000FB6F8947B
:104D20000F9288EB8AB90F900FBE0E94F82481176A
:104D300019F08FEF9FEF02C080E090E01F9108957F
:104D40008F929F92AF92BF92CF92DF92EF92FF929B
:104D50000F931F9389B0909090008091950086FFEB
:104D600006C0B2E0AB2EB12CC12CD12C0DC0599B8A
:104D700006C0A8E0AA2EB12CC12CD12C05C0F0E1B0
:104D8000AF2EB12CC12CD12C0E94B0117B018C0113
:104D9000282D3327892D9927982F8827282B392BC1
:104DA000442755272F5F3F4F4F4F5F4FC601B50137
:104DB0000E945A7A9B01AC01C801B7010E94AC7AEB
:104DC000CA01B9011F910F91FF90EF90DF90CF9032
:104DD000BF90AF909F908F90089540E050E060E0CA
:104DE00070E088E794E00E941B4640E050E060E0FD
:104DF00070E088EC94E00E941B468091F1078823C4
:104E000059F01092F107149840E050E060E070E033
:104E10008EE095E00E941B468091F007882319F0F0
:104E20001092F007129880E090E0089541E755E075
:104E30006EE774E288E794E00E941B46892B19F024
:104E40008FEF9FEF08954FE555E066E074E288EC40
:104E500094E00E941B46892B19F480E090E00895AD
:104E600040E050E060E070E088E794E00E941B467C
:104E70008FEF9FEF0895EF92FF920F931F937B01A7
:104E80008C0165FF0BC08091EE07882371F40FB68B
:104E9000F8940F9281E48093EE0705C00FB6F89462
:104EA0000F921092EE070F900FBEE0FE06C01A9A06
:104EB000129A81E08093F00707C08091F007882361
:104EC00019F01092F0071298E1FE10C040E050E097
:104ED00061E074E28EE095E00E941B46892BF9F4B4
:104EE0001C9A149881E08093F1070FC08091F1071C
:104EF000882359F01092F10740E050E060E070E044
:104F00008EE095E00E941B4614980E9416266E15AE
:104F10007F058007910719F480E090E002C08FEFD1
:104F20009FEF1F910F91FF90EF900895EF92FF92E6
:104F30000F931F937B018C010E9456268091950050
:104F400086FD11C0599B08C092E0EE0CFF1C001FAB
:104F5000111F9A95D1F707C083E0EE0CFF1C001FCC
:104F6000111F8A95D1F70E94B011A80197010E94E4
:104F7000AC7A2F5F3F4F4F4F5F4F56954795379510
:104F800027952150304029B9232F332720939000B3
:104F90000FB6F8940F9288EB8AB90F900FBE80E09D
:104FA00090E01F910F91FF90EF9008951F93182F9D
:104FB0000E945626812F992780FF13C081FF02C0CF
:104FC000129A01C0129882FF04C0809195008160FE
:104FD00003C0809195008E7F8093950059985E9ACA
:104FE0000FC085FF02C0599A01C059988091950061
:104FF0008E7F80939500809195008F7B80939500A4
:105000000FB6F8940F9288EB8AB90F900FBE0E94EA
:10501000FF25811719F08FEF9FEF02C080E090E02D
:105020001F9108951F93182F0E945626113071F07A
:10503000113018F01230C1F40DC0809195008F7EB0
:1050400080939500809195008F7D0CC08091950094
:10505000806103C0809195008F7E80939500809140
:1050600095008062809395000FB6F8940F9288EBBC
:105070008AB90F900FBE0E941525811719F08FEF86
:105080009FEF02C080E090E01F9108951F93182FBA
:105090000E945626113021F480919500877F05C02B
:1050A000123029F4809195008860809395000FB6A6
:1050B000F8940F9288EB8AB90F900FBE80919500FB
:1050C00083FF03C082E090E002C081E090E0181707
:1050D00019F08FEF9FEF02C080E090E01F910895DC
:1050E000CF93DF93DC01EB01FC0192A180A1891732
:1050F00019F481E090E013C0892F9927FC01EE0F8D
:10510000FF1FEA0FFB1F208131813983288301961D
:105110008F709070FD0193A382A380E090E0DF91F7
:10512000CF910895CF92DF92EF92FF920F931F934A
:10513000CF93DF938C017B01EC0188A1E82FFF273F
:105140006F010894C11CD11CC60160E170E00E948F
:10515000997A2AA133278217930719F481E090E006
:1051600011C0EE0FFF1FE00FF11FD7018D919C9131
:1051700091838083BFE0CB22DD24E801D9A2C8A2BD
:1051800080E090E0DF91CF911F910F91FF90EF9021
:10519000DF90CF900895FC0111A210A213A212A2D9
:1051A0000895CF93DF93CDB7DEB722970FB6F8946B
:1051B000DEBF0FBECDBF84B195B19A838983BE0196
:1051C0006F5F7F4F8091F4079091F5070E949228BE
:1051D00022960FB6F894DEBF0FBECDBFDF91CF9100
:1051E000089597B1987F982B97B90895369A0895A6
:1051F0008091F2079091F307019719F43798369848
:10520000379A08951F93182F0E94F828113840F5F7
:105210001430D1F0153038F4123071F0133090F4AE
:10522000112341F01DC01630A9F0163080F0173060
:10523000B9F412C0329809C03298319A309880E09F
:1052400090E010C0329809C0329A3198F7CF329A64
:10525000319804C0329AF1CF329A319A309AEFCF16
:1052600081E090E01F910895CF93DF93EC010E94BD
:10527000F828C130D10521F0C230D10521F402C097
:10528000359A01C03598D093F307C093F207DF91A8
:10529000CF91089582E090E00E94342925B785B728
:1052A000837E9091A805892B85BF85B7806285BFD5
:1052B000889585B78F7D85BF85B7837E2C71822BBE
:1052C00085BF0895CF93DF93EC010E94F828C13089
:1052D000D10541F0C130D10518F0229741F405C045
:1052E0003F9804C03F983E9802C03F9A3E9ADF9193
:1052F000CF910895BC018091F4079091F5070E9429
:105300007028992708958091F2079091F3070895E6
:10531000E091F407F091F50711A210A213A212A2D6
:1053200008958091F4079091F507892B39F587B19D
:10533000887F87B980E090E00E94622982E090E057
:105340000E94342986E00E94022982E290E00E94B5
:10535000000CFC019093F5078093F40711A210A2B2
:1053600013A212A240E050E061ED78E286EF93E0F4
:105370000E941B46892B11F4379A339A0895CF93D4
:10538000DF93EA019C0140E050E0FB0110C0D9012D
:105390000E94087B802D9081981721F0D901092E59
:1053A0000E94107B4F5F5F4F31962F5F3F4F4C172E
:1053B0005D0769F780E090E0DF91CF910895CF938A
:1053C000DF93EA01DC01FB01219724F00E94087BB6
:1053D0000192FACF80E090E0DF91CF910895509153
:1053E000740040917100487F403609F41AC141367B
:1053F00070F5483209F473C0493298F4403109F429
:1054000057C0413138F4442309F4F5C1483009F05C
:1054100040C24EC0483109F462C0403209F039C27E
:1054200091C0403409F4B5C0413438F4403309F434
:1054300089C0483309F02DC292C0403509F493C0A9
:10544000483509F4B4C0483409F023C27BC0483958
:1054500009F42AC14939B0F4483709F4E2C04937A0
:1054600038F4483609F4DDC0403709F012C2D9C01B
:10547000483809F419C1403909F4E9C0403809F045
:1054800008C2E5C0403B09F44CC1413B38F4403A06
:1054900009F41EC1483A09F0FCC143C1403C09F47B
:1054A00080C1483C09F47DC1483B09F0F2C140C1CC
:1054B00081E08093F6071092FF071092FE0710928A
:1054C0000508109204088091FC079091FD07209137
:1054D000F707892B09F421602093730021C02091E4
:1054E000FE073091FF078091FC079091FD07281778
:1054F0003907D8F4E091FE07F091FF078091FA0791
:105500009091FB07E80FF91F8081809373008091D1
:10551000FE079091FF0701969093FF078093FE0787
:10552000507455685093740008951092FD071092BE
:10553000FC078091020890910308892B19F05074A0
:10554000556AF0CF403219F0483409F04AC084E07F
:105550008093F8071092FD071092FC073EC08091DF
:105560007400806243C1E0910408F09105088091C5
:10557000000890910108E80FF91F80917300808363
:1055800080910408909105080196909305088093F6
:105590000408809104089091050820910208309138
:1055A000030801968217930708F4EEC0F6C0E09155
:1055B0000408F09105088091000890910108E80F17
:1055C000F91F8091730080838091040890910508F1
:1055D0000196909305088093040810920308109296
:1055E0000208E0916408F0916508309739F48FEF74
:1055F0009FEF909365088093640809C08FEFEF3F99
:10560000F80729F0848195810196958384838091A0
:10561000110890911208892B11F085EDE7C085E9FA
:10562000E5C08091110890911208892B09F4B5C04A
:1056300081E08093F607809173008093060885ECE3
:10564000809374001092140810921308089520910A
:1056500013083091140880911108909112082817AE
:105660003907B8F4E0911308F091140880910F08FD
:1056700090911008E80FF91F80917300808380914A
:1056800013089091140801969093140880931308BE
:1056900004C0109212081092110880911108909184
:1056A0001208892B09F070C08091FC079091FD07CA
:1056B000892B31F48091020890910308892B21F005
:1056C0008091740080666AC080917400806466C0B6
:1056D000E0916608F0916708309721F08091070803
:1056E000882381F08091FC079091FD07892B31F48C
:1056F0008091020890910308892B11F085EA76C009
:1057000085E874C08FEFEF3FF80729F08481958119
:1057100001969583848310921208109211085E7787
:1057200001CF81E08093F60710920E0810920D08C9
:1057300020910D0830910E0880910B0890910C0873
:105740002817390740F5E0910D08F0910E08809177
:10575000090890910A08E80FF91F8081809373006F
:1057600080910D0890910E08019690930E088093F9
:105770000D0820910D0830910E0880910B08909132
:105780000C082817390710F485EC08C010920C0893
:1057900010920B0802C01092730085E88093740089
:1057A0000895E0916808F0916908309739F48FEF17
:1057B0009FEF909369088093680809C08FEFEF3FCF
:1057C000F80729F0848195810196958384838091DF
:1057D000FC079091FD07892B31F48091020890918C
:1057E0000308892B11F085EE01C085EC80937400CD
:1057F0001092F60708958091740080618093740080
:105800001092F60782E08093F80780930708E091F2
:105810006608F0916708309739F48FEF9FEF909307
:1058200067088093660809C08FEFEF3FF80729F0FB
:1058300084819581019695838483E0916808F09135
:105840006908309739F48FEF9FEF90936908809340
:10585000680809C08FEFEF3FF80729F08481958130
:10586000019695838483E0916408F09165083097F0
:1058700039F48FEF9FEF9093650880936408089543
:105880008FEFEF3FF80729F084819581019695838A
:10589000848308958091F9071092F9079927089554
:1058A000809108081092080899270895AF92BF9236
:1058B000CF92DF92EF92FF920F931F93CF93DF93DC
:1058C000EB0124E083309207B9F024E084309207A2
:1058D0004CF424E081309207D9F08250944009F0D2
:1058E000AAC073C024E08430920771F089509440BC
:1058F000029708F0A0C005C08881880F816080935E
:10590000720080E090E099C0809172008883F9CFA6
:105910000E94B011660F771F881F991F2881398157
:105920004A815B810E94AC7A2F5F3F4F4F4F5F4FA0
:105930005695479537952795205130404040504027
:1059400079018A0116950795F794E7948DEFE8168B
:1059500083E0F80680E0080780E0180768F0790126
:105960008A0145E016950795F794E7944A95D1F793
:1059700080917100826003C0809171008D7F80935F
:1059800071002FEFE216F1040105110561F058F0E6
:1059900032E016950795F794E7943A95D1F7809100
:1059A0007100816003C0809171008E7F80937100CF
:1059B000D801C7010A97A109B109863F9105A10540
:1059C000B105C8F5E09270009CCF8091710080FF16
:1059D00006C028E0A22EB12CC12CD12C05C092E02B
:1059E000A92EB12CC12CD12C8091710081FF07C050
:1059F00084E0AA0CBB1CCC1CDD1C8A95D1F70E944C
:105A0000B0117B018C01209170003327442755276A
:105A1000C601B5010E945A7A9B01AC01205F3F4F3D
:105A20004F4F5F4FC801B7010E94AC7A288339837A
:105A30004A835B8366CF8FEF9FEFDF91CF911F91FA
:105A40000F91FF90EF90DF90CF90BF90AF900895AF
:105A50001F93CF93DF93CDB7DEB724970FB6F8949B
:105A6000DEBF0FBECDBF182F80E699E0A0E0B0E00A
:105A700089839A83AB83BC8340E050E06FEE79E288
:105A80008AE594E00E941B46892B19F08FEF9FEF67
:105A900017C0110F116010937200BE016F5F7F4F2E
:105AA00081E094E00E94562C80E88093740085E0A9
:105AB0008093740082E698E00E94EA0F80E090E014
:105AC00024960FB6F894DEBF0FBECDBFDF91CF9105
:105AD0001F91089590930A088093090870930C0809
:105AE00060930B08672B09F437C00FB6F8940F9238
:105AF00080916808909169088F5F9F4F21F4109200
:105B000069081092680885EC809374000F900FBEAE
:105B1000BA01A90188E698E00E943D10892B19F08E
:105B200081E0809307080FB6F8940F9210920C084A
:105B300010920B0880910708882339F0809107089C
:105B4000809308088FEF9FEF04C080910D0890911B
:105B50000E080F900FBE08950FB6F8940F92809123
:105B60007400809171008091FC079091FD07892B52
:105B700031F48091020890910308892B11F085EA95
:105B800003C01092F60785E8809374000F900FBE53
:105B900080E090E008950F931F93CF93DF93EC0183
:105BA0000FB6F8940F921092070850931208409382
:105BB00011087093100860930F088091F6078823EE
:105BC000B1F480917100887F883F89F48091FC074F
:105BD0009091FD07892B31F4809102089091030880
:105BE000892B11F085E601C085E4809374008091D3
:105BF0006608909167088F5F9F4F21F410926708A5
:105C000010926608B901A80186E698E00E943D104E
:105C1000892B61F00FB6F8940F9281E0809307080A
:105C200010921208109211080F900FBE0F900FBE25
:105C300080910708882319F02FEF3FEF07C02091CC
:105C4000130830911408809106088883C901DF91F8
:105C5000CF911F910F9108956F927F928F929F9293
:105C6000BF92CF92DF92EF92FF920F931F93CF9349
:105C7000DF93B82E4B01EA01390144EF51E060E0B7
:105C800070E082E698E00E943D10892B81F083E06D
:105C90008093F80782E698E00E94EA0F0FEF1FEF6B
:105CA0006CC06FE370E080E090E00E94260A809173
:105CB000F6078823B1F70FB6F8940F92BB0CB09299
:105CC000F7071092F807D093FD07C093FC07909256
:105CD000FB078092FA071093030800930208709262
:105CE0000108609200088091F607882399F42091BA
:105CF000740080917100887F883F61F48091110861
:105D0000909112082071892B11F0256601C025623F
:105D10002093740080916408909165088F5F9F4F75
:105D200021F410926508109264080F900FBEB7011D
:105D3000A60184E698E00E943D10892B31F081E0B5
:105D40008093F9070FEF1FEF14C00FB6F8940F926E
:105D50008091F807882339F08091F8078093F9073C
:105D60000FEF1FEF04C000910408109105080F9079
:105D70000FBE82E698E00E94EA0FC801DF91CF9142
:105D80001F910F91FF90EF90DF90CF90BF909F9069
:105D90008F907F906F900895FC018081918108958C
:105DA000CF92DF92EF92FF920F931F93CF93DF93E7
:105DB0006C01CB010E94DB307C018F5F9F4F71F43F
:105DC00040C00F5F1F4F32960830110559F487E12C
:105DD00090E090938B0880938A0833C003E010E032
:105DE000EFEAF5E080819181892B59F787E090E017
:105DF0000E945030EC01000F111F07551A4FD801B7
:105E0000CD93DC932097E9F0B701C6010E94E22F01
:105E100099838883D801ED91FC918F5F9F4F39F46E
:105E2000CF010E944D30F801118210820AC0F38226
:105E3000E2821482D801ED91FC9116821582CF0185
:105E400002C080E090E0DF91CF911F910F91FF9011
:105E5000EF90DF90CF9008950F931F93CF93DF9330
:105E6000CDB7DEB721970FB6F894DEBF0FBECDBF1A
:105E70008C01FB01898341E050E0BE016F5F7F4FE1
:105E8000808191810E943A30019711F00FEF1FEF4E
:105E9000C80121960FB6F894DEBF0FBECDBFDF91CB
:105EA000CF911F910F910895FC01CB01DF010D905F
:105EB0000020E9F71197AE1BBF0BAD01BF01FC013C
:105EC000808191810E943A3008959F92AF92BF9253
:105ED000CF92DF92EF92FF920F931F93CF93DF93B6
:105EE0005C01CB01EA010E94DB306C018F5F9F4FA8
:105EF00071F448C00F5F1F4F32960830110559F4F6
:105F000089E090E090938B0880938A083BC000E082
:105F100010E0E9EAF5E0808191818C179D0751F747
:105F200087E090E00E9450307C01E801CC0FDD1F3B
:105F3000C755DA4FF982E882E114F10419F1B6018C
:105F4000C5010E94E22FF70191838083E881F981E6
:105F50008F5F9F4F71F4CF010E944D3082E0801718
:105F600028F00F5F1F4F198308830CC01982188215
:105F700009C0D382C2821482E881F9811682158217
:105F8000CF0102C080E090E0DF91CF911F910F918F
:105F9000FF90EF90DF90CF90BF90AF909F900895CB
:105FA000CF93DF93EC01AA81BB81109719F4EB85A5
:105FB000FC8504C0ED01ED89FE89CD010995DF91D5
:105FC000CF910895EF92FF920F931F93CF93DF939A
:105FD000CDB7DEB729970FB6F894DEBF0FBECDBFA1
:105FE0007B018C01FE013196AE01475F5F4F03C01C
:105FF00021930F5F1F4F302F381BD8012C91222384
:1060000029F02A3319F0E417F50791F7CE0101962C
:10601000FC01E30FF11D10820E94A807DC01892B0F
:1060200049F482E090E090938B0880938A088FEF88
:106030009FEF13C0F80180818A3319F060E070E0AF
:1060400003C0B8016F5F7F4FFD01058D168D20E005
:1060500030E0A701CD01F801099529960FB6F89413
:10606000DEBF0FBECDBFDF91CF911F910F91FF908B
:10607000EF900895CF93DF93DC01EC01EA81FB817F
:10608000309719F4EF81F88503C0018CF28DE02D73
:10609000CD010995DF91CF9108950E94730C089569
:1060A0000E94000C9C01892B31F48CE090E09093CD
:1060B0008B0880938A08C9010895CF93DF93CDB7E9
:1060C000DEB722970FB6F894DEBF0FBECDBFAE018C
:1060D000455F5F4F5A83498369857A858F819885AB
:1060E0000E948F3022960FB6F894DEBF0FBECDBF50
:1060F000DF91CF910895EF92FF920F931F938C0140
:106100007B010E94FF79AC01B801F7018081918188
:106110000E94C8301F910F91FF90EF900895AF92A9
:10612000BF92CF92DF92EF92FF920F931F93CF9384
:10613000DF935C017B016A01CB010E94FF798C0136
:106140000F5F1F4FC8010E94000CEC01009719F46B
:106150000FEF1FEF11C0A801B7010E94EB79F50105
:10616000608171819601AE018AE390E30E942F3134
:106170008C01CE010E94730CC801DF91CF911F9159
:106180000F91FF90EF90DF90CF90BF90AF90089568
:10619000CF93DF93DC01EC01EA81FB81309719F4A6
:1061A000E985FA8503C0038CF48DE02DCD010995B6
:1061B000DF91CF910895FC018081823759F08737B4
:1061C00019F08136B1F403C081E093E41BC088E08C
:1061D00091E418C080E090E415C02B3219F022360B
:1061E00041F404C08E7F826093600CC09F7B9068F6
:1061F00009C086E190E090938B0880938A088FEF26
:106200009FEF089531962081222339F70895CF9288
:10621000DF92EF92FF920F931F93CF93DF936C0166
:106220007B018A01E90107C040E150E0B801C701E4
:10623000F60109956097C131D105B4F71C161D060A
:106240002CF4AE01B801C701F6010995DF91CF9199
:106250001F910F91FF90EF90DF90CF9008952F92B4
:106260003F924F925F926F927F928F929F92AF92E6
:10627000BF92CF92DF92EF92FF920F931F93CF9333
:10628000DF93CDB7DEB76B970FB6F894DEBF0FBEC6
:10629000CDBF998F888F7B8F6A8F1A0159011D8A14
:1062A0001C8AB10103C00894211C311CD101FC904F
:1062B000FF2019F0B5E2FB16B1F78101061B170BA1
:1062C00061F0A8018A8D9B8DE88DF98D09952C8947
:1062D0003D89200F311F3D8B2C8BFF2009F4E6C236
:1062E000F1013196198266241B8A1A8A4FEF442ED7
:1062F000542E02C05C01F101DF019D901D01B0E24E
:106300009B1621F489818823B1F703C02BE29216F2
:1063100011F49982F0CF3DE2931619F444E0642A17
:10632000EACF53E2951619F461E0662AE4CF70E3F0
:10633000971619F480E1682ADECF9CE6991619F4C5
:10634000A8E06A2AD8CFBAE79B16A9F22AE29216E9
:1063500091F4C5010296D501AD90BC90BB8AAA8A82
:10636000B7FEC8CFB4E06B2AF501F095E195FF4F79
:10637000FB8BEA8BBFCF2EE2921691F581818A3298
:1063800019F0442455241FC00894211C311CD50148
:106390004D905C90E2E0F0E0AE0EBF1E1BC08AE0C4
:1063A00090E0A201489F2001499F500C589F500C3B
:1063B0001124822F992787FD9095480E591E60ED74
:1063C0007FEF460E571E21813196822F80538A30EF
:1063D00030F31F0157FE8FCF3FEF432E532E8BCF4D
:1063E000892D8153893010F5892D9927C0979B8B72
:1063F0008A8B2AE030E012C04A895B89429FD00133
:10640000439FB00D529FB00D1124892F992787FD0E
:106410009095A80FB91FD097BB8BAA8B918131960D
:10642000892F80538A3040F31F0165CFF501792C05
:1064300057E65915E8F065E6961608F09FC170E535
:106440009716D1F1791548F085E4981609F496C1AC
:1064500097E4991609F096C191C1A3E69A1621F125
:10646000A91508F472C0B8E59B1609F08BC128C1C4
:1064700020E7921609F424C1291548F039E693164D
:1064800009F463C04FE6941609F07CC1CDC055E70E
:10649000951609F459C068E7961609F411C173E717
:1064A000971609F06FC124C082E090E0A80EB91ED3
:1064B00080818A8319826CC1A2E0B0E0AA0EBB1E63
:1064C000E080F180E114F10439F429EBC22E25E0DB
:1064D000D22E93E7792E19C0C7010E94FF79019649
:1064E0000E9450308C01B7010E94F879680106C003
:1064F00022E030E0A20EB31EC080D180C114D104CE
:1065000021F489EBC82E85E0D82E57FC12C0A201D9
:1065100060E070E0C6010E94087A009711F48201E1
:1065200011C08C199D098201841595055CF48C01BC
:1065300009C0D6010D900020E9F78D0101501040EF
:106540000C191D091982AAC1198263FE0CC024E02E
:1065500030E0A20EB31EE080F1800281138135E7A6
:106560009316B1F421C0D5011296F5010081118175
:10657000F5E79F1631F45D01980179010027112795
:1065800013C05D01A8017A010027F7FC0095102FC8
:1065900017FF0AC010950095F094E094E11CF11CDF
:1065A000011D111D8DE2898357FC02C05FEE65223B
:1065B000E114F1040105110539F44114510451F4B9
:1065C00002E1C02ED12C0CC06AE0E616F1040105F0
:1065D000110548F48E2D805D898B11E1C12ED12CDF
:1065E000CC0EDD1EC4C0B2E1CB2ED12CCC0EDD1EF4
:1065F000C801B7012AE030E040E050E00E94AC7AE8
:10660000605DD6016E936D01C801B7012AE030E0EC
:1066100040E050E00E94AC7A79018A0121153105F1
:106620004105510529F7A3C063FE09C024E030E00D
:10663000A20EB31E008111812281338109C042E084
:1066400050E0A40EB51E808191818C012227332752
:10665000198257FC02C05FEE652201151105210564
:10666000310549F44114510431F4A2E1CA2ED12C70
:10667000CC0EDD1E1FC0F2E1CF2ED12CCC0EDD1EC4
:10668000802F8770805DD6018E936D01E3E0369593
:10669000279517950795EA95D1F70115110521055D
:1066A000310571F760FE06C0803321F080E3FD0103
:1066B00082936F018E010C191D090E5E1F4F70C071
:1066C00020E7921671F442E050E0A40EB51E8081DE
:1066D00091818C012227332751E0652A78E7972E94
:1066E00014C063FE09C064E070E0A60EB71E00810E
:1066F00011812281338109C082E090E0A80EB91E89
:10670000808191818C012227332757FC02C09FEEA4
:106710006922A8E59A1619F040EC55E002C041ED57
:1067200055E0198262E1C62ED12CCC0EDD1EF80197
:10673000EF70F070E40FF51F8081F60182936F0116
:1067400094E036952795179507959A95D1F70115F9
:1067500011052105310559F760FE09C03197908276
:106760006F010894C108D10880E3D6018C938E0193
:106770000C191D090E5E1F4F792C12C0E4E0F0E0E9
:10678000AE0EBF1E992009F491C09A821982792C0D
:1067900082E0C82ED12CCC0EDD1E01E010E07EC0C0
:1067A0007801041515050CF472018981882319F00C
:1067B0000894E11CF11C4201262D33273F8B2E8BC0
:1067C000290134E1432255244114510461F42A89FA
:1067D0003B892E193F0942EE55E06A8D7B8D888DED
:1067E000998D0E9407318981882359F041E050E05A
:1067F000BE016F5F7F4F8A8D9B8DA88DB98DFD0186
:106800000995B0E14B16510461F42A893B892E1990
:106810003F0942EF55E06A8D7B8D888D998D0E94EE
:106820000731801A910A940142EF55E06A8D7B8D01
:10683000888D998D0E9407310115110539F0A80145
:10684000B6018A8D9B8DE88DF98D0995F0E57F164F
:1068500019F4C6010E944D302E8922FF0CC02A89EE
:106860003B892E193F0942EE55E06A8D7B8D888D5C
:10687000998D0E9407314A895B894E155F053CF06E
:106880006C897D89640F751F7D8B6C8B0ACD8C891B
:106890009D898E0D9F1D9D8B8C8B03CD780117FFDD
:1068A00002C0EE24FF248824992486CF8C899D89F8
:1068B0006B960FB6F894DEBF0FBECDBFDF91CF91C0
:1068C0001F910F91FF90EF90DF90CF90BF90AF900E
:1068D0009F908F907F906F905F904F903F902F9000
:1068E00008950F931F9300E010E023E030E046E0AE
:1068F00050E060E070E080E090E00E94EE3890931D
:1069000017088093160881E0809315081F910F9156
:1069100008956F927F928F929F92AF92BF92CF9283
:10692000DF92EF92FF920F931F93CF93DF93CDB738
:10693000DEB7C456D0400FB6F894DEBF0FBECDBF51
:1069400080911508882311F40E9471348E010F5F25
:106950001F4F80911608909117080E940639F80180
:10696000819391938F010E94E80BCE018B599F4F29
:106970000817190771F720E030E040E050E0FE0111
:106980003196B80181919191AA27BB27280F391F11
:106990004A1F5B1FE617F707A9F7CA01B90122E3EF
:1069A00030E040E050E00E94CE7A49015A01CA012D
:1069B000B90128EC39E140E050E00E945A7A2AE01F
:1069C00095958795779567952A95D1F7645F71407E
:1069D000804090405CF1EE24FF2487016E01089412
:1069E000C11CD11C85E6682E712C6C0E7D1EF60133
:1069F000819191916F01AA27BB27A5019401281BC2
:106A0000390B4A0B5B0BCA01B9010E945A7AE60E98
:106A1000F71E081F191FC614D70449F780E090E03D
:106A2000F2E3EF16F1040105110514F481E090E0A2
:106A3000CC59DF4F0FB6F894DEBF0FBECDBFDF914C
:106A4000CF911F910F91FF90EF90DF90CF90BF906B
:106A5000AF909F908F907F906F900895CF92DF922C
:106A6000EF92FF920F931F93CF93DF93EC010E945D
:106A70007134CE010A978B35910510F0CAE0D0E051
:106A8000CC24DD24EE24FF24870111C08091160858
:106A9000909117080E940639AA27BB27E80EF91E15
:106AA0000A1F1B1F0E94E80B0894C11CD11CCC16A6
:106AB000DD0664F3C801B70128EC39E140E050E09D
:106AC0000E945A7A9E01442737FD4095542F0E9418
:106AD000CE7ADA01C9013AE0B595A79597958795E1
:106AE0003A95D1F7DF91CF911F910F91FF90EF90E1
:106AF000DF90CF900895089584B7806884BF84BFE5
:106B0000089584B78F7784BF84BF0895EAE9F0E0E1
:106B10008081877F80838B9893988A9892988C98AD
:106B2000949815981D98A1E6B0E08C918F7B8C937A
:106B3000E2E6F0E080818F7B80838C918F7D8C9367
:106B400080818F7D80838C918F7E8C9380818F7EDE
:106B500080830895EAE9F0E08081886080838B9AE1
:106B6000939A8A98929A8C9A15980895882321F07E
:106B700084E00E943736089584E00E9444360895E8
:106B8000882321F085E00E943736089585E00E9431
:106B900044360895882321F087E00E944436089502
:106BA00087E00E9437360895189A939A8B9A80E06E
:106BB0000E947C070895882321F086E00E943736E2
:106BC00003C086E00E94443682E096E00E9486354B
:106BD00084B7806884BF84BF08950F931F9302E039
:106BE00016E0C8010E94863584B7806884BF84BFE0
:106BF00080E00E94DB3581E00E94CA3568EE73E0D8
:106C000080E090E00E94260A81E00E94DB3564EF7C
:106C100071E080E090E00E94260A80E00E94CA3580
:106C200084B78F7784BF84BFC8010E94AA3560ED06
:106C300077E080E090E00E94260A1F910F9108956E
:106C40000FB6F8940F92E82FFF27FE2FEE279081C2
:106C50009083C59A0000C5980F900FBE80931808C6
:106C60000895BD9A809118080E942036089521E069
:106C700030E002C0220F331F8A95E2F78091180896
:106C8000822B0E942036089521E030E002C0220FBE
:106C9000331F8A95E2F720958091180882230E947D
:106CA00020360895A0918208BB27FD01EE0FFF1F3B
:106CB000EE0FFF1FE459F74F8083618342832383E4
:106CC000CD01019665E070E00E94997A282F8093AB
:106CD000820880916B08281749F4822F9927019622
:106CE00065E070E00E94997A80936B080895809324
:106CF0000706609319084093080608951F93182FFC
:106D000080918008882319F4812F0E944C4981E0EA
:106D100090E002C0880F991F1A95E2F780952091A4
:106D20006A08282320936A081F9108951F93182F3B
:106D300080918008882319F4812F0E945A4981E0AC
:106D400090E002C0880F991F1A95E2F720916A0817
:106D5000282B20936A081F910895CF93DF93C82FA3
:106D6000DD27C0FF04C080E00E945A4903C080E0D4
:106D70000E944C49C1FF04C081E00E945A4903C0EF
:106D800081E00E944C49C2FF04C082E00E945A493F
:106D900003C082E00E944C49C3FF04C083E00E940C
:106DA0005A4903C083E00E944C49DF91CF91089576
:106DB000CF93DF93C0E0D0E080916A0899270C2E32
:106DC00002C0959587950A94E2F780FF04C08C2F46
:106DD0000E945A4903C08C2F0E944C492196C4300E
:106DE000D10551F7DF91CF9108958091820880936A
:106DF0006B080E94D8361092800808951F93182FB0
:106E00000E9468491092820810926B08112351F079
:106E100020E034E040E050E064E177E383E096E096
:106E20000E9404111F91089586E90E94640BE0916D
:106E30006B0880918208E81719F41092800845C009
:106E4000FF27EE0FFF1FEE0FFF1FE459F74F808162
:106E50008093800800E010E0802F0E944C490F5F73
:106E60001F4F04301105C1F780916B08A82FBB2775
:106E7000FD01EE0FFF1FEE0FFF1FE459F74F838157
:106E80008F3F11F08150838312818091800884307C
:106E900009F469C0853060F4813009F449C081305B
:106EA000A0F0823009F452C0833009F062C187C07B
:106EB000863009F4CEC0863008F4A3C0873009F4C8
:106EC000F9C0883009F055C127C180910806882390
:106ED00029F10E94B54020910706EFE32E9F900113
:106EE0001124442755270E94AC7A6F337105810520
:106EF0009105A0F460911908662321F021E04091EA
:106F0000080607C080916A08882331F421E041E037
:106F100061E084E00E9452361092810880918108DD
:106F20008F5F809381086FE370E080E090E00BC09A
:106F300081810E94AD366FE3169FB001112488272E
:106F400077FD8095982F0E94260A1BC181810E949F
:106F5000AD368FE3189FC00111247C010027F7FC98
:106F60000095102F21C080E00E94AD368FE3189F5E
:106F7000C00111247C010027F7FC0095102FC801E7
:106F8000B7010E94260A80918008882309F44FCF18
:106F9000E0916B08FF27EE0FFF1FEE0FFF1FE45974
:106FA000F74F81810E94AD36C801B7010E94260AC1
:106FB00080918008882309F43ACF80E01FC080E0E8
:106FC0000E94AD368FE3189FC00111247C01002779
:106FD000F7FC0095102FC801B7010E94260A809186
:106FE0008008882309F423CFE0916B08FF27EE0F78
:106FF000FF1FEE0FFF1FE459F74F81810E94AD364E
:10700000B5C080E00E945A49C12FDD278FE390E090
:107010009C01C29FC001C39F900DD29F900D11246F
:107020007C010027F7FC0095102FDD24C801B70173
:107030000E94260A80918008882391F18D2D0E945C
:107040004C49D3948D2D0E945A4933E0D31671F7E1
:1070500027C083E00E945A49C12FDD278FE390E0CB
:10706000FC01CE9FC001CF9F900DDE9F900D11249B
:107070007C010027F7FC0095102F63E0D62EC80195
:10708000B7010E94260A80918008882349F08D2D3F
:107090000E944C49DA948D2D0E945A49DD2079F7DF
:1070A0008FE390E0C89FB001C99F700DD89F700D0D
:1070B000112445CF80E00E945A498FE3189FC001F8
:1070C00011246C01EE24D7FCE094FE2C10E0C701E3
:1070D000B6010E94260A80918008882349F0812FFA
:1070E0000E944C491F5F812F0E945A49133079F743
:1070F00013E0C701B6010E94260A80918008882308
:1071000009F495CE812F0E944C491150812F0E9485
:107110005A491123B1F1EDCF80E00E945A4981E034
:107120000E945A4982E00E944C4983E00E944C49E7
:107130008FE3189FC00111247C010027F7FC009504
:10714000102FC801B7010E94260A80918008882369
:1071500009F46DCE80E00E944C4981E00E944C49C8
:1071600082E00E945A4983E00E945A49C801B7014F
:10717000EACEAA0FBB1FAA0FBB1FA459B74FFD0130
:10718000138280918008882309F451CE80916B0886
:10719000282F3327F901EE0FFF1FEE0FFF1FE459D1
:1071A000F74F8381882309F042CEC901019665E03B
:1071B00070E00E94997A2091820833278217930702
:1071C00011F40E94D83680916B089927019665E0EA
:1071D00070E00E94997A80936B0829CE0F931F93D9
:1071E000682B642B202B0FB6F8940F92379866B952
:1071F00027B9379A0F900FBE822F9927982F88278B
:107200007727862B972B1F910F910895AC01692F3B
:1072100077270FB6F8940F9287B126B1861719F425
:107220002F76241721F0379846B967B9379A369ADE
:107230003699FECF84B125B10F900FBE9927332721
:10724000322F2227822B932B08959C01E0918308F3
:10725000F0918408E657FD4F80819181EA58F24011
:107260008217930719F420E030E00EC0E157F94F80
:1072700080819181EF58F6408217930719F080E0E2
:1072800090E0089521E030E085E094E0AC01249F97
:10729000C001259F900D349F900D112486579D4F5E
:1072A0008E0F9F1F089580E090E00E942539FC0119
:1072B000892B19F481E090E0089580914308909122
:1072C000440891838083ED5FFB4F1182108280E040
:1072D00090E0089580914308909144080E942539D8
:1072E000FC01892B19F481E090E0089581E082830C
:1072F000ED5FFB4F1182108280E090E00895809155
:107300004308909144080E942539DC01892B19F427
:1073100080E090E00895AD5FBB4FED91FC91119737
:10732000A350B440EA0FFB1F1382FD011282CD016E
:10733000039608950F931F93DC01FC010190002038
:10734000E9F731970E2F081B043108F003E11127EC
:107350008091830890918408A801BD01805E924FBE
:107360000E944B7A8091830890918408080F191F1E
:10737000005E124FF80110821F910F9108958091C5
:107380008308909184088C5C924F0E94FC40089581
:1073900080918308909184088C5C924F0E941941DF
:1073A00008950F931F93CF93DF93CDB7DEB7229746
:1073B0000FB6F894DEBF0FBECDBF09851A85809148
:1073C0004308909144080E942539FC01892B71F0F3
:1073D0008281882359F09E01255F3F4F3A8329839C
:1073E000A801BF0187E19AE30E942F31CE010B96DD
:1073F0009A8389830E94C839AE01455F5F4F5A83E3
:107400004983B80180918508909186080E94F146D1
:107410008C010E94BF39C80122960FB6F894DEBFD6
:107420000FBECDBFDF91CF911F910F9108950F93A4
:107430001F93CF93DF938C010D5F1B4FF8012081C9
:107440003181CEEFD3E0C21BD30B4C175D0708F49C
:10745000EA010396AE01820F931F0E94157AF8018C
:10746000808191818C0F9D1F91838083CE01DF915C
:10747000CF911F910F910895EF92FF920F931F9359
:107480007C01062F80918308909184088C5C924F38
:107490000E94194180918508909186080E94CC2E07
:1074A0001127A801B7010E943A308091830890917A
:1074B00084088C5C924F0E94FC401F910F91FF90BA
:1074C000EF900895EF92FF920F931F93CF93DF9366
:1074D000CDB7DEB722970FB6F894DEBF0FBECDBF93
:1074E0008E01055F1F4FF801E190F1908F018091AF
:1074F0008308909184088C5C924F0E9419411A83F2
:107500000983A801B70180918508909186080E949F
:107510008F308C0180918308909184088C5C924F0D
:107520000E94FC40C80122960FB6F894DEBF0FBE41
:10753000CDBFDF91CF911F910F91FF90EF900895F4
:107540000F931F938C0180918308909184088C5C29
:10755000924F0E9419416091850870918608C80178
:107560000E94542F80918308909184088C5C924FE4
:107570000E94FC401F910F910895E0918308F091C3
:107580008408E256F24F24E641E0608182E00E94E6
:1075900052368091830890918408865C924F0E94B5
:1075A000A03A08950F931F93982FDB01E091830871
:1075B000F0918408E65CF24F8081EA53FD40882315
:1075C00021F5E256F24F9083FB0101900020E9F78C
:1075D00031970E2F061B043608F003E61127809121
:1075E000830890918408A801BD01865C924F0E9497
:1075F0004B7A8091830890918408080F191F065CCC
:10760000124FF80110820E94BD3A1F910F91089508
:107610008091830890918408805E924F0E94A03AE6
:1076200008950E94083BE0918308F0918408DF01EF
:10763000A15EB24FE25EF24F8081EE51FD4022E842
:10764000829FC00111248C56954F6C918E0F9F1F05
:107650000E943C3A0895CF93DF93EB019093860804
:10766000809385088FE99DE00E94EC0C909384083C
:1076700080938308009749F481EF93E09F938F9361
:107680000E94623A0F900F902BC0FE0101900020E3
:10769000E9F731974E2F4C1B453108F044E155274F
:1076A000BE01805E924F0E944B7A20E030E08091D4
:1076B000830890918408FC013B96118210823D96CC
:1076C0002F5F3F4F22333105C1F78C5C924F0E94F0
:1076D000E040E0918308F0918408E65CF24F10826C
:1076E000DF91CF9108956F927F929F92AF92BF9258
:1076F000CF92DF92EF92FF920F931F93CF93DF937E
:107700007C01A0908308B0908408650166247724EA
:107710008501962CF60183859485892BF9F0E80183
:1077200009900020E9F72197C01BD10BAE01B701EA
:10773000C8010E943D7A892B89F4F701EC0FFD1FE7
:107740008081803209F44AC0F70101900020E9F7F6
:107750003197EE19FF09CE17DF07A1F09394089433
:10776000611C711C035F1F4F8DE090E0C80ED91E95
:1077700092E36916710469F6E2E39E1619F481E05A
:1077800090E043C0292D33278DE090E0289FF00141
:10779000299FF00D389FF00D1124EA0DFB1DDF012C
:1077A0000D900020E9F71197AE1BBF0BAE0DBF1D6A
:1077B0008C91811111968DE090E0289FF001299F16
:1077C000F00D389FF00D1124EA0DFB1D0384F485A4
:1077D000E02DCD01099580E090E017C0262D3327DC
:1077E0008DE090E0289FF001299FF00D389FF00D6B
:1077F0001124EA0DFB1DDF010D900020E9F7119720
:10780000AE1BBF0BAE0DBF1DD5CFDF91CF911F912A
:107810000F91FF90EF90DF90CF90BF90AF909F902F
:107820007F906F900895CF93DF93EC01FC0101905E
:107830000020E9F73197E81BF90B3B97C0F09F93C5
:107840008F938BED94E09F938F930E94623A83EC29
:1078500094E09F938F930E94623A4DB75EB74A5F60
:107860005F4F0FB6F8945EBF0FBE4DBF3EC0A091F4
:107870008308B0918408FD0120E083859485892BDD
:10788000D9F02F5F3D962233C1F7DF93CF938FEA74
:1078900094E09F938F930E94623A84E994E09F93CF
:1078A0008F930E94623A8DB79EB706960FB6F894F2
:1078B0009EBF0FBE8DBF19C033278DE090E0FC0145
:1078C0002E9FC0012F9F900D3E9F900D1124A80F59
:1078D000B91FFD0174876387209183083091840864
:1078E000BE01820F931F0E94367ADF91CF910895D7
:1078F0002F923F924F925F926F927F928F929F92C0
:10790000AF92BF92CF92DF92EF92FF920F931F93AD
:10791000CF93DF93CDB7DEB723970FB6F894DEBFD2
:107920000FBECDBF7C01062F498322241FEF3324D5
:10793000442455246624772488249924AA24BB242B
:10794000C0908308D0908408C5018C0D9D1D9B8339
:107950008A83FC0183859485892B09F45DC0402FBF
:107960005527B701CF010E943D7A892B09F054C0F9
:10797000F981FF2349F11F3F19F091E0392E08C02A
:1079800085EF94E09F938F930E94623A0F900F903F
:107990008091830890918408880D991D0E94A03AD7
:1079A0002394822D65E00E94797A992319F483EF5C
:1079B00094E002C081EF94E09F938F930E94623A1B
:1079C000102F0F900F9028C01F3F11F0202F20C0C4
:1079D000EA81FB8101900020E9F731971E2F8A810F
:1079E000181B6A817B81C7010E94367A15C0122F4D
:1079F00011C0822F9927D701A80FB91FF301EC0DF1
:107A0000FD1DE80FF91F9C918081981781F72F5F6A
:107A1000211778F381E0382E0894411C511CEDE0C9
:107A2000F0E0AE0EBF1E8E0E9F1E6E0E7F1EF2E3A6
:107A30004F16510409F084CF1F3F19F4802F992766
:107A400023C0332031F4F701E10FF11D80E2808380
:107A50001F5F8981882379F08FEE94E09F938F9345
:107A60000E94623A0E94083B612FC7010E943C3A83
:107A70000F900F9007C0612F601BC701800F911DF1
:107A80000E943C3A812F992723960FB6F894DEBFC7
:107A90000FBECDBFDF91CF911F910F91FF90EF905F
:107AA000DF90CF90BF90AF909F908F907F906F901E
:107AB0005F904F903F902F900895DF92EF92FF924A
:107AC0000F931F93CF93DF93CDB7DEB723970FB6F6
:107AD000F894DEBF0FBECDBF86E90E94640B0E9402
:107AE000113BEE24DD24FF248091850890918608C7
:107AF0000E94CC2E41E050E0BE016F5F7F4F0E949C
:107B000031478F3F39F486E694E09F938F930E942C
:107B1000623AE2C1813041F78091850890918608F0
:107B20000E94CC2E0E947749882369F099279F9361
:107B30008F9381E594E09F938F930E94623A0F9018
:107B40000F900F900F9099819B3109F0BCC010E00D
:107B500080918508909186080E94CC2E212F332792
:107B600027FD309542E050E0421B530BBE016F5F92
:107B70007F4F620F731F0E943147180F123044F37A
:107B800089818B3509F04BC08A818134D1F42E2D47
:107B90003327E0918308F0918408E25EF24F808100
:107BA0009927821B930B059665E070E00E94997AF5
:107BB0000497A9F1DD2011F4EE2089F1C9010496A2
:107BC0000EC0E0918308F0918408823471F4E25E83
:107BD000F24F8081E81619F18E2D9927019665E004
:107BE00070E00E94997AE82E1AC0E25EF24FE080BF
:107BF00016C081508C9388E090E09F938F939F9361
:107C00008F938BE494E09F938F930E94623A8DB799
:107C10009EB706960FB6F8949EBF0FBE8DBFE0913B
:107C20008308F0918408DF01A15EB24F8C91882314
:107C300001F7E25EF24F4081EE51FD40E41609F497
:107C400052CF2E2D332782E890E0289F8001299F74
:107C5000100D389F100D11240C56154FBF01600FE9
:107C6000711F32E8F32E4F9DC00111248C56954FA1
:107C700042E850E08E0F9F1F0E944B7A809183084C
:107C800090918408800F911F0E94A03A80918308F0
:107C900090918408825E924FDC01EC918E519D4060
:107CA000EF9DF0011124EC56F54FE80FF91FDF01AD
:107CB0000D900020E9F71197AE1BBF0B815E924F2C
:107CC000FC01A08310CF9A3019F09D3009F08FC0CD
:107CD000A0918308B0918408A15EB24F4C918E911F
:107CE000AE51BD40992722E830E0829FF001839F8A
:107CF000F00D929FF00D1124EA0FFB1FE40FF11D10
:107D0000EC56F54F108289E494E09F938F930E9484
:107D1000623AE0918308F0918408E15EF24F0F909F
:107D20000F908081EF51FD40882309F45DC0E25E31
:107D3000F24F80818F010E511D4022E8829FC001C9
:107D400011248C56954F080F191FC8010E94733BD0
:107D5000882361F01F930F9382E394E09F938F93A6
:107D60000E94623A0F900F900F900F90E09183085D
:107D7000F0918408E25EF24F80818F5F8083E09112
:107D80008308F0918408E25EF24F8081853019F417
:107D9000108221E0D22EE0918308F0918408E25E07
:107DA000F24FE190108220E030E042E850E0A091F4
:107DB0008308B0918408A25EB24F8C91AE51BD4051
:107DC0009927849FF001859FF00D949FF00D112459
:107DD000EA0FFB1FE20FF31FEC56F54F10822F5FE7
:107DE0003F4F2238310519F70E94083B7CCE98306E
:107DF00019F09F3709F044C0E0918308F09184089E
:107E0000E15EF24F8081882309F46DCE88E090E036
:107E10009F938F939F938F938CE294E09F938F9384
:107E20000E94623AE0918308F0918408E15EF24F8B
:107E3000808181508083A0918308B0918408A15EE5
:107E4000B24F4C918E91AE51BD40992722E830E05F
:107E5000829FF001839FF00D929FF00D1124EA0F95
:107E6000FB1FE40FF11DEC56F54F1082FF248DB778
:107E70009EB706960FB6F8949EBF0FBE8DBF34CE48
:107E8000E0918308F09184089930C9F48F01015E74
:107E9000124FE25EF24F8081EE51FD4022E8829F58
:107EA000C00111248C56954F4F2DD8016C918E0F27
:107EB0009F1F0E94783CF8018083F39415CEE15E09
:107EC000F24F80818F3759F489E194E09F938F932B
:107ED0000E94623A0E94113B0F900F9005CE892FAD
:107EE00099279F938F9386E194E09F938F930E94AD
:107EF000623AA0918308B0918408A15EB24F4C9180
:107F00008E91AE51BD40992722E830E0829FF0016A
:107F1000839FF00D929FF00D1124EA0FFB1FE40FD9
:107F2000F11DEC56F54F89818083E0918308F09133
:107F30008408E15EF24F80818F5F8083FF240F9081
:107F40000F900F900F90D0CD9B01882359F42050B3
:107F50003C4F40E050E065EB7FE389E096E00E9413
:107F6000041108950E945D3D08950E945D3DFFCF7C
:107F700065EC7FE384E196E00E94133C65E870E4E1
:107F800088E196E00E94133C0895AF92BF92CF9291
:107F9000DF92EF92FF920F931F93CF93DF93CDB7B2
:107FA000DEB72A970FB6F894DEBF0FBECDBF8C01A7
:107FB0001A86198629E0A22EB12CAC0EBD1EBF92E6
:107FC000AF92CE0101969F938F9395E0C92ED12C4D
:107FD000CC0EDD1EDF92CF92CE0103969F938F933E
:107FE0008CE196E09F938F931F930F930E94D3464B
:107FF0002DB73EB7245F3F4F0FB6F8943EBF0FBE7C
:108000002DBF03973CF02D814B81698589810E94AA
:1080100052366AC04AE050E06CE276E0C8010E9445
:108020003D7A892B19F40E94F5365EC087E0E82E70
:10803000F12CEC0EFD1EFF92EF9287E396E09F93EA
:108040008F931F930F930E94D3462DB73EB72A5F9D
:108050003F4F0FB6F8943EBF0FBE2DBF019721F4DE
:108060008F810E94963640C0FF92EF928CE396E09B
:108070009F938F931F930F930E94D3462DB73EB7C4
:108080002A5F3F4F0FB6F8943EBF0FBE2DBF01973A
:1080900021F48F810E947E3627C0DF92CF92FF921B
:1080A000EF92BF92AF9282E496E09F938F931F93DB
:1080B0000F930E94D3462DB73EB7265F3F4F0FB6B2
:1080C000F8943EBF0FBE2DBF039731F44D816F81F1
:1080D00089850E94773608C08BE496E09F938F9342
:1080E0000E94D1390F900F902A960FB6F894DEBFF8
:1080F0000FBECDBFDF91CF911F910F91FF90EF90F9
:10810000DF90CF90BF90AF9008958AE090E00E94FA
:108110002E359C0168EE73E00E94997A6AE070E067
:108120000E94997A7F936F93C90168EE73E00E9471
:10813000997A7F936F9385EE96E09F938F930E9439
:10814000D1398DB79EB706960FB6F8949EBF0FBE75
:108150008DBF089560931A0870931B0880931C08C4
:1081600090931D0840938708089580918708813077
:1081700089F40E9419099B01AC0180911A08909121
:108180001B08A0911C08B0911D08280F391F4A1F19
:108190005B1F10C00E9419099B01AC0180911A0855
:1081A00090911B08A0911C08B0911D08281B390B49
:1081B0004A0B5B0BCA01B90108950E941909089581
:1081C000FC0113821282158214821182108208959A
:1081D000FC0184819581892B61F02281338180911A
:1081E0004308909144082817390719F08FEF9FEF43
:1081F000089580E090E00895FC0122813381809110
:108200004308909144082817390719F08FEF9FEF22
:10821000089584819581019795838483892B19F032
:1082200080E090E00895CF010E94EA0F80E090E0A6
:108230000895CF93DF93EC012A813B81809143081D
:10824000909144082817390741F40BC040E050E0F2
:1082500060E070E0CE010E94A6108C819D81892B88
:10826000A9F780914308909144089B838A838C816D
:108270009D8101969D838C83DF91CF910895FC01B0
:1082800084819581892B61F022813381809143081B
:10829000909144082817390719F08FEF9FEF089540
:1082A000CF010E94194180E090E008950F931F9341
:1082B000CF93DF93FC01C189D289EDA9FEA909956D
:1082C0008C01892B49F4CF5BDF4FE881F98160E0B5
:1082D00072EC81E090E00995C801DF91CF911F9188
:1082E0000F910895CF93DF93EC01EA81FB81018820
:1082F000F289E02D0FB6F8940F9264A575A50F9042
:108300000FBE88279927DF91CF910895CF92DF92F2
:10831000EF92FF920F931F93CF93DF93EC018B01AA
:108320007A0169018C819D81288539850FB6F89481
:108330000F92198618860F900FBE2617370789F0FF
:10834000232B21F0009711F00E944D3001151105EB
:1083500009F1C8010E945030009729F48FEF9FEF78
:108360001BC0672BB9F09D838C83998388839B8383
:108370008A83800F911F9F838E83FD86EC86DF8624
:10838000CE861B861A860FB6F8940F921987088737
:108390000F900FBE80E090E0DF91CF911F910F9181
:1083A000FF90EF90DF90CF900895CF92DF92EF9201
:1083B000FF920F931F93CF93DF938A01DA01CD9041
:1083C000DD90ED90FC902C2DFC01C189D289F1E06B
:1083D00067307F0709F464C081E068307807ECF407
:1083E00091E06330790709F44AC0A1E064307A076C
:1083F00054F4B1E061307B0799F1E1E062307E072F
:1084000009F0CCC030C0F1E065307F0709F442C00C
:10841000665071400CF041C03AC091E06B30790772
:1084200009F4A8C0A1E06C307A0754F4B1E06930D7
:108430007B0709F441C06A5071400CF076C033C02C
:10844000F1E06D307F0709F49FC081E06D3078075F
:108450000CF495C091E06E30790709F09FC099C087
:10846000CF5BDF4F5FC0CD5BDF4FE881F9810995BE
:10847000D8016D937D938D939C93139736C1CB5BFD
:10848000DF4FE881F9818C2D09958C0130C1C95BE2
:10849000DF4F0BC0C75BDF4FF4CFC55BDF4F05C0BD
:1084A000C35BDF4FEECFC15BDF4FE881F9810995F8
:1084B0009927AA27BB2714C1C6FC03C000E010E01F
:1084C00011C0FE01B29626853785448555856085A5
:1084D0007185CF010E9486418C01892B19F4EBAD87
:1084E000FCAD0995C7FE10C00115110509F0FFC0CC
:1084F000FE01709626853785448555856085718592
:10850000CF010E9486418C010115110509F0EFC0D1
:10851000CF5ADF4F8FE39FEFAFEFBFEFC822D922D3
:10852000EA22FB22E881F9815DC0CD5ADF4FE88164
:10853000F981C355D04009959B01AC01D8016D93D9
:108540007D938D939C9313978CA59DA5892B31F4D6
:108550002064F80120833183428353838A8D9B8D6D
:10856000892B09F0C2C0F80180819181A281B38179
:108570008068B7C0C886D986EA86FB86B6C088857B
:108580009985AA85BB85ACC0CC86DD86EE86FF8644
:10859000ACC08C859D85AE85BF85A2C0FB01EF5028
:1085A000F140E931F10540F4EA5BFF4FEE0FFF1FA8
:1085B0000590F491E02D09940FEF1FEF98C088818A
:1085C0009981AA81BB81222311F0806422C08F7B14
:1085D00020C088819981AA81BB8186FF27C021C0E4
:1085E000EDADFEADC701B60109954FCFEF96E8811D
:1085F000F9810995F801608371838283938375C043
:1086000088819981AA81BB81222311F0806801C0F1
:108610008F7788839983AA83BB8367C0888187FF0C
:1086200005C081E090E0A0E0B0E05AC0D8011D9202
:108630001D921D921C92139758C0CB5ADF4FE881B0
:10864000F981822F21CFC95ADF4F2FCFFE017096BB
:108650002685378544855585B601CF010E94864120
:108660008C01892B09F043C0EBADFCAD09953FC0EF
:10867000888D998D33C0FE01B29626853785448555
:108680005585B601CF010E948641FFCE8AA59BA5E4
:1086900025C00FB6F8940F92DD8ECC8E1AC08C8D4B
:1086A0009D8D1CC00FB6F8940F92DF8ECE8E11C038
:1086B0008E8D9F8D13C00FB6F8940F92DFA6CEA6B5
:1086C00008C08EA59FA50AC00FB6F8940F92D9AA2C
:1086D000C8AA0F900FBE09C088A999A9AA27BB27CD
:1086E000F80180839183A283B38300E010E0C80186
:1086F000DF91CF911F910F91FF90EF90DF90CF907E
:108700000895CF92DF92EF92FF920F931F93CF9332
:10871000DF936C018A01FC01C189D28983E0E82ED4
:10872000F12CE422F522E114F10481F028E330E099
:1087300048E250E060E470E0CE0140960E9486413D
:10874000892BA1F4F1E0EF16F10499F020EF30E06D
:1087500040ED50E060E071E0CE0182960E948641DB
:10876000892B39F08C899D890E944D300FEF1FEFC6
:108770002CC086E090E00E945030009739F48C893C
:108780009D890E944D308EA19FA1EECF0070107C7C
:10879000288139814A815B810050104811F42F777C
:1087A00001C02068288339834A835B838C01FC01E4
:1087B00011821082D382C28215821482F1E0EF16F8
:1087C000F10419F0EBADFCAD0995C801DF91CF9133
:1087D0001F910F91FF90EF90DF90CF900895CF936E
:1087E000DF93DC01EC01EA81FB81C189D289019729
:1087F0008E5F9F4F18F08FEF9FEF19C0CD010E9441
:108800004D3020E030E040E050E060E070E0CE012C
:1088100040960E94864120E030E040E050E060E079
:1088200070E0CE0182960E94864180E090E0DF9168
:10883000CF910895CF92DF92EF92FF920F931F9303
:10884000CF93DF937C016A01EC0160960FB6F89438
:108850000F928A859B85860F971F9B878A8713C0F7
:10886000F70181AD92ADFC010995F701448555856D
:1088700066857785CE0140960E943D10892B51F484
:108880000FB6F8940F920A851B850F900FBEC01685
:10889000D10630F3C801DF91CF911F910F91FF9066
:1088A000EF90DF90CF9008956F927F928F929F927A
:1088B000AF92BF92CF92DF92EF92FF920F931F93EE
:1088C000CF93DF93CDB7DEB722970FB6F894DEBF14
:1088D0000FBECDBF4A015901FC01E188F288A0E139
:1088E0006A2E712C6E0C7F1CF30180859185892B7B
:1088F00021F4FFEFCF2EDF2E9BC06115710549F4E7
:1089000040E050E060E070E0C7010E941A446C0152
:108910008FC0F70180819181A281B3819C01AD015B
:10892000E9E05695479537952795EA95D1F7217057
:108930002A8327E0B695A795979587952A95D1F72D
:10894000817089830FB6F8940F92F30142855385A5
:108950000F900FBE8B01CC24DD2460E070E050C08E
:108960009A01260F371FF301868597852817390747
:1089700078F044855585C7010E941A44AC01F30183
:10898000848595858417950708F452C060E070E0EF
:10899000A114B10419F0F801849102C0D8018C919E
:1089A000B981B13069F48A3081F4EA81E13019F09B
:1089B000F2E0F98303C082E08A8389838DE00AC0F4
:1089C0009981923011F4A1E0A9830F5F1F4F0894A1
:1089D000C11CD11CD301ED91FC911197819311968B
:1089E000FC93EE932D913C91F3018681978128179A
:1089F000390721F484819581918380836F5F7F4F54
:108A0000C814D9040CF4ACCF6115710589F00FB608
:108A1000F8940F92F30182859385860F971F9387B1
:108A200082870F900FBEF70181AD92ADFC010995D1
:108A3000C60122960FB6F894DEBF0FBECDBFDF9100
:108A4000CF911F910F91FF90EF90DF90CF90BF904B
:108A5000AF909F908F907F906F90089521E030E0CD
:108A6000FC01828193810E945444089520E030E00B
:108A7000FC01828193810E9454440895AF92BF9279
:108A8000CF92DF92EF92FF920F931F93CF93DF93DA
:108A90007B015A01EC01EA81FB8101891289E8011D
:108AA000A296688579856115710519F48FEF9FEF9E
:108AB000A1C0E114F10461F42E853F854C855D85EC
:108AC000CE010E948641E801EBADFCAD09951AC0CC
:108AD0000FB6F8940F926A857B850F900FBE6115D3
:108AE000710599F4F80183AD94ADFC010995F80185
:108AF0004085518562857385CE0140960E943D1068
:108B0000892B31F380E090E075C0D701F8018081B6
:108B100087FF35C0CC24DD24EE24FF245AE02BC08F
:108B2000E616F70609F44FC0EA81FB814191FB8309
:108B3000EA832A813B818E819F812817390721F49E
:108B40008C819D819B838A834D3011F04A3051F492
:108B5000F80184A9882311F0841751F4F80144AB7B
:108B60005D9303C0F80114AA4D930894C11CD11C55
:108B70000894E11CF11CCA14DB0490F221C06B01C3
:108B8000A616B70608F4650140E050E0D70114C00E
:108B9000EA81FB8181918C93FB83EA832A813B816B
:108BA0008E819F812817390721F48C819D819B83B9
:108BB0008A834F5F5F4F11964C155D0549F776012B
:108BC000E114F104B1F00FB6F8940F928A859B85F9
:108BD0008E199F099B878A870F900FBE2A853B8538
:108BE0008C859D852817390720F4E801EBADFCAD95
:108BF0000995C601DF91CF911F910F91FF90EF90E2
:108C0000DF90CF90BF90AF900895FC01808191815B
:108C1000A281B3810196A11DB11D80839183A2839E
:108C2000B383268137812115310521F08481958117
:108C3000F90109950895EF92FF920F931F93CF9337
:108C4000DF93EC017B018A01E885F985309719F4FF
:108C500080E090E005C060E070E080E090E0099581
:108C60001D830C83FF82EE82DF91CF911F910F91C4
:108C7000FF90EF900895CF93DF93EC01E885F9859D
:108C8000309719F48FEF9FEF05C060E070E081E14D
:108C900090E00995DF91CF910895CF93DF93EC0198
:108CA000E885F985309719F48FEF9FEF05C060E0F4
:108CB00070E082E190E00995DF91CF9108950F93E4
:108CC0001F93CF93DF93CDB7DEB724970FB6F894F9
:108CD000DEBF0FBECDBF8C017C836B83FC01208582
:108CE00031852115310519F48FEF9FEF17C0BE01B3
:108CF0006F5F7F4F80E290E0F9010995009771F472
:108D0000F80120853185BE016D5F7F4F81E290E0E3
:108D1000F9010995009711F489819A8124960FB67B
:108D2000F894DEBF0FBECDBFDF91CF911F910F91A1
:108D300008950F931F93CF93DF93CDB7DEB724979A
:108D40000FB6F894DEBF0FBECDBF8C017C836B8362
:108D5000FC01208531852115310519F48FEF9FEF36
:108D600017C0BE016F5F7F4F88E190E0F901099560
:108D7000009771F4F80120853185BE016D5F7F4F4A
:108D800089E190E0F9010995009711F489819A81B0
:108D900024960FB6F894DEBF0FBECDBFDF91CF9102
:108DA0001F910F910895CF93DF93CDB7DEB7229730
:108DB0000FB6F894DEBF0FBECDBFAE01455F5F4F6B
:108DC0005A83498369857A858F8198850E941347E4
:108DD00022960FB6F894DEBF0FBECDBFDF91CF91C4
:108DE0000895FC01CB019A0160817181AC018AE395
:108DF00090E30E942F310895CF93DF93EC0180E040
:108E000090E0DB0105C02D933196F983E88301964C
:108E10008417950729F0E881F9812081222399F7A9
:108E2000DF91CF910895CF93DF93CDB7DEB722972F
:108E30000FB6F894DEBF0FBECDBF9A019A83898327
:108E4000AB01BE016F5F7F4F8CEF96E40E944447F9
:108E500022960FB6F894DEBF0FBECDBFDF91CF9143
:108E60000895CF93DF93DC01EC01EA81FB81309719
:108E700019F4ED81FE8103C00788F08DE02DCD014E
:108E80000995DF91CF9108952F923F924F925F9273
:108E90006F927F928F929F92AF92BF92CF92DF920A
:108EA000EF92FF920F931F93CF93DF93CDB7DEB76F
:108EB00063970FB6F894DEBF0FBECDBF3C014B01E8
:108EC0002A01590122243324FF24D2011C911123A9
:108ED00009F494C10894411C511C812F99270E94C8
:108EE000F37A892B99F041E050E0BE016F5F7F4F2C
:108EF000C401F3010995019741F7898199270E94DF
:108F0000F37A892B81F7A1E0FA2EDFCF153289F0B1
:108F1000FF2059F441E050E0BE016F5F7F4FC40174
:108F2000F3010995019709F0A5C08981811761F2C4
:108F300065C1F20181912F01853291F4FF2059F42E
:108F400041E050E0BE016F5F7F4FC401F30109951E
:108F5000019709F08FC08981853209F4B5CF4EC1E0
:108F6000982FCC24DD2400E02AE030E09A3211F47E
:108F7000026016C09C3611F4016012C0892F805324
:108F80008A3090F4A601429F6001439FD00C529F0B
:108F9000D00C1124C90ED11C80ED9FEFC80ED91E34
:108FA000D2019D912D01E2CF9F3609F450C1903737
:108FB00048F4933609F44FC1993661F0992309F4C6
:108FC00043C149C0933721F0983709F044C005C028
:108FD00012E042C013E0EE2441C0006113E0F0E172
:108FE000EF2E3CC001FD12C024C0FF2059F440E127
:108FF00050E0BE016E5F7F4FC401F3010995181662
:109000001906C4F5E0EFFFEFCE0EDF1EF1E1CF163B
:10901000D10458F7FF2009F07EC0A601BE016E5FA3
:109020007F4FC401F3010995181619060CF473C09B
:1090300021C0FF2009F06EC0D5016D917C91A60181
:10904000C401F301099518161906A4F4E2E0F0E052
:10905000AE0EBF1E5FC013E0EAE0EE2EFF2071F4FB
:1090600041E050E0BE016F5F7F4FC401F3010995FD
:10907000019721F0222009F4E7C0C0C0F9808F2DAC
:1090800099270E94F37A892B59F7123009F048C0CA
:10909000C114D10419F47FEFC72ED72E01FF17C0DA
:1090A0000894C108D108C114D104A9F141E050E0ED
:1090B000BE016F5F7F4FC401F3010995019759F518
:1090C000898199270E94F37A892B29F5E9CFD50167
:1090D0000D911C91F801F1928F010894C108D108FB
:1090E000C114D10489F041E050E0BE016F5F7F4FB1
:1090F000C401F3010995019739F4F9808F2D99275F
:109100000E94F37A892B31F342E050E0A40EB51EA1
:10911000D8011C9233942394D7CE61E0F62E6AC016
:10912000133009F0D1CEC60101970F9718F05FE018
:10913000C52ED12C102F1C62FE013296FB8BEA8BC0
:1091400054C09981903349F4EE2019F4106148E03D
:10915000E42E15FF20C0137D32C0892F8153873044
:1091600018F4EE20C1F406C0892F8853823048F4E9
:10917000EE2019F43AE0E32E0EC0F8E0FE15C8F533
:109180000AC0892F8154863018F08052863028F426
:109190004AE04E1570F5137E12C09D3211F09B32DD
:1091A00021F412FF26C01B7F0AC0983719F09835AA
:1091B00009F0B3CF14FF1DC01F7E20E1E22EAA8963
:1091C000BB899D93BB8BAA8BB2E0CB16D10450F028
:1091D00041E050E0BE016F5F7F4FC401F30109958C
:1091E000019739F40894C108D108C114D10409F0D9
:1091F000A8CFFF24012F112703FF03C0832D992738
:1092000032C001FD1FC0EA89FB8910824E2D55270F
:1092100060E070E0CE0102960E94847795012E5F97
:109220003F4F00FF08C0D501ED91FC916083718331
:109230008283938305C0D501ED91FC917183608396
:1092400059013394239441CE8FEF9FEF0CC013E06C
:1092500098E0E92E03CFC114D10409F0C3CE81E018
:10926000C82ED12CBFCE63960FB6F894DEBF0FBECA
:10927000CDBFDF91CF911F910F91FF90EF90DF90C5
:10928000CF90BF90AF909F908F907F906F905F90A6
:109290004F903F902F900895882321F0813011F056
:1092A000823019F40E9444360895833011F40E94EC
:1092B00044360895882321F0813011F0823019F46A
:1092C0000E9437360895833011F40E94373608958E
:1092D0000E94313680E00E944C4981E00E944C4956
:1092E00082E00E944C4983E00E944C490895DF923D
:1092F000EF92FF920F931F93CF93DF93CDB7DEB71B
:1093000024970FB6F894DEBF0FBECDBF8C017E014F
:109310000894E11CF11CA7016AE071E00E94D02FC3
:1093200029813A814B815C81DA01C9018770907093
:10933000A070B0700097A105B10511F4DD2411C033
:1093400087E0D82ED22287E090E0A0E0B0E08983C9
:109350009A83AB83BC83A70169E071E0C8010E94D6
:10936000D02F8D2D992724960FB6F894DEBF0FBE0F
:10937000CDBFDF91CF911F910F91FF90EF90DF90C4
:109380000895CF92DF92EF92FF920F931F93CF93A6
:10939000DF936C01EB01E42EFF243BC08E01020F32
:1093A000131FC6010E94CC2E41E050E0B8010E947C
:1093B0003147F8010081083011F00F3761F4FF20C8
:1093C00041F182E097E09F938F930E94D139FA9404
:1093D0000F900F901EC00A3011F00D3049F486E056
:1093E00097E09F938F930E94D1390F900F901AC0EE
:1093F000802F992787FD90959F938F9388E097E022
:109400009F938F930E94D139F3940F900F900F90F8
:109410000F902F2D33278E2D992701972817390765
:109420000CF4BCCFCF0DD11D1882F3948F2D99274A
:10943000DF91CF911F910F91FF90EF90DF90CF9030
:109440000895FC01808199279F938F9381819927AB
:109450009F938F93828199279F938F9383819927DD
:109460009F938F93848199279F938F9385819927C9
:109470009F938F938BE097E09F938F930E94D139B6
:109480008DB79EB70E960FB6F8949EBF0FBE8DBFD8
:1094900008955F926F927F928F929F92AF92BF9248
:1094A000CF92DF92EF92FF920F931F93CF93DF93B0
:1094B0004C013B01EC0101C0219688818032E1F32F
:1094C000530195E0592E1881E12EFF24E7FCF0941A
:1094D000C7010E94E97A892B89F10981C02EDD2418
:1094E000C7FCD094C6010E94E97A892B39F11A335E
:1094F00014F4105305C0C7010E94027B182F1755A2
:109500000A331CF4802F805304C0C6010E94027BE2
:1095100087551295107F182BF5011583CE01029601
:109520005520A9F08A818A3349F423965A940894E5
:10953000A108B108FFEF5F1659F0C5CFF301A0E312
:10954000B8E086E00D900192815019F0FBCFEC015C
:109550004E01C401DF91CF911F910F91FF90EF90C9
:10956000DF90CF90BF90AF909F908F907F906F9043
:109570005F9008950F931F93FC01808199279F931B
:109580008F93818199279F938F93828199279F93AE
:109590008F93838199279F938F93848199279F939A
:1095A0008F93858199279F938F938BE097E09F936B
:1095B0008F930EE118E01F930F930E94274B8DB7F6
:1095C0009EB740960FB6F8949EBF0FBE8DBFC801E0
:1095D0001F910F910895AF92BF92CF92DF92EF92B9
:1095E000FF920F931F93CF93DF937C015B016A017E
:1095F000EC0100E010E018C0EA0DFB1D8081992706
:109600009F938F9389E297E09F938F93DF93CF93FC
:109610000E94274BC80FD91F8DB79EB706960FB66D
:10962000F8949EBF0FBE8DBFE02FFF270F5F1F4F27
:10963000EC15FD0508F3C701DF91CF911F910F9144
:10964000FF90EF90DF90CF90BF90AF900895CF93B1
:10965000DF93CDB7DEB722970FB6F894DEBF0FBE0B
:10966000CDBFAE01455F5F4F5A83498369857A85D7
:109670008F8198850E94454B22960FB6F894DEBFE5
:109680000FBECDBFDF91CF910895CF93DF93CDB7BC
:10969000DEB722970FB6F894DEBF0FBECDBF9A8318
:1096A00089839A01AB01BE016F5F7F4F86E69BE421
:1096B0000E942F31E981FA81108222960FB6F89428
:1096C000DEBF0FBECDBFDF91CF910895EF92FF9225
:1096D0000F931F937C018A01FC01808191810E947C
:1096E000157AF70180819181800F911F918380838A
:1096F000C8011F910F91FF90EF900895CB0108953D
:1097000008950895FC01E95DFD4F619371933183E4
:1097100020837697518340830895FC01ED5BFD4FD4
:10972000718360833C97518340830895FC01EB581B
:10973000FD4F61937193518340830895FC01EE596D
:10974000FC4F61937193518340830895AF92BF9210
:10975000CF92DF92EF92FF920F931F93CF93DF93FD
:109760006C01A42EB22EFC01E758FD4F20E0808151
:1097700091818617970731F02F5F77962A3009F489
:109780004BC0F5CF822F992727E130E0829FE0017F
:10979000839FD00D929FD00D1124CC0DDD1DC65797
:1097A000DD4F8881CA58D2408530B1F5C601815E4F
:1097B0009D4F0E94E876FE01E257FD4F80818F5F4A
:1097C000808382E0F7018083FE01E558FD4F8081B0
:1097D000E701898321818A2D99278370907034E075
:1097E000880F991F3A95E1F7282BBB0CBB0CBB0CDB
:1097F000BB0CBB0CBB0C2B292A830B83812F992715
:109800008C83B701C6010E942850FC01BF01882744
:1098100077FD8095982F04C06DEF7EEF8FEF9FEF5F
:10982000DF91CF911F910F91FF90EF90DF90CF903C
:10983000BF90AF900895CF92DF92EF92FF920F9377
:109840001F93CF93DF93EC015CE6C52E53E0D52E3A
:10985000C80ED91E60E070E00E943266F601A08555
:10986000B185109751F0FD01E480F58006811781E4
:109870002D913D914D915C910CC04FEFE42E4FEF37
:10988000F42E4FEB042F4FEF142F2FEF3FE140E06A
:1098900050E060E070E0CE010E947D66F6014681F6
:1098A00057814115510531F060E070E0CE010E9412
:1098B000B96826C01F921F9281E08F931F921F925A
:1098C000DF93CF930E94046982E090E09F938F938F
:1098D0001F921F9282E08F931F921F92DF93CF936C
:1098E0000E940469CE59DC4F19821882C256D340B7
:1098F0008DB79EB740960FB6F8949EBF0FBE8DBF32
:10990000F601A281B381109719F04D915C9102C0CC
:1099100040E45FE160E070E0CE010E94A564F601E2
:10992000A689B789109719F04D915C9102C040E06B
:1099300050E260E070E0CE010E940464F601A28D66
:10994000B38D109711F04C9101C043E060E070E0DE
:10995000CE010E946C63F601A285B385109711F0C9
:109960004C9101C040E060E070E0CE010E94626274
:10997000F601A685B785109711F04C9101C041E022
:1099800060E070E0CE010E944561F601A089B189D6
:10999000109711F04C9101C041E060E070E0CE0101
:1099A0000E94AC60F601A481B581109739F04D9109
:1099B0005C9160E070E0CE010E94D973F601A4854D
:1099C000B585109769F0FD01E580F680038114816B
:1099D0004D915C91228160E070E0CE010E94DD61DA
:1099E000F601A289B389109749F02D913D914D91CF
:1099F0005C9160E070E0CE010E94BE62F601448995
:109A000055894115510529F060E070E0CE010E94B2
:109A10002B68F601A08DB18D109731F04C9160E06C
:109A200070E0CE010E949A65D601ED91FC913097CD
:109A300011F0608101C063E0CE010E94957460E086
:109A400070E0CE010E941C6ADF91CF911F910F91AF
:109A5000FF90EF90DF90CF9008958F929F92AF92FA
:109A6000BF92DF92EF92FF920F931F93CF93DF93FA
:109A7000EC01FC01EA5BFD4F80819181892B09F0AB
:109A800096C0809143089091440891838083EDE0D3
:109A9000AE2EB12CAC0EBD1EC5010E94E8767DE64F
:109AA000E72E72E0F72EEC0EFD1EC7010E94E8764D
:109AB0008E01085B1D4FC8010E94E876C7010E9415
:109AC000DA76C8010E94DA76FE01EE59FC4F8080FA
:109AD000918081E89BE4918380838A819B810E94AD
:109AE000CC2E40E052EC61E070E00E948A5281E0AE
:109AF00088870E94ED35CF58DD4F19921882C257E2
:109B0000D24069E7E62E62E0F62EEC0EFD1EDD2463
:109B1000F70181898823A1F18FEF9FEF93838283DF
:109B2000808191818F5F9F4F49F1D7014D915C9169
:109B300000E01FEF2FEF3FEF6FEF7FEFCE010E94AE
:109B4000E7558C018F5F9F4F81F7F7018189853041
:109B500091F4FE01EB58FD4FC958DD4F2881398142
:109B6000C757D240D7014D915C910190F081E02D13
:109B700068E083E00995F70111830083F701118AFA
:109B8000D39487E190E0E80EF91E9AE0D91609F027
:109B9000BFCFCE010E941B4CCE59DC4F99828882E8
:109BA000C5010E94DA76CC51D14019821882DF912A
:109BB000CF911F910F91FF90EF90DF90BF90AF90EA
:109BC0009F908F900895CF93DF93CDB7DEB72C97FA
:109BD0000FB6F894DEBF0FBECDBF4C01AE014D5F96
:109BE0005F4FBE016F5F7F4FC4010E9484513C01F3
:109BF000009709F476C0DC018C91833009F448C0E9
:109C0000843021F0823009F06CC005C0B301C4017A
:109C10000E94695A66C0F3010281602F77276F7036
:109C20007070762F662781819927682B792BC40164
:109C30000E948654F3018183492F55272281207F7A
:109C4000242B2283F401E95DFD4FAB80BC80CD80E5
:109C5000DE80E980FA8002950F70202F237049E2A0
:109C600052E0840E951E0190F081E02D0695069538
:109C7000AC01B301D4018D919C910995EAEEFFEFFF
:109C80008E0E9F1ED4018D939C93EDEEFDEF27C0A9
:109C9000F301628177276F707070762F662781815C
:109CA0009927682B792BC4010E94865423E432E063
:109CB000820E931ED401ED91FC912DEB3DEF820EAF
:109CC000931E2981AC01B301C401099547E352E019
:109CD000840E951ED4018D939C93E9ECFDEF8E0EBE
:109CE0009F1E21E732E0820E931ED4018C91EFE893
:109CF000FDEF8E0E9F1E882309F440C08401065795
:109D00001D4FAA24BB248DE7C82E82E0D82EC80C94
:109D1000D91CB9E8EB2EB2E0FB2EE80CF91CF401DB
:109D20008785908918161906D4F4838594851816AA
:109D30001906ACF4D8018C91823089F484E08C93BC
:109D4000F701408142954F704370B601C4010E94F3
:109D5000656EF401EF58FD4F808181508083089437
:109D6000A11CB11C27E130E0E20EF31EC20ED31E8F
:109D7000095E1F4F3AE0A316B10489F642E752E0AC
:109D8000840E951ED4018C91EEE8FDEF8E0E9F1E81
:109D9000882309F451C0A9E7EA2EA2E0FA2EE80CC4
:109DA000F91CAA24BB24FDE7CF2EF2E0DF2EC80C5D
:109DB000D91CF40187859089181619067CF58385CE
:109DC00094851816190654F5F7018689882331F50C
:109DD00084E090E09A838983DE011796F60186E09D
:109DE00001900D928150E1F7D7016D917C910FE2C6
:109DF00017E02981AE01495F5F4FC4010E94396DB0
:109E0000611571058105910549F483E0F701868BA1
:109E1000F401EE58FD4F8081815080830894A11C8D
:109E2000B11C27E130E0C20ED31EE20EF31E3AE071
:109E3000A316B10409F0BDCF0E94E80BCFCE0F935B
:109E40001F938B01BA0141E050E00E94CA67C8012C
:109E50001F910F9108950F931F93CF93DF938C0160
:109E600088E893E00E94EC0C009719F4C0E0D0E081
:109E700053C0EC011983088360E070E0815E9D4F60
:109E80000E94FF7660E070E0CE01825C9D4F0E94F0
:109E9000FF7661E070E0CE01885B9D4F0E94FF7607
:109EA000CE010E94BE5281E090E090938908809399
:109EB0008808CE010E943256C95DDD4F8FE19FE4D4
:109EC0008993999319821882669719821882E0966D
:109ED0008EE79BE4998388832C9719821882EE96EB
:109EE00080E89BE48993999319821882C757D240DE
:109EF00020E034E0AE0163EE7DE484E397E00E946D
:109F00000411CE010E941B4CAE014A595C4F60E027
:109F100070E0CE010E94D669CE01DF91CF911F91F2
:109F20000F91089504960E94DA76089504960E948F
:109F3000E8760895AF92BF92CF92DF92EF92FF92B0
:109F40000F931F93CF93DF93CDB7DEB763970FB611
:109F5000F894DEBF0FBECDBF5C017B016A01DE015C
:109F60001196ECE3F7E083E101900D928150E1F767
:109F700080913608882341F089E095E09F938F9384
:109F80000E9464770F900F9000E010E011C0C501AF
:109F90000E94CC2EA601401B510BB701600F711F10
:109FA0000E943A302FEF8F3F920781F1080F191F5F
:109FB0000C151D0560F380913608882301F100E03F
:109FC00010E012C0F70181917F0199279F938F9331
:109FD00082E095E09F938F930E9464770F5F1F4FFD
:109FE0000F900F900F900F900C151D0559F780E002
:109FF00095E09F938F930E9464770F900F90C50117
:10A000000E942C778F5F9F4F51F406C0BE016F5F97
:10A010007F4F8BE00E94D23A8FEF9FEF02C080E02B
:10A0200090E063960FB6F894DEBF0FBECDBFDF9110
:10A03000CF911F910F91FF90EF90DF90CF90BF9045
:10A04000AF900895FC01828193810E949A4F0895F8
:10A05000EF92FF920F931F93CF93DF937C018B01BD
:10A06000FB014081423029F1433020F4413009F0B6
:10A070004BC006C0433041F1443009F045C02AC00E
:10A08000FB018381C82FDD2723969281892F869536
:10A090008695833021F5892F9927982F882721814C
:10A0A0003327822B932B93700397C9F4F7014087D2
:10A0B00016C0FB0184819927D82FCC27838199274B
:10A0C000C82BD92B24960BC0FB018381C82FDD2719
:10A0D000239605C0FB018281C82FDD272296C70188
:10A0E0000E94964F2196AE01B801C7010E942250EE
:10A0F0008C01C7010E94924F8FEFF701818B17FDF2
:10A1000003C080E090E002C08FEF9FEFDF91CF911E
:10A110001F910F91FF90EF9008954F925F926F9271
:10A120007F928F929F92AF92BF92CF92DF92EF92E7
:10A13000FF920F931F93CF93DF93CDB7DEB7C95430
:10A14000D0400FB6F894DEBF0FBECDBF3C012B014F
:10A150005A01FC01E280F380DE019296EFE4F7E021
:10A1600082E101900D928150E1F7DE015396E1E624
:10A17000F7E08FE001900D928150E1F7DE01D49677
:10A18000E0E7F7E086E101900D928150E1F7DE0112
:10A190001596E6E8F7E08EE001900D928150E1F728
:10A1A000CC24DD2462C0C7010E94CC2EA5014C192D
:10A1B0005D09B2016C0D7D1D0E9431474C018F5F1E
:10A1C0009F4F09F45DC0C7010E94CC2E8E010F5F26
:10A1D0001F4FA8016AE071E00E94D02FF301808533
:10A1E000882369F087E090E0A0E0B0E089839A835B
:10A1F000AB83BC83C7010E94CC2EA80130C029814B
:10A200003A814B815C81DA01C90187709070A0703E
:10A21000B0700097A105B10531F120FF04C0BE0167
:10A220006D5E7F4F0BC021FF04C0BE016C5C7F4F91
:10A2300005C022FF06C0BE016B5F7F4F8BE00E940E
:10A24000D23A87E090E0A0E0B0E089839A83AB83C4
:10A25000BC83C7010E94CC2EAE014F5F5F4F69E007
:10A2600071E00E94D02FC80CD91CCA14DB0408F47A
:10A270009ACF80913608882361F480E090E02CC06A
:10A28000BE016E5D7F4F8BE00E94D23A8FEF9FEF51
:10A2900023C000E010E0720112C0F70181917F013C
:10A2A00099279F938F938DE095E09F938F930E94C2
:10A2B00064770F5F1F4F0F900F900F900F900A154C
:10A2C0001B0559F78BE095E09F938F930E9464776D
:10A2D00080E090E00F900F90C75BDF4F0FB6F894CF
:10A2E000DEBF0FBECDBFDF91CF911F910F91FF90C9
:10A2F000EF90DF90CF90BF90AF909F908F907F9026
:10A300006F905F904F900895CF92DF92EF92FF92FF
:10A310000F931F93CF93DF93CDB7DEB7A1970FB6FF
:10A32000F894DEBF0FBECDBF7C016B018A01FC013A
:10A3300082819381DE011296E4E9F7E020E2019048
:10A340000D922150E1F70E94CC2E41E050E0BE0179
:10A350006F5F7F4F0E943147019709F0C9C080911C
:10A360003608882371F0898199279F938F9389EF0D
:10A3700094E09F938F930E9464770F900F900F90BB
:10A380000F9089818330C1F1843009F45FC082303D
:10A3900009F096C00E941909F801608371838283D5
:10A3A000938323E132E0E20EF31EF7010081118175
:10A3B0002DEE3DEFE20EF31E8981F801819344E01A
:10A3C00050E0BF01C7010E948D50892B09F090C059
:10A3D000F80184819927582F442783819927482B96
:10A3E000592BF601518340834115510509F473C07F
:10A3F000B8016B5F7F4F23C027E332E0E20EF31E0C
:10A40000F7010081118129EC3DEFE20EF31EF80106
:10A41000819343E050E0BF01C7010E948D50892B1A
:10A4200009F066C0F8018381482F5527F601518352
:10A430004083882309F44FC0B8016C5F7F4FC70188
:10A440000E948D50892B09F446C052C087010F5ECF
:10A450001E4FF801819342E050E0BF01C7010E9406
:10A460008D50892B09F044C0F8018281482F55276F
:10A47000F60151834083882341F0B8016D5F7F4F1F
:10A48000C7010E948D50892B99F5F701808588239B
:10A4900011F1F80181818E30F1F49581892F869533
:10A4A0008695C9F4892F9927982F882724813327E7
:10A4B000822B932B9370892B71F4F70110860BC0BC
:10A4C000F70180858823A1F4BE016E5F7F4F8CE089
:10A4D0000E94D23A0DC080913608882359F087EF48
:10A4E00094E09F938F930E9464770F900F9002C027
:10A4F00000E010E0C801A1960FB6F894DEBF0FBED1
:10A50000CDBFDF91CF911F910F91FF90EF90DF9022
:10A51000CF9008950F931F93CF93DF93CDB7DEB7FE
:10A5200024970FB6F894DEBF0FBECDBF8C014983D0
:10A530005A836B837C8340E050E060E070E00E94CF
:10A540003A3084E60E949811AE014F5F5F4F61E0A0
:10A5500071E0C8010E94D02F892B19F08FEF9FEF77
:10A5600002C080E090E024960FB6F894DEBF0FBEE4
:10A57000CDBFDF91CF911F910F9108952F923F9200
:10A580004F925F926F927F928F929F92AF92BF9203
:10A59000CF92DF92EF92FF920F931F93CF93DF93AF
:10A5A000CDB7DEB724970FB6F894DEBF0FBECDBF90
:10A5B0002C0161E070E004960E94FF7640E060E0CC
:10A5C00070E0F201808191810E94C407892B09F01B
:10A5D0001BC1F2018081918164EB77E002960E94B9
:10A5E000D02EF201938382830E94CC2E1816190676
:10A5F0000CF00AC1F201828193810E94CC2E40E0CE
:10A6000052EC61E070E00E948A52892B09F0FCC094
:10A6100019821A821B821C82F201828193810E941C
:10A62000CC2E1E010894211C311CA10165E071E0B3
:10A630000E94D02F892B09F0E7C088E090E0A0E0CD
:10A64000B0E089839A83AB83BC83F20182819381DA
:10A650000E94CC2EA10163E071E00E94D02F892BD3
:10A6600009F0D2C081E090E0A0E0B0E089839A8355
:10A67000AB83BC83F201828193810E94CC2EA10125
:10A6800067E071E00E94D02F892B09F0BDC01982CC
:10A690001A821B821C82F201828193810E94CC2E3D
:10A6A000A10163E171E00E94D02F892B09F0ACC0B9
:10A6B00083E090E0A0E0B0E089839A83AB83BC8321
:10A6C000F201828193810E94CC2EA10161E171E0AF
:10A6D0000E94D02F892B09F097C0F2011086828149
:10A6E00093810E94CC2E40E050E060E070E00E9438
:10A6F000314780E092E0A0E0B0E089839A83AB83A9
:10A70000BC83F201828193810E94CC2EA1016BE176
:10A7100071E00E94D02F3C01882477FC8094982C13
:10A72000F201828193810E94CC2EA1016DE171E042
:10A730000E94D02FAA2797FDA095BA2F680E791EE8
:10A740008A1E9B1E84EF91E0A0E0B0E089839A838B
:10A75000AB83BC83F201828193810E94CC2EA10144
:10A7600062E271E00E94D02F7C01F201828193812C
:10A770000E94CC2EA10166E271E00E94D02F5C0104
:10A78000CC24B7FCC094DC2C0027F7FC0095102FDC
:10A79000AE0CBF1CC01ED11E82EC91E0A0E0B0E068
:10A7A00089839A83AB83BC83F201828193810E9467
:10A7B000CC2EA10160E271E00E94D02FAA2797FD64
:10A7C000A095BA2F680E791E8A1E9B1EF201828107
:10A7D00093810E94CC2EA10164E271E00E94D02FEF
:10A7E000AA2797FDA095BA2FA80EB91ECA1EDB1E78
:10A7F0006A0C7B1C8C1C9D1C6114710481049104E7
:10A8000019F480E090E002C08FEF9EEF24960FB61F
:10A81000F894DEBF0FBECDBFDF91CF911F910F9196
:10A82000FF90EF90DF90CF90BF90AF909F908F9070
:10A830007F906F905F904F903F902F900895089574
:10A84000CF93DF93FC01E45BFD4F20E030E0EC01AF
:10A85000C459DD4FDF0180819181009731F46D9300
:10A860007C93288380E090E00FC08617970719F447
:10A870008EEF9FEF09C02F5F3F4F12963296203127
:10A88000310549F78FEF9FEFDF91CF910895DC01FC
:10A89000A45BBD4F20E0ED91FC911197309751F0F2
:10A8A000808191818617970729F48281938184178B
:10A8B000950731F02F5F1296203169F7E0E0F0E064
:10A8C000CF010895DC01A657BD4F20E030E04FEFE7
:10A8D0005FEFFC01E758FD4F8C91882361F481E024
:10A8E000818B8089806F808B518340835383428327
:10A8F000158A168A09C02F5F3F4F779657962A30E0
:10A90000310551F72FEF3FEFC90108952FEF6F3F4A
:10A910007207D1F0FC01E558FD4F20E030E0DC018A
:10A92000A758BD4F8785853041F480819181861776
:10A93000970719F48D919C9108952F5F3F4F57967B
:10A9400077962A30310571F78FEF9FEF0895FC015C
:10A95000E758FD4F20E030E0DC01A558BD4F81896C
:10A96000853041F4808191818617970719F48D9184
:10A970009C9108952F5F3F4F579677962A30310567
:10A9800071F78FEF9FEF08958F929F92AF92BF92D2
:10A99000CF92DF92EF92FF920F93CF93DF93EC0170
:10A9A0004B015A016901CA5BDD4F28813981C654C8
:10A9B000D2402115310539F0809143089091440827
:10A9C0002817390721F0CE010D960E94E876033052
:10A9D00021F485E3E816F10421F0CE0109960E94E6
:10A9E000E87681E0F6018083000F000F0283E182A8
:10A9F000A114B10409F04501C401DF91CF910F9179
:10AA0000FF90EF90DF90CF90BF90AF909F908F908E
:10AA100008959C01FC01E459FD4F80818F3F39F07E
:10AA20008FEF8083C90183599D4F0E94DA76089584
:10AA30008F929F92AF92BF92CF92DF92EF92FF924E
:10AA40000F931F93CF93DF93EC017B014A016901C0
:10AA5000672B99F18DE6A82E82E0B82EAC0EBD1EB4
:10AA6000C5010E94E876F701D182C0821383028378
:10AA700013861286B701CE010E9420540097E9F098
:10AA8000FFEF8F3F9F0739F468EE73E080E090E0BE
:10AA90000E94260AEFCF8E5F9F4F61F7CE010E9482
:10AAA0001F54C5010E94DA76CE010D960E94DA7617
:10AAB00060E07FEF8FEF9FEF3BC0BE016F5E7F4F87
:10AAC000CE010E9428508C01CA5BDD4F288139815C
:10AAD000C654D2402115310539F080914308909138
:10AAE00044082817390721F0CE010D960E94DA7626
:10AAF0000115110531F0B801882777FD8095982F51
:10AB000017C0E114F10481F0892871F440E050E0AD
:10AB100060E070E0C7010A960E943D10F701648171
:10AB200075818681978104C060E070E080E090E0EC
:10AB3000DF91CF911F910F91FF90EF90DF90CF9019
:10AB4000BF90AF909F908F900895FF920F931F93A7
:10AB5000CF93DF93EC01F62E062F1127000F111F64
:10AB60000C0F1D1F045B1D4FD801ED91FC91248338
:10AB7000358346835783CF010A960E94AA0FD801D6
:10AB8000ED91FC9111978FEF9FEF938782871D9234
:10AB90001C92C459DD4F8881CC56D2408F1519F4D0
:10ABA000CE010E940955DF91CF911F910F91FF9027
:10ABB0000895FC019A01AB01E459FD4F6081EC5608
:10ABC000F2406F3F19F0CF010E94A55508956F9292
:10ABD0007F928F929F92AF92BF92CF92DF92EF922D
:10ABE000FF920F931F93CF93DF934C015B013A01C8
:10ABF00068017901EC01C45BDD4F2FEF3FEF00E00E
:10AC000010E0E881F9813097B9F08281938186154F
:10AC1000970591F48FEFA8168FEFB80629F0808181
:10AC200091818A159B0541F4A7019601602FC4010B
:10AC30000E94A55520E030E00F5F1F4F22960031A3
:10AC40001105F9F6C901DF91CF911F910F91FF9086
:10AC5000EF90DF90CF90BF90AF909F908F907F90BC
:10AC60006F9008951F93CF93DF93EC011FEF198B23
:10AC700061E070E009960E94FF76CF5EDE4F188398
:10AC8000C151D140FE01E45BFD4F80E01192119271
:10AC90008F5F8031D9F7DE01A758BD4F20E030E04B
:10ACA0004FEF5FEFBE0167577D4FFD01118A11968F
:10ACB0005C934E9353834283FB0180818F7C80831E
:10ACC0002F5F3F4F695E7F4F57962A30310569F7F6
:10ACD000CF58DD4F1882C157D24061E070E0CE01FD
:10ACE0000D960E94FF7660E070E0CE0183599D4F83
:10ACF0000E94FF76CE010E940955FE01ED5EFD4FD8
:10AD0000C75EDD4FD183C083C951D240CE01875C7D
:10AD10009D4FC95CDD4F99838883DF91CF911F914F
:10AD200008950F931F93CF93DF93EC018B01FB01E9
:10AD30004381442319F40E9409550AC055275095B0
:10AD400041955F4F662757FD6095762F0E94D95534
:10AD5000F80164817727CE0109960E94CD76DF91B4
:10AD6000CF911F910F9108953F924F925F926F92F2
:10AD70007F928F929F92AF92BF92CF92DF92EF928B
:10AD8000FF920F931F93CF93DF93CDB7DEB7269734
:10AD90000FB6F894DEBF0FBECDBF5C017B01FB0197
:10ADA00033968281382E369436949927D82ECC2427
:10ADB00081819927C82AD92A8FEF93E0C822D92206
:10ADC00093E0391609F4CCC0931538F0A1E03A1697
:10ADD00081F0A31508F455C021C3B5E03B1609F472
:10ADE00063C23B1608F4AAC1EFE33E1609F0FDC2A8
:10ADF000E5C2FCE0CF16D10409F43FC03DE0C31624
:10AE0000D10439F182E0C816D10409F0EEC218E489
:10AE1000812E12E0912E8A0C9B1CC4010E94847624
:10AE20004FEF5FEF64E071E0C5010E944754FC0101
:10AE3000892B59F004811581268137814FEF5FEF0F
:10AE400064E071E0C5010E94E755C4010E94DA7612
:10AE5000CCC24FEF5FEF64E07DE0C5010E94475434
:10AE600020E030E0DE011196F701379681918D9355
:10AE70002F5F3F4F26303105C9F7C5010E940955A4
:10AE8000B4C29DE0C916D10409F440C0AEE0CA16B0
:10AE9000D10450F4B9E0CB16D10481F0ECE0CE1629
:10AEA000D10409F0A2C219C0FEE0CF16D104E9F125
:10AEB0003FE0C316D10409F098C24BC0FB01808566
:10AEC0009927582E442487819927482A592A818511
:10AED000682E7724882499249FC2FB0180859927B6
:10AEE000582E442487819927482A592A8681882305
:10AEF00009F0CAC282859927982F88272185332790
:10AF0000822B932B3C0188249924C2C2FB018085AB
:10AF10009927582E442487819927482A592A8681BF
:10AF20009927909581959F4FAEC0FB01868188231C
:10AF300009F0A7C280859927982F88272781332772
:10AF4000822B932B3C01882499244FEF442E542EBE
:10AF50009FC2FB0186819927909581959F4F72C072
:10AF6000F7E1CF16D10409F464C038E1C316D10467
:10AF7000D0F489E0C816D10409F48BC09AE0C91650
:10AF8000D10430F4A3E0CA16D10409F02EC229C0BE
:10AF9000B4E1CB16D10409F483C0E5E1CE16D104A7
:10AFA00009F023C246C0F6E3CF16D10409F45AC013
:10AFB00037E3C316D10458F489E1C816D10409F463
:10AFC00068C093E2C916D10409F00FC215C0A7E307
:10AFD000CA16D104E9F1B4E4CB16D10409F005C2D4
:10AFE00028C0E5E4F2E0AE0EBF1ED5011C92EBEBEB
:10AFF000FDEFAE0EBF1EF9C1FB0180859927AA2780
:10B00000BB276624782E892E9A2E81859927AA2718
:10B01000BB27DC0199278827278133274427552719
:10B02000822B932BA42BB52B682A792A8A2A9B2A58
:10B03000DFC1F70180859927982F8827278133273B
:10B04000822B932B3C01882477FC8094982CD0C1D0
:10B05000FB0180859927582E442487819927482A07
:10B06000592AD7C1FB0180859927582E442487810E
:10B070009927482A592A82859927982F8827218538
:10B080003327822B932B3C01882477FC8094982CC7
:10B09000C3C1F7018781682E772488249924A8C129
:10B0A0004FEF5FEF6CE074E1C5010E9447549C01D3
:10B0B000FC010085118584819581A681B781893F36
:10B0C0009105A105B10544F088EF90E0A0E0B0E063
:10B0D00084839583A683B7836624772410C0492C84
:10B0E0005524D201AE0DBF1DFD018781400E511EBA
:10B0F000D2018C930894611C711C882379F0962CE2
:10B10000462D552766277727F90184819581A681E9
:10B11000B781481759076A077B070CF3F901848147
:10B120009581A681B781481759076A077B0709F4FB
:10B130009A94090D111DD8011C9257C1B3E0CB168A
:10B14000D10409F44AC0E4E0CE16D10430F4F1E0B1
:10B15000CF16D10409F049C10BC035E0C316D104A4
:10B1600009F452C089E0C816D10409F03EC185C077
:10B170004FEF5FEF60E171E0C5010E944754FC01B1
:10B18000A085B185F70187818C9320853327818540
:10B190009927982F8827282B392BFD01328321836B
:10B1A000F7018285FD018383F70123853327848599
:10B1B0009927982F8827282B392BFD013583248345
:10B1C000F7012585332786859927982F8827282BEF
:10B1D000392BFD013783268308C14FEF5FEF60E114
:10B1E00073E0C5010E944754FC0140855185D70199
:10B1F00014969A01285F3F4F8D91FA018193AF0118
:10B20000E217F307C9F7F1C083E292E0A80EB91E76
:10B21000FB0180859927982F882727813327822B48
:10B22000932BD5018D939C93EFE1F0E0AE0EBF1E02
:10B23000F7018185D5018C93EEEBFDEFAE0EBF1EBD
:10B24000F70163857727762F662782859927682BF4
:10B25000792BC501815E9D4F0E94CD76F7016585F2
:10B260007727762F662784859927682B792BC50148
:10B27000825C9D4F0E94CD76B8C04FEF5FEF60E1DA
:10B2800079E0C5010E944754FC0140855185D701F2
:10B2900017969A012A5F3F4F8D91FA018193AF0172
:10B2A000E217F307C9F7A1C0F5E0CF16D10419F1F1
:10B2B00037E0C316D10409F440C083E0C816D104B6
:10B2C00009F0ACC0FB0180859927582E4424878162
:10B2D0009927482A592AB201C5010E948654AC0117
:10B2E00064E173E0C5010E944754FC01A085B1856B
:10B2F000F70181858DC0FB0180859927582E442454
:10B3000087819927482A592AB201C5010E9486548B
:10B31000AC0164E175E0C5010E944754FC01A085C1
:10B32000B185F70182859927982F882721853327B2
:10B33000822B932B8D939C936CC04FEF5FEF64E156
:10B3400077E0C5010E944754FC01A085B1851097A4
:10B3500029F0F701858599278D939C93F7018285C4
:10B360009927AA27BB276624782E892E9A2E248512
:10B37000332744275527522F4427332722278385F5
:10B380009927AA27BB27DC0199278827282B392B47
:10B390004A2B5B2B81859927AA27BB27282B392B82
:10B3A0004A2B5B2B622A732A842A952A62E0660C58
:10B3B000771C881C991C6A95D1F71AC0F2E1CF1648
:10B3C000D10499F4F501E45BFD4F20E00081118187
:10B3D0000115110531F0D8018D919C918C5F92413E
:10B3E00059F02F5F3296203189F766247724430184
:10B3F0005FEF452E552E10C0F80162817381C501A3
:10B400000E94A7542C01F801A085B185F70187811E
:10B410008C9366247724430111E007C066247724C7
:10B4200043014FEF442E542E10E0F701868188230C
:10B4300049F09927909581959F4F3C01882477FC8E
:10B440008094982CFFEF4F16FFEF5F0619F44FEF33
:10B450005FEF05C0B201C5010E948654AC01112303
:10B46000C9F07C2D6627832D9927880F991F880F97
:10B47000991F682B792B94018301C5010E94E75520
:10B4800009C08FEF482E582EF701868111E0D1CFE9
:10B4900011E0D8CFF70163817727C50109960E9493
:10B4A000CD7626960FB6F894DEBF0FBECDBFDF91E6
:10B4B000CF911F910F91FF90EF90DF90CF90BF90B1
:10B4C000AF909F908F907F906F905F904F903F9044
:10B4D00008952F923F924F925F926F927F928F9238
:10B4E0009F92AF92BF92CF92DF92EF92FF920F9313
:10B4F0001F93CF93DF93CDB7DEB72A970FB6F8949B
:10B50000DEBF0FBECDBF6C014B01FB0181818331DA
:10B5100009F459C0843128F5853009F427C38630F1
:10B5200078F4823009F489C0833020F4813009F046
:10B5300040C057C0833009F4AEC18430D1F57EC21B
:10B540008F3009F4FBC3803130F4873009F48AC3AB
:10B550008E3079F5EFC3803109F4DEC5823149F5CB
:10B5600036C08B3109F4D8C58C3170F4863109F4BA
:10B570001CC5873118F48431E1F41FC0873109F408
:10B5800024C58831B1F4C8C5823209F456C083326B
:10B5900030F48C3109F429C58D3159F44CC58F3EF6
:10B5A00019F08F3F31F419C08B0181E0E82EF12CA6
:10B5B0008BC58401EE24FF2498C5D601A558BD4F44
:10B5C00060E070E086C48B01EE24FF247BC4D601CA
:10B5D000A358BD4F20E030E0B5C38B01EE24FF241B
:10B5E00062C5FB010381002379F0112710950195B5
:10B5F0001F4F222717FD2095322F4FEF5FEF64E09A
:10B6000071E0C6010E94E7554FEF5FEF64E071E023
:10B61000C6010E944754FC010481158126813781AF
:10B620004FEF5FEF64E071E0C6010E94E755C6018D
:10B63000885B9D4F0E94DA766FC54FEF5FEF64E045
:10B6400071E0C6010E9447548C01FC01E084F18442
:10B65000B401AA24BB2418861F82B1E12B2E312C01
:10B66000280C391C02C1F801848195818A0D9B1D2B
:10B670002FE030E0829FD001839FB00D929FB00DEC
:10B680001124EF81F885E80DF91DAE0DBF1D34962C
:10B6900086E001900D928150E1F7F8018481958157
:10B6A0008A0D9B1DAFE06A2E712C869DD001879D6F
:10B6B000B00D969DB00D1124AE0DBF1DFB019285FE
:10B6C0009F70FD018681807F892B8683F8018481AC
:10B6D00095818A0D9B1D869DD001879DB00D969DFD
:10B6E000B00D1124AE0DBF1DFB0193859295907F87
:10B6F000FD0186818F70892B8683F4018181F80199
:10B7000044815581FB0195855684823209F052C0EF
:10B710004A0D5B1D469D9001479D300D569D300D95
:10B7200011242E0D3F1D3A8729872485332744276E
:10B730005527892F9927AA27BB27BA2FA92F982FDA
:10B740008827282B392B4A2B5B2B852D9927AA2755
:10B75000BB27DC0199278827282B392B4A2B5B2B09
:10B76000E985FA852783308741875287F8018481EC
:10B7700095818A0D9B1D869DD001879DB00D969D5C
:10B78000B00D1124AE0DBF1DFB0120893327322FD0
:10B790002227878599279068282B392BFD0134872C
:10B7A0002387F1018081992787FD9095FD01968778
:10B7B00085874CC04A0D5B1D469D9001479D300D0D
:10B7C000569D300D11242E0D3F1D3A872987292FB4
:10B7D000332744275527852D9927AA27BB27BA2F1A
:10B7E000A92F982F8827282B392B4A2B5B2BFB015D
:10B7F00087859927AA27BB27DC0199278827282B2B
:10B80000392B4A2B5B2BE985FA85278330874187C3
:10B810005287F801848195818A0D9B1D869DD001F8
:10B82000879DB00D969DB00D1124AE0DBF1DFB017F
:10B8300021893327322F2227808999279068282B46
:10B84000392BFD0134872387168615860894A11CA1
:10B85000B11C2F813885225F3F4F38872F838EE0C0
:10B8600090E0280E391E625F7F4FF4012381822F02
:10B870009927A816B9060CF4F6CEF80184819581B3
:10B88000A681B781820F911DA11DB11D848395836F
:10B89000A683B78341C48B010A5F1F4FDE01119657
:10B8A000F80186E001900D928150E1F7A9817A813B
:10B8B0006B815C814D819E81F601E358FD4F20E054
:10B8C00030E08585882391F080818A1779F4818121
:10B8D000871761F48281861749F48381851731F4D3
:10B8E0008481841719F48581891739F02F5F3F4FC0
:10B8F00077962A30310529F701C487E190E0289F27
:10B90000D001299FB00D389FB00D1124A758BD4F0D
:10B91000AC0DBD1DED90FC90119734C0C6010E9486
:10B9200062549C0197FDF8C387E190E0289FD00105
:10B93000299FB00D389FB00D1124A758BD4FAC0DF5
:10B94000BD1DCD010496A80126E0FA010190AF01CA
:10B95000FC010192CF012150C1F784E0FD01818BF0
:10B96000809188089091890811969C938E930196F6
:10B970009093890880938808019720892F7C206103
:10B98000208B7C01FD017189872F8350F401938105
:10B99000823008F045C0992361F0FD01118A8FEFD4
:10B9A0009FEF8D939C9393838283F40183819927E6
:10B9B00039C085E0FD01818BF40124813327858125
:10B9C0009927982F8827282B392BFD013383228331
:10B9D000F40194859F70FD018089807F892B808B85
:10B9E000128A86010B581D4F27E732E0C20ED31E84
:10B9F000F6012081318189E89DEFC80ED91E4D9155
:10BA00005C9160E0733009F461E081E06827D8015F
:10BA1000ED91FC9182E009958701222733270AC026
:10BA2000892F9927909581959F4F8C01222717FD8B
:10BA30002095322FA70164E075E004C1E2E6F3E04F
:10BA4000CE0EDF1ED6018D919C91EEE9FCEFCE0E5D
:10BA5000DF1E892B09F460C38B010D5F1F4FDE01D0
:10BA60001196F80186E001900D928150E1F7F40102
:10BA7000E184F284B384C6010E946254AC018F5FFA
:10BA80009F4F09F449C387E190E0489FD001499F47
:10BA9000B00D589FB00D1124A358BD4FAC0DBD1D66
:10BAA000C80126E0FC010190CF010D922150D1F791
:10BAB00087E190E0489F3001499F700C589F700CBF
:10BAC00011246C0C7D1C25E832E0620E731E2E2DB5
:10BAD0003327442755278F2D9927AA27BB27BA2F0D
:10BAE000A92F982F8827282B392B4A2B5B2B8B2D9E
:10BAF0009927AA27BB27DC0199278827282B392BD0
:10BB00004A2B5B2BD3012D933D934D935C9313975D
:10BB1000EBE7FDEF6E0E7F1ED301A757BD4FF4017B
:10BB200094859F708C91807F892B8C93809188085D
:10BB30009091890829E732E0620E731EF301918328
:10BB400080830196909389088093880821E130E0F2
:10BB5000620E731E82E0F30181938C918F7C806171
:10BB60008C931082F601EF58FD4F2BC2FB018581AB
:10BB70009927582F442784819927482B592BD60180
:10BB8000A558BD4F60E070E0E9E7AE2EE2E0BE2EC2
:10BB9000AC0CBD1C9501FD018785882371F08D914A
:10BBA0009C9111978417950741F4D901ED90FC9071
:10BBB000F4010381002371F049C06F5F7F4F87E17B
:10BBC00090E0A80EB91E295E3F4F57966A30710566
:10BBD00011F7A2C2F501118A8FEF9FEF9383828341
:10BBE0009183808380898F7C808BF601EB58FD4F99
:10BBF00027E732E0C20ED31ED6012D913C9189E891
:10BC00009DEFC80ED91EA081B181A701F401668104
:10BC100083E0FD010995F401038111271095019539
:10BC20001F4F222717FD2095322FA70164E076E0F1
:10BC3000C6010E94E75506EF1EEF2FEF3FEFA70169
:10BC40006FEF7FEFC6010E94E75566C2112710957E
:10BC500001951F4F222717FD2095322FA70164E081
:10BC600076E0F0CF4FEF5FEF64E079E1C6010E942C
:10BC700047547C01FC014084518484819581A681D4
:10BC8000B781893F9105A105B10544F088EF90E0A7
:10BC9000A0E0B0E084839583A683B783540100E0DD
:10BCA00010E020E030E011C0F5018285F201E40FE0
:10BCB000F51F80838A019B010F5F1F4F2F4F3F4F5E
:10BCC0000894A11CB11C882369F03801B901A801AE
:10BCD000F70184819581A681B781481759076A07C2
:10BCE0007B0714F3F70184819581A681B7814817FA
:10BCF00059076A077B0719F4089461087108460C14
:10BD0000571CD2011C92F4010381002349F0112732
:10BD1000109501951F4F222717FD2095322F05C042
:10BD20008301222717FD2095322F4FEF5FEF64E04C
:10BD300079E188CFC6010E94B456EEC1C6010E94C7
:10BD40009156EAC1A4014D5F5F4F9C91FA01818138
:10BD50009817F1F4FD019181FA0182819817C1F4DD
:10BD6000FD019281FA018381981791F4FD0193817D
:10BD7000FA018481981761F4FD019481FA018581AB
:10BD8000981731F4FD019581FA018681981739F0F1
:10BD90002F5F3F4F57962A303105A1F6BDC187E18D
:10BDA00090E0289F7001299FF00C389FF00C11241F
:10BDB000EC0CFD1C29E732E0E20EF31ED701AD903A
:10BDC000BC90E7E8FDEFEE0EFF1EF40103810023B7
:10BDD00051F01127109501951F4F222717FD20952F
:10BDE000322FA501ABC0D701A757BD4FF4019285F3
:10BDF00093709295907F8C918F7C892B8C93028588
:10BE0000112722273327A50168E07BE0C6010E94A5
:10BE1000E7552AE832E0E20EF31ED7018C91853017
:10BE200009F07AC1F601EB58FD4F27E732E0C20E68
:10BE3000D31ED6012D913C9189E89DEFC80ED91EE5
:10BE4000A081B181A50160E0F4018285FD01099521
:10BE500063C1F80167817727762F66278681992746
:10BE6000682B792BC601815E9D4F0E94BE76F8013A
:10BE700085819927382F222784819927282B392BD0
:10BE8000D601A558BD4F40E050E0B60162577D4F46
:10BE90008D919C9111978217930739F4F80196813F
:10BEA000DB018C91891B8C9308C04F5F5F4F695EEB
:10BEB0007F4F57964A30510559F70894E11CF11C01
:10BEC0000C5F1F4FF40183819927E816F9060CF2E5
:10BED00023C18D919C9111975796F40125813327A9
:10BEE000322F222744815527242B352B3F70821770
:10BEF000930731F06F5F7F4F6A30710551F70CC1C6
:10BF000087E190E0689FD001699FB00D789FB00DE8
:10BF10001124AC0DBD1DA758BD4F4D915C911197DB
:10BF2000A957B240F4010381002359F0112710955D
:10BF300001951F4F222717FD2095322F68E07BE0E7
:10BF400081CEA557BD4FF40186818D9386818823CC
:10BF500059F080859927982F882727813327822BAE
:10BF6000932B8D939C9302C01D921C9287E190E0CD
:10BF7000689FF001699FF00D789FF00D1124EC0D82
:10BF8000FD1DE457FD4F0081118122273327322FF9
:10BF9000212F102F0027F40186819927AA27BB277C
:10BFA000082B192B2A2B3B2B4BCEDE011196FB01C4
:10BFB000339686E001900D928150E1F7F601EE583C
:10BFC000FD4F80818F5F8083A7C0DE011196FB014A
:10BFD000339686E001900D928150E1F7BE016F5FCC
:10BFE0007F4FC6010E94AC6D97C0FB01658177272A
:10BFF000762F662784819927682B792BC6010E94AA
:10C000008654AC01F4010381002329F01127109517
:10C0100001951F4F09C0F40107811127102F002738
:10C0200086819927082B192B222717FD2095322F5F
:10C0300064E07FE107CEFB0165817727762F6627D5
:10C0400084819927682B792BC6010E948654AC0104
:10C05000F4010381002329F01127109501951F4F4A
:10C0600009C0F40107811127102F00278681992725
:10C07000082B192B222717FD2095322F64E07FE033
:10C08000E1CDF801828199279F938F9387EB97E009
:10C090009F938F930E943D770894E11CF11C0F90B1
:10C0A0000F900F900F900F5F1F4FF401828199271F
:10C0B000E816F90634F330C0F801838199270E940D
:10C0C0005D770894E11CF11C0F5F1F4FF401828122
:10C0D0009927E816F90684F31FC0F8018281992791
:10C0E0000E945D770894E11CF11C0F5F1F4FF40163
:10C0F00082819927E816F90684F30EC0E2E6F3E0A0
:10C10000CE0EDF1ED6018D919C91EEE9FCEFCE0E96
:10C11000DF1E892B09F402CC21E131E0C20ED31ECF
:10C120008FEFD6018C932A960FB6F894DEBF0FBE20
:10C13000CDBFDF91CF911F910F91FF90EF90DF90D6
:10C14000CF90BF90AF909F908F907F906F905F90B7
:10C150004F903F902F9008958F929F92AF92BF92F1
:10C16000CF92DF92EF92FF920F931F93CF93DF93C3
:10C17000CDB7DEB72C970FB6F894DEBF0FBECDBF9C
:10C180006C014B01142F9CE6A92E93E0B92EAC0C48
:10C19000BD1C96012F5E3F4F83E4E82EF12C03E097
:10C1A000AB01BE016F5F7F4FC6010E94C4547C018A
:10C1B000F50180899189892B39F481E090E00E9412
:10C1C000000CF501918B808BF501A089B1891C933E
:10C1D00081E0F601848B158B0FEF1FEF2CE033E429
:10C1E000A401B701C6010E9418552C960FB6F89409
:10C1F000DEBF0FBECDBFDF91CF911F910F91FF909A
:10C20000EF90DF90CF90BF90AF909F908F90089568
:10C21000AF92BF92CF92DF92EF92FF920F931F9354
:10C22000CF93DF93CDB7DEB72C970FB6F894DEBF70
:10C230000FBECDBF6C015B019C012F5E3F4F42E4FE
:10C24000E42EF12C03E0AB01BE016F5F7F4F0E9433
:10C25000C454F601148A0FEF1FEF2CE032E4A5015D
:10C26000BC01C6010E9418552C960FB6F894DEBF8B
:10C270000FBECDBFDF91CF911F910F91FF90EF9037
:10C28000DF90CF90BF90AF9008958F929F92AF9222
:10C29000BF92CF92DF92EF92FF920F931F93CF93B3
:10C2A000DF93CDB7DEB72C970FB6F894DEBF0FBE85
:10C2B000CDBF6C014B01142F6CE6A62E63E0B62EA9
:10C2C000A80EB91E9C012F5E3F4F55E4E52EF12CC0
:10C2D00003E0A401BE016F5F7F4F0E94C4547C0144
:10C2E000F50186859785892B39F481E090E00E94DD
:10C2F000000CF50197878687F501A685B7851C9305
:10C3000081E0F601848B158B0FEF1FEF2CE035E4F5
:10C31000A401B701C6010E9418552C960FB6F894D7
:10C32000DEBF0FBECDBFDF91CF911F910F91FF9068
:10C33000EF90DF90CF90BF90AF909F908F90089537
:10C34000AF92BF92CF92DF92EF92FF920F931F9323
:10C35000CF93DF93CDB7DEB72C970FB6F894DEBF3F
:10C360000FBECDBF6C015B019C012F5E3F4F74E49B
:10C37000E72EF12C03E0A501BE016F5F7F4F0E9405
:10C38000C454F601148A0FEF1FEF2CE034E4A5012A
:10C39000BC01C6010E9418552C960FB6F894DEBF5A
:10C3A0000FBECDBFDF91CF911F910F91FF90EF9006
:10C3B000DF90CF90BF90AF9008952F923F924F9211
:10C3C0005F926F927F928F929F92AF92BF92CF9225
:10C3D000DF92EF92FF920F931F93CF93DF93CDB72E
:10C3E000DEB72D970FB6F894DEBF0FBECDBF6C0140
:10C3F0001B014A012D87380127018CE6A82E83E016
:10C40000B82EAC0CBD1C96012F5E3F4F03E3E02E0F
:10C41000F12C03E0AB01BE016F5F7F4FC6010E94AC
:10C42000C4547C01F50184859585892B39F487E016
:10C4300090E00E94000CF50195878487F501A485A2
:10C44000B58511969C928E928D85FD018283F501B2
:10C45000A485B585FD01748263825682458287E09A
:10C46000F601848B858A892D9927868B8D85878B0C
:10C47000608E872D9927818F428E852D9927838FF6
:10C480000FEF1FEF2CE033E3A101B701C6010E94BB
:10C4900018552D960FB6F894DEBF0FBECDBFDF91B5
:10C4A000CF911F910F91FF90EF90DF90CF90BF90B1
:10C4B000AF909F908F907F906F905F904F903F9044
:10C4C0002F9008958F929F92AF92BF92CF92DF925A
:10C4D000EF92FF920F931F93CF93DF93CDB7DEB709
:10C4E0002C970FB6F894DEBF0FBECDBF6C014B0189
:10C4F000142F2CE6A22E23E0B22EA80EB91E9C010A
:10C500002F5E3F4F91E3E92EF12C03E0AB01BE011A
:10C510006F5F7F4FC6010E94C4547C01F501828584
:10C520009385892B39F481E090E00E94000CF5019D
:10C5300093878287F501A285B3851C9381E0F6017C
:10C54000848B158B0FEF1FEF2CE031E3A401B701B3
:10C55000C6010E9418552C960FB6F894DEBF0FBE88
:10C56000CDBFDF91CF911F910F91FF90EF90DF90A2
:10C57000CF90BF90AF909F908F9008954F925F9211
:10C580006F927F928F929F92AF92BF92CF92DF92E3
:10C59000EF92FF920F931F93CF93DF93CDB7DEB748
:10C5A0002C970FB6F894DEBF0FBECDBF6C012B01E8
:10C5B00049015A016CE6662E63E0762E680E791EFC
:10C5C0009C012F5E3F4F54E2E52EF12C03E0A201C7
:10C5D000BE016F5F7F4F0E94C4547C01F3018289CA
:10C5E0009389892B39F484E090E00E94000CF301D8
:10C5F000938B828BF301A289B3898D929D92AD9228
:10C60000BC92139783E0F601848B858ABB27AB2D00
:10C610009A2D892D868BC501AA27BB27878B0FEF03
:10C620001FEF2CE034E2A201B701C6010E941855A9
:10C630002C960FB6F894DEBF0FBECDBFDF91CF9121
:10C640001F910F91FF90EF90DF90CF90BF90AF9030
:10C650009F908F907F906F905F904F900895AF92D2
:10C66000BF92CF92DF92EF92FF920F931F93CF93DF
:10C67000DF93CDB7DEB72C970FB6F894DEBF0FBEB1
:10C68000CDBF6C015B019C012F5E3F4F73E2E72E33
:10C69000F12C03E0A501BE016F5F7F4F0E94C454DF
:10C6A000F601148A0FEF1FEF2CE033E2A501BC0165
:10C6B000C6010E9418552C960FB6F894DEBF0FBE27
:10C6C000CDBFDF91CF911F910F91FF90EF90DF9041
:10C6D000CF90BF90AF9008958F929F92AF92BF92EC
:10C6E000CF92DF92EF92FF920F931F93CF93DF933E
:10C6F000CDB7DEB72C970FB6F894DEBF0FBECDBF17
:10C700006C014B01142FFCE6AF2EF3E0BF2EA80EF8
:10C71000B91E9C012F5E3F4FEAE1EE2EF12C03E0A3
:10C72000AB01BE016F5F7F4F0E94C4547C01F501D5
:10C73000828D938D892B39F481E090E00E94000C6A
:10C74000F501938F828FF501A28DB38D1C9381E04B
:10C75000F601848B158B0FEF1FEF2CE03AE1A4015B
:10C76000B701C6010E9418552C960FB6F894DEBF8B
:10C770000FBECDBFDF91CF911F910F91FF90EF9032
:10C78000DF90CF90BF90AF909F908F900895AF9221
:10C79000BF92CF92DF92EF92FF920F931F93CF93AE
:10C7A000DF93CDB7DEB72C970FB6F894DEBF0FBE80
:10C7B000CDBF6C015B019C012F5E3F4FA9E1EA2ECA
:10C7C000F12C03E0AB01BE016F5F7F4F0E94C454A8
:10C7D000F601148A0FEF1FEF2CE039E1A501BC012F
:10C7E000C6010E9418552C960FB6F894DEBF0FBEF6
:10C7F000CDBFDF91CF911F910F91FF90EF90DF9010
:10C80000CF90BF90AF9008956F927F928F929F923A
:10C81000AF92BF92CF92DF92EF92FF920F931F934E
:10C82000CF93DF93CDB7DEB72C970FB6F894DEBF6A
:10C830000FBECDBF6C013B014A010CE6A02E03E008
:10C84000B02EA80EB91E9C012F5E3F4F18E1E12EBD
:10C85000F12C03E0AB01BE016F5F7F4F0E94C45417
:10C860007C01F50186899789892B39F482E090E073
:10C870000E94000CF501978B868BF501A689B7897C
:10C880008D929C9282E0F601848B858A892D99276E
:10C89000868B0FEF1FEF2CE038E1A301B701C60133
:10C8A0000E9418552C960FB6F894DEBF0FBECDBF70
:10C8B000DF91CF911F910F91FF90EF90DF90CF907C
:10C8C000BF90AF909F908F907F906F900895AF92A0
:10C8D000BF92CF92DF92EF92FF920F931F93CF936D
:10C8E000DF93CDB7DEB72C970FB6F894DEBF0FBE3F
:10C8F000CDBF6C015B019C012F5E3F4F87E1E82EAD
:10C90000F12C03E0AB01BE016F5F7F4FC6010E94B7
:10C91000C454F601148A0FEF1FEF2CE037E1A50194
:10C92000BC01C6010E9418552C960FB6F894DEBFC4
:10C930000FBECDBFDF91CF911F910F91FF90EF9070
:10C94000DF90CF90BF90AF9008956F927F928F92BB
:10C950009F92AF92BF92CF92DF92EF92FF920F938E
:10C960001F93CF93DF93CDB7DEB72C970FB6F89414
:10C97000DEBF0FBECDBF6C013B014A015CE6A52EB8
:10C9800053E0B52EA80EB91E9C012F5E3F4F46E125
:10C99000E42EF12C03E0AB01BE016F5F7F4F0E94DC
:10C9A000C4547C01F50182819381892B39F482E0A2
:10C9B00090E00E94000CF50193838283F501A2812F
:10C9C000B3818D929C9282E0F601848B858A892DB9
:10C9D0009927868B0FEF1FEF2CE036E1A301B701FB
:10C9E000C6010E9418552C960FB6F894DEBF0FBEF4
:10C9F000CDBFDF91CF911F910F91FF90EF90DF900E
:10CA0000CF90BF90AF909F908F907F906F90089540
:10CA1000AF92BF92CF92DF92EF92FF920F931F934C
:10CA2000CF93DF93CDB7DEB72C970FB6F894DEBF68
:10CA30000FBECDBF6C015B019C012F5E3F4F65E1D6
:10CA4000E62EF12C03E0A501BE016F5F7F4F0E942F
:10CA5000C454F601148A0FEF1FEF2CE035E1A50155
:10CA6000BC01C6010E9418552C960FB6F894DEBF83
:10CA70000FBECDBFDF91CF911F910F91FF90EF902F
:10CA8000DF90CF90BF90AF9008954F925F926F92DA
:10CA90007F928F929F92AF92BF92CF92DF92EF924E
:10CAA000FF920F931F93CF93DF93CDB7DEB72C97F1
:10CAB0000FB6F894DEBF0FBECDBF4C012B013A017B
:10CAC000A22E9C012F5E3F4F74E1E72EF12C03E074
:10CAD000A201BE016F5F7F4F0E94C454FC017186AA
:10CAE0006086BB24CC24DD24A482B582C682D78292
:10CAF000F401148A0FEF1FEF2CE034E1A201BC0116
:10CB0000C4010E9418552C960FB6F894DEBF0FBED4
:10CB1000CDBFDF91CF911F910F91FF90EF90DF90EC
:10CB2000CF90BF90AF909F908F907F906F905F90CD
:10CB30004F9008958F929F92AF92BF92CF92DF92C3
:10CB4000EF92FF920F931F93CF93DF93CDB7DEB792
:10CB50002C970FB6F894DEBF0FBECDBF6C014B0112
:10CB6000142FFCE6AF2EF3E0BF2EA80EB91E9C01D9
:10CB70002F5E3F4FEAE0EE2EF12C03E0AB01BE0149
:10CB80006F5F7F4F0E94C4547C01F501808D918DB1
:10CB9000892B39F481E090E00E94000CF501918F1F
:10CBA000808FF501A08DB18D1C9381E0F601848BFF
:10CBB000158B0FEF1FEF2CE03AE0A401B701C6017F
:10CBC0000E9418552C960FB6F894DEBF0FBECDBF4D
:10CBD000DF91CF911F910F91FF90EF90DF90CF9059
:10CBE000BF90AF909F908F900895AF92BF92CF92D9
:10CBF000DF92EF92FF920F931F93CF93DF93CDB706
:10CC0000DEB72C970FB6F894DEBF0FBECDBF6C0118
:10CC10005B019C012F5E3F4FA9E0EA2EF12C03E05F
:10CC2000AB01BE016F5F7F4F0E94C454F601148AAE
:10CC30000FEF1FEF2CE039E0A501BC01C6010E94F7
:10CC400018552C960FB6F894DEBF0FBECDBFDF91FE
:10CC5000CF911F910F91FF90EF90DF90CF90BF90F9
:10CC6000AF900895AF92BF92CF92DF92EF92FF9272
:10CC70000F931F93CF93DF93CDB7DEB72C970FB6EB
:10CC8000F894DEBF0FBECDBF6C015B01FC01EB5B16
:10CC9000FD4F8081882329F06BEF7EEF8FEF9FEFB0
:10CCA0001BC081E0808396012F5E3F4FB3E0EB2EE7
:10CCB000F12C03E0AB01BE016F5F7F4FC6010E9404
:10CCC000C454F601148A0FEF1FEF2CE033E0A501E6
:10CCD000BC01C6010E9418552C960FB6F894DEBF11
:10CCE0000FBECDBFDF91CF911F910F91FF90EF90BD
:10CCF000DF90CF90BF90AF9008952F923F924F92C8
:10CD00005F926F927F928F929F92AF92BF92CF92DB
:10CD1000DF92EF92FF920F931F93CF93DF93CDB7E4
:10CD2000DEB72E970FB6F894DEBF0FBECDBF6C01F5
:10CD30007E876D8729013A01470158015CE6252E5F
:10CD400053E0352E280E391E9C012F5E3F4F41E0E7
:10CD5000E42EF12C03E0AB01BE016F5F7F4F0E9418
:10CD6000C4547C01F10180859185892B39F488E0D8
:10CD700090E00E94000CF10191878087F101A0856D
:10CD8000B1854D925D926D927C921397FD018482E4
:10CD90009582A682B78288E0F601848B858ABB27BC
:10CDA000AB2D9A2D892D868BC501AA27BB27878B92
:10CDB0008B2D9927AA27BB27808F418EBB27A72DB4
:10CDC000962D852D828FC301AA27BB27838F872DA0
:10CDD0009927AA27BB27848F0FEF1FEF2CE031E0A4
:10CDE0004D855E85B701C6010E9418552E960FB677
:10CDF000F894DEBF0FBECDBFDF91CF911F910F9191
:10CE0000FF90EF90DF90CF90BF90AF909F908F906A
:10CE10007F906F905F904F903F902F9008954F922A
:10CE20005F926F927F928F929F92AF92BF92CF92BA
:10CE3000DF92EF92FF920F931F93CF93DF93CDB7C3
:10CE4000DEB72C970FB6F894DEBF0FBECDBF6C01D6
:10CE50002B013A014901BA010E94A7545C018FEFEE
:10CE6000A8168FEFB80629F46DEF7EEF8FEF9FEFD6
:10CE700021C096012F5E3F4FE7E3EE2EF12C03E039
:10CE8000A201BE016F5F7F4FC6010E94C45424E01F
:10CE9000F601248BA58A2B2D3327268B878A292DF3
:10CEA0003327208F83012CE037E3A201BC01C601A8
:10CEB0000E9418552C960FB6F894DEBF0FBECDBF5A
:10CEC000DF91CF911F910F91FF90EF90DF90CF9066
:10CED000BF90AF909F908F907F906F905F904F909A
:10CEE00008956F927F928F929F92AF92BF92CF924E
:10CEF000DF92EF92FF920F931F93CF93DF93CDB703
:10CF0000DEB72C970FB6F894DEBF0FBECDBF6C0115
:10CF10003B014A01BA010E94A7545C018FEFA81699
:10CF20008FEFB80629F46DEF7EEF8FEF9FEF1DC0F6
:10CF300096012F5E3F4FB6E3EB2EF12C03E0A301E9
:10CF4000BE016F5F7F4FC6010E94C45422E0F6010C
:10CF5000248BA58A2B2D3327268B84012CE036E3E6
:10CF6000A301BC01C6010E9418552C960FB6F89477
:10CF7000DEBF0FBECDBFDF91CF911F910F91FF900C
:10CF8000EF90DF90CF90BF90AF909F908F907F9069
:10CF90006F9008956F927F928F929F92AF92BF92FF
:10CFA000CF92DF92EF92FF920F931F93CF93DF9375
:10CFB000CDB7DEB72C970FB6F894DEBF0FBECDBF4E
:10CFC0006C013B014A010E94A7545C018FEFA81637
:10CFD0008FEFB80629F46DEF7EEF8FEF9FEF26C03D
:10CFE00096012F5E3F4F85E3E82EF12C03E040E0F1
:10CFF00050E0BE016F5F7F4FC6010E94C45485E0C0
:10D00000F601848B81E0858BA68A8B2D9927878BEF
:10D01000808E892D9927818F83012CE035E340E0B4
:10D0200050E060E070E0C6010E9418552C960FB6E3
:10D03000F894DEBF0FBECDBFDF91CF911F910F914E
:10D04000FF90EF90DF90CF90BF90AF909F908F9028
:10D050007F906F9008956F927F928F929F92AF9280
:10D06000BF92CF92DF92EF92FF920F931F93CF93D5
:10D07000DF93CDB7DEB72C970FB6F894DEBF0FBEA7
:10D08000CDBF6C013B015A012CE6822E23E0922E8B
:10D09000880E991E9C012F5E3F4F93E1E92EF12CE3
:10D0A00003E0AB01BE016F5F7F4FC6010E94C45415
:10D0B0007C01F40184899589892B59F489EF90E0EA
:10D0C0000E94000CDC01F401958B848BA850BF4FAB
:10D0D0001C92F50101900020E9F73197EA19FB094C
:10D0E000E83FF10518F049EF50E003C0AF014F5F92
:10D0F0005F4FB501F401848995890E94157A88EF04
:10D10000F601848BF50120E030E0D6015596922F90
:10D1100080818D938081882351F09F5F2F5F3F4FE7
:10D120003196283F310599F7983F09F497EFF601BA
:10D13000E90FF11D158A0FEF1FEF2CE033E1A3017A
:10D14000B701C6010E9418552C960FB6F894DEBFA1
:10D150000FBECDBFDF91CF911F910F91FF90EF9048
:10D16000DF90CF90BF90AF909F908F907F906F9007
:10D1700008958F929F92AF92BF92CF92DF92EF92DB
:10D18000FF920F931F93CF93DF93CDB7DEB72C970A
:10D190000FB6F894DEBF0FBECDBF6C014B015A0134
:10D1A0009C012F5E3F4F45E0E42EF12C03E0AB01E4
:10D1B000BE016F5F7F4F0E94C4547C01F501408126
:10D1C00055274F5F5F4FB501C60144960E94157AFF
:10D1D0000FEF1FEF2CE035E0A401B701C6010E945C
:10D1E00018552C960FB6F894DEBF0FBECDBFDF9159
:10D1F000CF911F910F91FF90EF90DF90CF90BF9054
:10D20000AF909F908F900895AF92BF92DF92EF9270
:10D21000FF920F931F93CF93DF93CDB7DEB7229783
:10D220000FB6F894DEBF0FBECDBFAE84BF84DA88E0
:10D23000BCE6EB2EB3E0FB2EEA0CFB1CCE014396C2
:10D240009A838983F70186819781892B39F48CE051
:10D2500090E00E94000CF70197838683F701868196
:10D260009781DC011196FC01D182BD016F5F7F4F78
:10D27000F7012681378181E0F90180838D2D81506E
:10D28000823008F069C0E981FA813296FA83E98335
:10D2900032978081FD0181836F5F7F4F813079F00C
:10D2A000813040F0823009F443C06EEE7FEF8FEFA3
:10D2B0009FEF6CC0F701A681B78182E04CC0E98185
:10D2C000FA813496FA83E983529142913291229104
:10D2D000FB0121938F01BB27A52F942F832FFB01E7
:10D2E0008183B8016F5F7F4F9A0144275527F8016A
:10D2F00021838B010F5F1F4FE981FA813496FA83F6
:10D30000E983B291A29192918291FB018183B8014C
:10D310006F5F7F4F292F3A2F4B2F5527F80121831D
:10D32000CD01AA27BB27FB0181836E5F7F4F0FC012
:10D33000E981FA813296FA83E983CB01B291A29115
:10D3400026E00D90FC010192CF012150D1F7F701A9
:10D35000A681B78188E08C93F2E0DF1679F4E98149
:10D36000FA813296FA83E98332978081FB018083C8
:10D37000F701A681B7818C918F5F8C93F70146816D
:10D38000578168897989C5010E94B96822960FB6CC
:10D39000F894DEBF0FBECDBFDF91CF911F910F91EB
:10D3A000FF90EF90DF90BF90AF9008958F929F9283
:10D3B000AF92BF92CF92DF92EF92FF920F931F93A3
:10D3C000CF93DF93CDB7DEB72C970FB6F894DEBFBF
:10D3D0000FBECDBF6C015B014A019C012F5E3F4F28
:10D3E00089E0E82EF12C04E0AB01BE016F5F7F4FB6
:10D3F000C6010E94C454FC0191868086F601148AFD
:10D400000FEF1FEF20E139E0A501BC01C6010E942A
:10D4100018552C960FB6F894DEBF0FBECDBFDF9126
:10D42000CF911F910F91FF90EF90DF90CF90BF9021
:10D43000AF909F908F900895AF92BF92CF92DF925E
:10D44000EF92FF920F931F93CF93DF93CDB7DEB789
:10D450002C970FB6F894DEBF0FBECDBF6C015B01F9
:10D460009C012F5E3F4F95E0E92EF12C04E0AB01CB
:10D47000BE016F5F7F4FC6010E94C454F601148A3B
:10D480000FEF1FEF20E135E0A501BC01C6010E94AE
:10D4900018552C960FB6F894DEBF0FBECDBFDF91A6
:10D4A000CF911F910F91FF90EF90DF90CF90BF90A1
:10D4B000AF900895AF92BF92CF92DF92EF92FF921A
:10D4C0000F931F93CF93DF93CDB7DEB72C970FB693
:10D4D000F894DEBF0FBECDBF6C015B019C012F5ED7
:10D4E0003F4F44E0E42EF12C04E0AB01BE016F5F3E
:10D4F0007F4F0E94C454F601148A0FEF1FEF20E102
:10D5000034E0A501BC01C6010E9418552C960FB647
:10D51000F894DEBF0FBECDBFDF91CF911F910F9169
:10D52000FF90EF90DF90CF90BF90AF9008958F92D3
:10D530009F92AF92BF92CF92DF92EF92FF920F93A2
:10D540001F93CF93DF93CDB7DEB72C970FB6F89428
:10D55000DEBF0FBECDBF6C015B014A019C012F5E97
:10D560003F4F53E0E52EF12C04E0AB01BE016F5FAD
:10D570007F4F0E94C454FC0191868086F601148A74
:10D580000FEF1FEF20E133E0A501BC01C6010E94AF
:10D5900018552C960FB6F894DEBF0FBECDBFDF91A5
:10D5A000CF911F910F91FF90EF90DF90CF90BF90A0
:10D5B000AF909F908F900895AF92BF92CF92DF92DD
:10D5C000EF92FF920F931F93CF93DF93CDB7DEB708
:10D5D0002C970FB6F894DEBF0FBECDBF6C015B0178
:10D5E0009C012F5E3F4F62E0E62EF12C04E0A50186
:10D5F000BE016F5F7F4F0E94C454F601148A0FEF83
:10D600001FEF20E132E0A501BC01C6010E941855C0
:10D610002C960FB6F894DEBF0FBECDBFDF91CF9131
:10D620001F910F91FF90EF90DF90CF90BF90AF9040
:10D6300008958F929F92AF92BF92CF92DF92EF9216
:10D64000FF920F931F93CF93DF93CDB7DEB72C9745
:10D650000FB6F894DEBF0FBECDBF6C014B015A016F
:10D660009C012F5E3F4F71E0E72EF12C04E0A401F6
:10D67000BE016F5F7F4F0E94C454FC01B186A0863B
:10D680001482158216821782F601148A0FEF1FEF9B
:10D6900020E131E0A401BC01C6010E9418552C967E
:10D6A0000FB6F894DEBF0FBECDBFDF91CF911F91B3
:10D6B0000F91FF90EF90DF90CF90BF90AF909F9031
:10D6C0008F9008956F927F928F929F92AF92BF92A8
:10D6D000CF92DF92EF92FF920F931F93CF93DF933E
:10D6E000CDB7DEB72C970FB6F894DEBF0FBECDBF17
:10D6F0006C014B013A01BA010E94A7545C018FEF03
:10D70000A8168FEFB80629F46DEF7EEF8FEF9FEF2D
:10D710001EC096012F5E3F4F4FE1E42EF12C01E039
:10D72000A401BE016F5F7F4FC6010E94C45422E076
:10D73000F601248BA58A2B2D3327268B830124E029
:10D740003FE140E050E0BC01C6010E9418552C9614
:10D750000FB6F894DEBF0FBECDBFDF91CF911F9102
:10D760000F91FF90EF90DF90CF90BF90AF909F9080
:10D770008F907F906F9008950F931F938B0124E0FB
:10D7800031E140E050E060E070E00E9418551F91E8
:10D790000F9108954F925F926F927F928F929F9216
:10D7A000AF92BF92CF92DF92EF92FF920F931F93AF
:10D7B000CF93DF93CDB7DEB72C970FB6F894DEBFCB
:10D7C0000FBECDBF6C014B012A013901BA010E9485
:10D7D000A7545C018FEFA8168FEFB80629F46DEF00
:10D7E0007EEF8FEF9FEF22C096012F5E3F4F7FE0CD
:10D7F000E72EF12C01E0A401BE016F5F7F4FC6014F
:10D800000E94C45424E0F601248BA58A2B2D3327D3
:10D81000268B678A272D3327208F820124E03FE063
:10D8200040E050E0BC01C6010E9418552C960FB68E
:10D83000F894DEBF0FBECDBFDF91CF911F910F9146
:10D84000FF90EF90DF90CF90BF90AF909F908F9020
:10D850007F906F905F904F9008956F927F928F921C
:10D860009F92AF92BF92CF92DF92EF92FF920F936F
:10D870001F93CF93DF93CDB7DEB72C970FB6F894F5
:10D88000DEBF0FBECDBF6C013B014A01122FBA01B2
:10D890000E94A7545C018FEFA8168FEFB80629F4F9
:10D8A0006DEF7EEF8FEF9FEF1EC096012F5E3F4F13
:10D8B000B6E0EB2EF12C01E0A301BE016F5F7F4FBC
:10D8C000C6010E94C45423E0F601248BA58A2B2DA7
:10D8D0003327268B178B840124E036E0A301BC019B
:10D8E000C6010E9418552C960FB6F894DEBF0FBEE5
:10D8F000CDBFDF91CF911F910F91FF90EF90DF90FF
:10D90000CF90BF90AF909F908F907F906F90089531
:10D91000AF92BF92CF92DF92EF92FF920F931F933D
:10D92000CF93DF93CDB7DEB72C970FB6F894DEBF59
:10D930000FBECDBF6C015B019C012F5E3F4F12E01B
:10D94000E12EF12C01E0AB01BE016F5F7F4F0E9421
:10D95000C454F601148A0FEF1FEF24E032E0A50152
:10D96000BC01C6010E9418552C960FB6F894DEBF74
:10D970000FBECDBFDF91CF911F910F91FF90EF9020
:10D98000DF90CF90BF90AF9008952F923F924F922B
:10D990005F926F927F928F929F92AF92BF92CF923F
:10D9A000DF92EF92FF920F931F93CF93DF93CDB748
:10D9B000DEB72D970FB6F894DEBF0FBECDBF2C019A
:10D9C0003B011A012D874801AE2C9C012F5E3F4F71
:10D9D00089E1E82EF12C01E040E050E0BE016F5FEC
:10D9E0007F4FC2010E94C454DC01FC0191868086F5
:10D9F000BB24CC24DD24A482B582C682D7828AE0EF
:10DA0000F201848BC2014596A30126E0FA01019040
:10DA1000AF01FC010192CF012150C1F78D85F201C8
:10DA2000838F148E258E832D9927868F0FEF1FEFFE
:10DA300024E039E140E050E0BD01C2010E941855E8
:10DA40002D960FB6F894DEBF0FBECDBFDF91CF91FC
:10DA50001F910F91FF90EF90DF90CF90BF90AF900C
:10DA60009F908F907F906F905F904F903F902F90FE
:10DA700008954F925F927F928F929F92AF92BF9242
:10DA8000CF92DF92EF92FF920F931F93CF93DF938A
:10DA9000CDB7DEB72C970FB6F894DEBF0FBECDBF63
:10DAA0006C012B014A01722E58019C012F5E3F4FE1
:10DAB0009DE0E92EF12C01E040E050E0BE016F5FF7
:10DAC0007F4FC6010E94C4548C0187E1F601848B0C
:10DAD000D6015596F40186E001900D928150E1F750
:10DAE000F601738EA501D60160E070E0272D332783
:10DAF0000DC07A01FA018191AF01FD01848F119669
:10DB0000F7018081882329F06F5F7F4F62177307C9
:10DB100081F7F80191868086820124E03DE040E0B3
:10DB200050E060E070E0C6010E9418552C960FB6D8
:10DB3000F894DEBF0FBECDBFDF91CF911F910F9143
:10DB4000FF90EF90DF90CF90BF90AF909F908F901D
:10DB50007F905F904F900895AF92BF92CF92DF92E7
:10DB6000EF92FF920F931F93CF93DF93CDB7DEB762
:10DB70002C970FB6F894DEBF0FBECDBF5C016B01D2
:10DB80009C012F5E3F4F4CE0E42EF12C01E040E081
:10DB900050E0BE016F5F7F4F0E94C45486E0F501E4
:10DBA000848BD5015596F60101900D928150E1F7D5
:10DBB0000FEF1FEF24E03CE040E050E060E070E059
:10DBC000C5010E9418552C960FB6F894DEBF0FBE03
:10DBD000CDBFDF91CF911F910F91FF90EF90DF901C
:10DBE000CF90BF90AF9008956F927F928F929F9247
:10DBF000AF92BF92CF92DF92EF92FF920F931F935B
:10DC0000CF93DF93CDB7DEB72C970FB6F894DEBF76
:10DC10000FBECDBF6C013B015A0149010E94A754C0
:10DC20008F5F9F4F29F46DEF7EEF8FEF9FEF38C02E
:10DC300096012F5E3F4F5BE0E52EF12C01E040E0C6
:10DC400050E0BE016F5F7F4FC6010E94C45486E161
:10DC5000F601848BD6015596F50186E001900D9270
:10DC60008150E1F7A401D60120E030E0FA01808183
:10DC7000FD01838FFA018081882341F02F5F3F4FA0
:10DC80004F5F5F4F11962F30310581F7830124E0FC
:10DC90003BE040E050E060E070E0C6010E941855B3
:10DCA0002C960FB6F894DEBF0FBECDBFDF91CF919B
:10DCB0001F910F91FF90EF90DF90CF90BF90AF90AA
:10DCC0009F908F907F906F900895AF92BF92CF9268
:10DCD000DF92EF92FF920F931F93CF93DF93CDB715
:10DCE000DEB72C970FB6F894DEBF0FBECDBF5C0138
:10DCF0006B01142F9C012F5E3F4F69E0E62EF12C43
:10DD000001E040E050E0BE016F5F7F4F0E94C454CD
:10DD100087E0F501848BD5015596F60186E00190E8
:10DD20000D928150E1F7F501138F0FEF1FEF24E003
:10DD300039E040E050E060E070E0C5010E94185515
:10DD40002C960FB6F894DEBF0FBECDBFDF91CF91FA
:10DD50001F910F91FF90EF90DF90CF90BF90AF9009
:10DD600008958F929F92AF92BF92CF92DF92EF92DF
:10DD7000FF920F931F93CF93DF93CDB7DEB72C970E
:10DD80000FB6F894DEBF0FBECDBF5C014B016A0138
:10DD90009C012F5E3F4F78E0E72EF12C01E0A401BB
:10DDA000BE016F5F7F4F0E94C454BC0186E0F50145
:10DDB000848BD5015596F60101900D928150E1F7C3
:10DDC0000FEF1FEF24E038E0A401C5010E941855B1
:10DDD0002C960FB6F894DEBF0FBECDBFDF91CF916A
:10DDE0001F910F91FF90EF90DF90CF90BF90AF9079
:10DDF0009F908F9008952F923F924F925F926F92D3
:10DE00007F928F929F92AF92BF92CF92DF92EF92CA
:10DE1000FF920F931F93CF93DF93CDB7DEB72D976C
:10DE20000FB6F894DEBF0FBECDBF5C011B014A01E7
:10DE300039010D8727011C2DBA010E94F6756D5F0F
:10DE40007E4F8F4F9F4F29F069EF7EEF8FEF9FEF4F
:10DE5000DBC0F4014081D501A358BD4F20E030E084
:10DE60008C91841749F5FD019181F4018181981706
:10DE700019F5FD019281F40182819817E9F4FD0101
:10DE80009381F40183819817B9F4FD019481F40121
:10DE90008481981789F4FD019581F4018581981793
:10DEA00059F4FD018585833009F4A5C0823009F459
:10DEB0009DC0843009F49AC02F5F3F4F57962A3097
:10DEC000310571F6D501A657BD4F40E050E020E086
:10DED00030E0F501E757FD4F8C91853039F48081B2
:10DEE00082958F70837011F44F5F5F4F2F5F3F4FAC
:10DEF000779657962A30310579F7473051050CF05F
:10DF00007FC0C5010E9462546C018F5F9F4F09F46E
:10DF100077C095012F5E3F4F05E0E02EF12C01E028
:10DF2000A101BE016F5F7F4FC5010E94C454BC01B7
:10DF30008DE0F501848BD5015596F40186E00190C2
:10DF40000D928150E1F7F501638E872D9927848F1B
:10DF50002D85258F168E478E852D992780A311A399
:10DF600087E190E0C89EF001C99EF00DD89EF00DAB
:10DF70001124E358FD4FEA0DFB1DD40186E00D90FE
:10DF800001928150E1F787E190E0C89EF001C99EBF
:10DF9000F00DD89EF00D1124EA0DFB1DE657FD4F44
:10DFA00083E08083EA58F240809188089091890844
:10DFB000DF01A758BD4F11969C938E9301969093C5
:10DFC000890880938808E757FD4F1295110F110FAC
:10DFD000107C80818F70812B80830D911C9124E0B7
:10DFE00035E0A101C5010E9418550EC067EF7EEF14
:10DFF0008FEF9FEF09C068EF7EEF8FEF9FEF04C0B8
:10E000006CEF7EEF8FEF9FEF2D960FB6F894DEBF8B
:10E010000FBECDBFDF91CF911F910F91FF90EF9079
:10E02000DF90CF90BF90AF909F908F907F906F9038
:10E030005F904F903F902F9008956F927F928F92B4
:10E040009F92AF92BF92CF92DF92EF92FF920F9387
:10E050001F93CF93DF93CDB7DEB72C970FB6F8940D
:10E06000DEBF0FBECDBF4C013B01B42EA22E680116
:10E070009C012F5E3F4F91E0E92EF12C01E0AB01B6
:10E08000BE016F5F7F4FC4010E94C4547C01C40174
:10E09000885B9D4F0E94E876F701148215821682F4
:10E0A0001782D186C08685E0F401848B83E3858B5B
:10E0B0008BE8868B8EE9878B8B2D813308F080E38C
:10E0C000F401808FAA2011F481E0A82EF401A18E22
:10E0D0000FEF1FEF24E031E0A301B701C4010E945C
:10E0E00018552C960FB6F894DEBF0FBECDBFDF914A
:10E0F000CF911F910F91FF90EF90DF90CF90BF9045
:10E10000AF909F908F907F906F9008956F927F92C5
:10E110008F929F92AF92BF92CF92DF92EF92FF9237
:10E120000F931F93CF93DF93CDB7DEB72C970FB626
:10E13000F894DEBF0FBECDBF6C013B014A01BA01AE
:10E140000E94A7545C018FEFA8168FEFB80629F440
:10E150006DEF7EEF8FEF9FEF1DC096012F5E3F4F5B
:10E1600046E0E42EF12C02E0A301BE016F5F7F4F79
:10E17000C6010E94C45422E0F601248BA58A2B2DEF
:10E180003327268B840128E036E0A301BC01C601B9
:10E190000E9418552C960FB6F894DEBF0FBECDBF67
:10E1A000DF91CF911F910F91FF90EF90DF90CF9073
:10E1B000BF90AF909F908F907F906F9008952F9217
:10E1C0003F924F925F926F927F928F929F92AF9207
:10E1D000BF92CF92DF92EF92FF920F931F93CF9354
:10E1E000DF93CDB7DEB72C970FB6F894DEBF0FBE26
:10E1F000CDBF6C011B012A0149013801BA010E94FF
:10E20000A7545C018FEFA8168FEFB80629F46DEFC5
:10E210007EEF8FEF9FEF25C096012F5E3F4FE5E029
:10E22000EE2EF12C02E0A101BE016F5F7F4FC6010F
:10E230000E94C45426E0F601248BA58A2B2D332797
:10E24000268B878A292D3327208F618E272D332710
:10E25000228F820128E035E0A101BC01C6010E94A5
:10E2600018552C960FB6F894DEBF0FBECDBFDF91C8
:10E27000CF911F910F91FF90EF90DF90CF90BF90C3
:10E28000AF909F908F907F906F905F904F903F9056
:10E290002F9008956F927F928F929F92AF92BF922C
:10E2A000CF92DF92EF92FF920F931F93CF93DF9362
:10E2B000CDB7DEB72C970FB6F894DEBF0FBECDBF3B
:10E2C0006C013B014A01BA010E94A7545C018FEF27
:10E2D000A8168FEFB80629F46DEF7EEF8FEF9FEF52
:10E2E0001DC096012F5E3F4FB4E0EB2EF12C02E0F3
:10E2F000A301BE016F5F7F4FC6010E94C45422E09C
:10E30000F601248BA58A2B2D3327268B840128E048
:10E3100034E0A301BC01C6010E9418552C960FB62B
:10E32000F894DEBF0FBECDBFDF91CF911F910F914B
:10E33000FF90EF90DF90CF90BF90AF909F908F9025
:10E340007F906F9008952F923F924F925F926F92BD
:10E350007F928F929F92AF92BF92CF92DF92EF9275
:10E36000FF920F931F93CF93DF93CDB7DEB76097E4
:10E370000FB6F894DEBF0FBECDBF5C017E876D8700
:10E38000588B4F874901380127011601BA010E94B5
:10E39000A7546C018FEFC8168FEFD80629F46DEFE4
:10E3A0007EEF8FEF9FEF30C095012F5E3F4F53E020
:10E3B000E52EF12C02E04D855E85BE016F5F7F4F3B
:10E3C000C5010E94C4542AE0F501248BC58A2D2D75
:10E3D0003327268B878A292D3327208F618E272D7F
:10E3E0003327228F438E252D3327248F258E232DEF
:10E3F0003327268F0F85188928E033E04D855E8509
:10E40000BC01C5010E94185560960FB6F894DEBF96
:10E410000FBECDBFDF91CF911F910F91FF90EF9075
:10E42000DF90CF90BF90AF909F908F907F906F9034
:10E430005F904F903F902F9008952F923F924F9270
:10E440005F926F927F928F929F92AF92BF92CF9284
:10E45000DF92EF92FF920F931F93CF93DF93CDB78D
:10E46000DEB72C970FB6F894DEBF0FBECDBF6C01A0
:10E470001B012A0149013801BA010E94A7545C011D
:10E480008FEFA8168FEFB80629F46DEF7EEF8FEFB0
:10E490009FEF25C096012F5E3F4FB1E0EB2EF12C90
:10E4A00002E0A101BE016F5F7F4FC6010E94C4540C
:10E4B00026E0F601248BA58A2B2D3327268B878A0D
:10E4C000292D3327208F618E272D3327228F82011C
:10E4D00028E031E0A101BC01C6010E9418552C962C
:10E4E0000FB6F894DEBF0FBECDBFDF91CF911F9165
:10E4F0000F91FF90EF90DF90CF90BF90AF909F90E3
:10E500008F907F906F905F904F903F902F900895E5
:10E51000AF92BF92CF92DF92EF92FF920F931F9331
:10E52000CF93DF93CDB7DEB72C970FB6F894DEBF4D
:10E530000FBECDBF6C015B019C012F5E3F4F1EE003
:10E54000E12EF12C02E0AB01BE016F5F7F4F0E9414
:10E55000C454F601148A0FEF1FEF28E03EE0A50136
:10E56000BC01C6010E9418552C960FB6F894DEBF68
:10E570000FBECDBFDF91CF911F910F91FF90EF9014
:10E58000DF90CF90BF90AF9008954F925F926F92BF
:10E590007F928F929F92AF92BF92CF92DF92EF9233
:10E5A000FF920F931F93CF93DF93CDB7DEB72C97D6
:10E5B0000FB6F894DEBF0FBECDBF6C012B013A0140
:10E5C0004901BA010E94A7545C018FEFA8168FEF92
:10E5D000B80629F46DEF7EEF8FEF9FEF21C0960113
:10E5E0002F5E3F4F4DE0E42EF12C02E0A201BE0170
:10E5F0006F5F7F4FC6010E94C45424E0F601248B54
:10E60000A58A2B2D3327268B878A292D3327208F08
:10E61000830128E03DE0A201BC01C6010E9418551B
:10E620002C960FB6F894DEBF0FBECDBFDF91CF9111
:10E630001F910F91FF90EF90DF90CF90BF90AF9020
:10E640009F908F907F906F905F904F9008956F9202
:10E650007F928F929F92AF92BF92CF92DF92EF9272
:10E66000FF920F931F93CF93DF93CDB7DEB72C9715
:10E670000FB6F894DEBF0FBECDBF6C013B014A015F
:10E68000BA010E94A7545C018FEFA8168FEFB8065D
:10E6900029F46DEF7EEF8FEF9FEF1DC096012F5E87
:10E6A0003F4F6CE0E62EF12C02E0A301BE016F5F4C
:10E6B0007F4FC6010E94C45422E0F601248BA58A34
:10E6C0002B2D3327268B840128E03CE0A301BC01DD
:10E6D000C6010E9418552C960FB6F894DEBF0FBEE7
:10E6E000CDBFDF91CF911F910F91FF90EF90DF9001
:10E6F000CF90BF90AF909F908F907F906F90089534
:10E700006F927F928F929F92AF92BF92CF92DF9241
:10E71000EF92FF920F931F93CF93DF93CDB7DEB7A6
:10E720002C970FB6F894DEBF0FBECDBF6C013B0136
:10E730004A01BA010E94A7545C018FEFA8168FEF1F
:10E74000B80629F46DEF7EEF8FEF9FEF1DC09601A5
:10E750002F5E3F4FE9E0EE2EF12C02E0A301BE0157
:10E760006F5F7F4FC6010E94C45422E0F601248BE4
:10E77000A58A2B2D3327268B840128E039E0A301BD
:10E78000BC01C6010E9418552C960FB6F894DEBF46
:10E790000FBECDBFDF91CF911F910F91FF90EF90F2
:10E7A000DF90CF90BF90AF909F908F907F906F90B1
:10E7B00008956F927F928F929F92AF92BF92CF9265
:10E7C000DF92EF92FF920F931F93CF93DF93CDB71A
:10E7D000DEB72C970FB6F894DEBF0FBECDBF6C012D
:10E7E0003B014A011CE6A12E13E0B12EA80EB91E72
:10E7F0009C012F5E3F4FBFE0EB2EF12C02E0AB01FE
:10E80000BE016F5F7F4F0E94C4547C01F50184817B
:10E810009581892B39F482E090E00E94000CF5018B
:10E8200095838483F501A481B5818D929C9282E0C9
:10E83000F601848B858A892D9927868B0FEF1FEF30
:10E8400028E03FE0A301B701C6010E9418552C96AD
:10E850000FB6F894DEBF0FBECDBFDF91CF911F91F1
:10E860000F91FF90EF90DF90CF90BF90AF909F906F
:10E870008F907F906F9008958F929F92AF92BF92EA
:10E88000CF92DF92EF92FF920F931F93CF93DF937C
:10E89000CDB7DEB72C970FB6F894DEBF0FBECDBF55
:10E8A0006C014B015A01122FBA010E94A7548F5FCD
:10E8B0009F4F29F46DEF7EEF8FEF9FEF23C09601FE
:10E8C0002F5E3F4F0BE0E02EF12C02E0A401BE01D1
:10E8D0006F5F7F4FC6010E94C4547C0187E0F60140
:10E8E000848BA6014B5E5F4FB501C6010E944E7638
:10E8F000F601138F850128E03BE0A401B701C601B2
:10E900000E9418552C960FB6F894DEBF0FBECDBFEF
:10E91000DF91CF911F910F91FF90EF90DF90CF90FB
:10E92000BF90AF909F908F9008956F927F928F923B
:10E930009F92BF92CF92DF92EF92FF920F931F931D
:10E94000CF93DF93CDB7DEB72C970FB6F894DEBF29
:10E950000FBECDBF6C01B62E8C0104591C4FD801DF
:10E960008D919C91892B39F481E090E00E94000CFC
:10E97000F80191838083D801ED91FC91B082B2E0DF
:10E98000BB16D9F1BB1538F0BB20C1F0E1E0BE16D3
:10E9900009F07AC00AC0F4E0BF1609F1BF1628F1E9
:10E9A00085E0B81609F070C012C0BAE0BB2E612C29
:10E9B000A4E87A2EA3E08A2E912C27C0FCE0BF2E7B
:10E9C000612CE8E07E2EE7E08E2E912C1EC073E0D5
:10E9D000B72E612C6BE4762E812C912C16C0612C05
:10E9E00056E9752E812C912C10C046E0B42E612C76
:10E9F00031EE732E812C912C08C028E0B22E612CB0
:10EA000092EC792E91E0892E912C96012F5E3F4F4A
:10EA10008FE0E82EF12C0FE340E050E0BE016F5F85
:10EA20007F4FC6010E94C4547C0185E0F601848BAF
:10EA300083E0858B168A178AB08E118E0FEF1FEF39
:10EA40002CEF3FE0A701B701C6010E9418556115E0
:10EA5000710581059105C1F4F601828193810E94BF
:10EA6000CC2EB401A3010E948A52892B69F440E0A4
:10EA700050E060E070E0C7010A960E943D1060E03F
:10EA800070E080E090E004C06FEF7EEF8FEF9FEFCB
:10EA90002C960FB6F894DEBF0FBECDBFDF91CF919D
:10EAA0001F910F91FF90EF90DF90CF90BF909F90BC
:10EAB0008F907F906F900895FC01E758FD4F20E004
:10EAC00030E0DC01A757BD4F8189853071F480812A
:10EAD00091818617970749F48C9182958F70837086
:10EAE000682F77278827992708952F5F3F4F5796DC
:10EAF00077962A30310541F76DEF7EEF8FEF9FEF6C
:10EB00000895CF93DF93FC01E758FD4F20E030E0FC
:10EB1000EC01C557DD4F81898530B1F48081918149
:10EB20008617970789F489819A81AA27BB2722270C
:10EB3000382F492F5A2F88819927AA27BB27282B9E
:10EB4000392B4A2B5B2B0BC02F5F3F4F6796779675
:10EB50002A30310501F72DEF3EEF4FEF5FEFCA018D
:10EB6000B901DF91CF910895FC01E758FD4F20E0F6
:10EB700030E0DC01AB57BD4F8189853051F4808195
:10EB800091818617970729F46D917D918D919C91C4
:10EB900008952F5F3F4F579677962A30310561F7DA
:10EBA0006DEF7EEF8FEF9FEF0895DC01A758BD4F0B
:10EBB00030E020E0FD018189853079F4611571052F
:10EBC00059F0E22FFF27EE0FFF1FE60FF71F8D9181
:10EBD0009C911197918380832F5F3F5F57963A30C6
:10EBE00049F7622F7727882799270895CF93DF93D6
:10EBF000DB01FC01E358FD4F20E030E0AC01475859
:10EC00005D4F8585853009F590818C919817E9F4E1
:10EC10009181ED0189819817C1F492818A819817B9
:10EC2000A1F493818B81981781F494818C8198173A
:10EC300061F495818D81981741F4FA018081918169
:10EC40009C01B901882799270CC02F5F3F4F495E6F
:10EC50005F4F77962A303105A1F66DEF7EEF8FEF8B
:10EC60009FEFDF91CF910895FC01E758FD4F20E021
:10EC70008189853051F4808191818617970729F425
:10EC800060E070E080E090E008952F5F77962A3092
:10EC900079F76DEF7EEF8FEF9FEF0895FC01E75856
:10ECA000FD4FA0E0B0E09C0123583D4F81898530A5
:10ECB00089F4808191818617970761F4DA01F9015F
:10ECC00086E001900D928150E1F760E070E080E015
:10ECD00090E008951196295E3F4F7796AA30B105CE
:10ECE00029F76DEF7EEF8FEF9FEF0895DB01FC01B9
:10ECF000EA59FC4F86E001900D928150E1F760E007
:10ED000070E080E090E00895FC018281938100979B
:10ED100019F48FEF9FEF089501979383828380E02A
:10ED200090E0089569E976E78DEB97E00E94133C47
:10ED30000895CF93DF93C0913708D091380819C058
:10ED4000E881F981828193819F938F93FF93EF9361
:10ED500082EC97E09F938F930E94D1390A80DB81E8
:10ED6000C02D8DB79EB706960FB6F8949EBF0FBE06
:10ED70008DBF209729F7DF91CF910895FC01828103
:10ED80009381680F791F73836283892B19F4CF01F4
:10ED90000E94AA0F80E090E00895FC018281938197
:10EDA00073836283892B19F4CF010E94AA0F80E03C
:10EDB00090E00895FC018281938101969383828380
:10EDC000019719F4CF010E945B0F80E090E0089555
:10EDD000CF93DF93EC0107C040E050E060E070E0CB
:10EDE000CE010E943D108A819B810097A9F3019773
:10EDF0009B838A8380E090E0DF91CF9108950F9309
:10EE00001F93CF93DF938C01FC01118210827383D7
:10EE10006283C0913708D0913808209759F484E074
:10EE200090E00E94EC0CFC01909338088093370826
:10EE30000CC0EC018A819B810097D9F784E090E0B7
:10EE40000E94EC0CFC019B838A8311830083DF9179
:10EE5000CF911F910F910895FC0140E050E060E0D8
:10EE600070E0808191810E943A30892B19F08FEFF8
:10EE70009FEF089580E090E00895CF93DF93CDB7A2
:10EE8000DEB722970FB6F894DEBF0FBECDBFFE01EE
:10EE9000379661917191FA83E983AF018091AB0557
:10EEA0009091AC050E94F14622960FB6F894DEBF11
:10EEB0000FBECDBFDF91CF9108956091AB057091EA
:10EEC000AC050E942C2F0895CF93DF93CDB7DEB70A
:10EED00022970FB6F894DEBF0FBECDBFFE01379666
:10EEE00061917191FA83E983AF018091AB059091B3
:10EEF000AC050E948F3022960FB6F894DEBF0FBE8D
:10EF0000CDBFDF91CF9108953F924F925F926F9264
:10EF10007F928F929F92AF92BF92CF92DF92EF92A9
:10EF2000FF920F931F93CF93DF938C012B01EA0184
:10EF30006115710519F0FB0191838083209749F0D9
:10EF4000CE010297839728F060E070E080E090E0C7
:10EF5000F6C0F801E1908F018E2D99270E94F37A77
:10EF6000892BB9F7FDE2EF1631F4F801E1908F013A
:10EF700081E0382E07C0FBE2EF1619F4F801E190AA
:10EF80008F013324209719F0C031D105C1F4F0E38B
:10EF9000EF1679F4F8018081883711F0883549F44B
:10EFA000F801E1800E5F1F4FF2E03F2AC0E1D0E0A0
:10EFB00006C0209721F480E3E816E9F427C0C830A2
:10EFC000D10531F1C930D10524F4C230D10531F574
:10EFD0000CC0CA30D10589F0C031D105F9F4A12C9B
:10EFE000B12CC12CB8E0DB2E26C0A12CB12CC12C39
:10EFF000A0E4DA2E20C0CAE0D0E0FCECAF2EFCEC9E
:10F00000BF2EFCECCF2EFCE0DF2E15C0C8E0D0E018
:10F01000A12CB12CC12CE0E1DE2E0DC09E014427B5
:10F0200037FD4095542F60E070E080E090E80E944A
:10F03000AC7A59016A0120E030E040E050E060E045
:10F040003E01882477FC8094982C70EDF72EFE0CFE
:10F05000E9E0EF1570F48E2D81548A3118F499ECA3
:10F06000F92E06C08E2D81568A3150F589EAF82E88
:10F07000FE0C8F2D99278C179D0714F567FD1CC07A
:10F08000A216B306C406D506B0F0CA01B901A401A0
:10F0900093010E945A7A9B01AC012F0D311D411D35
:10F0A000511D2130F0E03F07F0E04F07F0E85F0727
:10F0B00010F461E001C06FEFF801E1908F01C5CF5E
:10F0C0004114510481F0662331F001501040F201E7
:10F0D0001183008308C031FE1AC002501040F201B3
:10F0E0001183008314C067FF12C030FE05C020E00A
:10F0F00030E040E050E804C02FEF3FEF4FEF5FE714
:10F1000082E290E090938B0880938A0816C030FECC
:10F1100008C050954095309521953F4F4F4F5F4F18
:10F120000CC057FF0AC082E290E090938B08809356
:10F130008A082FEF3FEF4FEF5FE7CA01B901DF9178
:10F14000CF911F910F91FF90EF90DF90CF90BF90E4
:10F15000AF909F908F907F906F905F904F903F9077
:10F1600008952F923F924F925F926F927F928F926B
:10F170009F92AF92BF92CF92DF92EF92FF920F9346
:10F180001F93CF93DF93CDB7DEB723970FB6F894D5
:10F19000DEBF0FBECDBF9B838A831B016A01611551
:10F1A000710519F0FB0191838083C114D10449F0EA
:10F1B000C6010297839728F040E050E060E070E0DD
:10F1C000EFC0EA81FB811191FB83EA83812F9927AC
:10F1D0000E94F37A892BA9F71D3241F4EA81FB8161
:10F1E0001191FB83EA83F1E0F98308C01B3229F413
:10F1F000EA81FB811191FB83EA831982C114D10456
:10F2000021F0F0E1CF16D10439F51033A1F4EA81F1
:10F21000FB818081883711F0883569F4EA81FB81B0
:10F2200011813296FB83EA83F981F260F98360E110
:10F23000C62ED12C11C0C114D10471F4103359F56C
:10F240005FEF852E5FEF952E5FEFA52E5FE1B52E68
:10F2500048E0C42ED12C38C08AE0C816D104F1F0A1
:10F2600090E1C916D10429F0E8E0CE16D104F9F4F2
:10F2700009C03FEF832E3FEF932E3FEFA32E3FE0D9
:10F28000B32E22C02FEF822E2FEF922E2FEFA22E21
:10F290002FE1B22E19C09AE0C92ED12C89E9882E0F
:10F2A00089E9982E89E9A82E89E1B82E0DC096012A
:10F2B000442737FD4095542F6FEF7FEF8FEF9FEF7F
:10F2C0000E94AC7A49015A0140E050E060E070E0F1
:10F2D00030E02601662457FC6094762C212F2053C1
:10F2E0002A3060F0812F81548A3110F4275006C0F3
:10F2F000812F81568A3160F5212F2755822F99273A
:10F300008C159D052CF537FD1DC084169506A606A7
:10F31000B706B8F0E22EFF2400271127CB01BA016F
:10F32000A30192010E945A7AAB01BC014E0D5F1DF0
:10F33000601F711F4E155F056007710710F031E007
:10F3400001C03FEFEA81FB811191FB83EA83C6CFC5
:10F350002114310479F0332321F08A819B810197B4
:10F3600006C0F981F1FF06C08A819B810297F101F5
:10F3700091838083F981F0FF07C070956095509567
:10F3800041955F4F6F4F7F4F37FF0AC082E290E099
:10F3900090938B0880938A084FEF5FEF6FEF7FEFBA
:10F3A000CB01BA0123960FB6F894DEBF0FBECDBFD6
:10F3B000DF91CF911F910F91FF90EF90DF90CF9051
:10F3C000BF90AF909F908F907F906F905F904F9085
:10F3D0003F902F900895FB01DC0140FF05C002C063
:10F3E00005900D9205900D9242505040C8F7089537
:10F3F000FB01DC0105900D920020E1F70895FC016E
:10F4000005900020E9F7809590958E0F9F1F089535
:10F41000FC014150504030F001900616D1F7319771
:10F42000CF010895882799270895FB01DC0140FF4B
:10F4300005C002C001900D9201900D9242505040C3
:10F44000C8F70895DC0140FF03C001C06D936D93C0
:10F4500042505040D8F70895FB01DC018D91019096
:10F46000801911F40020D1F7990B0895FB01DC01FC
:10F4700001900D920020E1F70895FB01DC0141505D
:10F48000504030F08D910190801919F40020B9F7A7
:10F49000881B990B0895FB01DC014150504048F056
:10F4A00001900D920020C9F701C01D9241505040BB
:10F4B000E0F70895629FD001739FF001829FE00DF5
:10F4C000F11D649FE00DF11D929FF00D839FF00DE3
:10F4D000749FF00D659FF00D9927729FB00DE11D8F
:10F4E000F91F639FB00DE11DF91FBD01CF0111246C
:10F4F0000895991B79E004C0991F961708F0961B90
:10F50000881F7A95C9F780950895AA1BBB1B51E106
:10F5100007C0AA1FBB1FA617B70710F0A61BB70B83
:10F52000881F991F5A95A9F780959095BC01CD0128
:10F53000089597FB092E07260AD077FD04D0E5DF52
:10F5400006D000201AF4709561957F4F0895F6F764
:10F55000909581959F4F0895A1E21A2EAA1BBB1B7F
:10F56000FD010DC0AA1FBB1FEE1FFF1FA217B3078F
:10F57000E407F50720F0A21BB30BE40BF50B661FA5
:10F58000771F881F991F1A9469F760957095809569
:10F5900090959B01AC01BD01CF01089597FB092E09
:10F5A00005260ED057FD04D0D7DF0AD0001C38F452
:10F5B00050954095309521953F4F4F4F5F4F08959F
:10F5C000F6F790958095709561957F4F8F4F9F4F7F
:10F5D0000895082E8062813624F087360CF4089551
:10F5E0002BC0802D36C0911127C0803251F08A3057
:10F5F00041F08C3031F08D3021F0893011F08B30BA
:10F6000099F708958F931DD08F9109F08062089526
:10F61000E199FECFBFBBAEBBE09A11960DB2089543
:10F62000E199FECFBFBBAEBB0DBA11960FB6F894F1
:10F63000E29AE19A0FBE089599278827089585FDDB
:10F64000FBCF80629111F8CF8136ECF38B37DCF77A
:0EF6500008959111F1CF80538A50E0F708958C
:10F65E00722B005B73656E736F5D24000A23202D81
:10F66E002D2D2D2D2D2D2D2D2D2D2D2D2D2D2D2DBC
:10F67E002D2D2D2D2D2D2D2D2D2D2D2D2D2D2D2DAC
:10F68E002D2D2D2D2D2D2D000A232053656E736FDC
:10F69E003A20612053656E736F722D44656D6F2035
:10F6AE00286329203230303520455448205A75724F
:10F6BE006963680A0032303036313231382D3134D8
:10F6CE0030320023202D2D2D2D2D2D2D2D2D2D2D98
:10F6DE002D2D2D2D2D2D2D2D2D2D2D2D2D2D2D2D4C
:10F6EE002D2D2D2D2D2D2D2D2D2D2D2D2D0A006D4C
:10F6FE006F6E006865617000746872656164730096
:10F70E0074696D6572730062617400697271007262
:10F71E006567006E657400636D6420007665720027
:10F72E003A4D435F5354415254003A4D435F454E58
:10F73E0044008204AA04D204F0040E050004280436
:10F74E0046049604BE0418050A0432046E04DC0452
:10F75E00FA048C04A004C8047804F60364041E049E
:10F76E005004E6040405220514043C04D407D4070F
:10F77E00D4075A04B4040000010002000300040080
:10F78E00050006000700080009000A000B000C0027
:10F79E000D000E000F0010001200140016001800CD
:10F7AE001A001C001E002000220024002600280043
:10F7BE002A002C002E003100350039003D0041009A
:10F7CE00450049004D005100550059005D00610093
:10F7DE00650069006D0073007B0083008B00930051
:10F7EE009B00A300AB00B300BB00C300CB00D30053
:10F7FE00DB00E300EB00F7000701170127013701DB
:10F80E00470157016701770187019701A701B701EA
:10F81E00C701D701E701FF011F023F025F027F020E
:10F82E009F02BF02DF02FF021F033F035F037F033E
:10F83E009F03BF03DF030F044F048F04CF040F0594
:10F84E004F058F05CF050F064F068F06CF060F0704
:10F85E004F078F07CF072F08AF082F09AF092F0AC1
:10F86E00AF0A2F0BAF0B2F0CAF0C2F0DAF0D2F0EB2
:10F87E00AF0E2F0FAF0F64646464646464646464D9
:10F88E006464646463636363636363636363636336
:10F89E006362626262626262616161616160606044
:10F8AE00605F5F5F5E5E5D5D5D5C5C5B5B5A595980
:10F8BE00585757565554535251504F4E4D4B4A4927
:10F8CE0047454442403E3C3A383634312F2C2A29A3
:10F8DE0028282727262625252524242423232323C9
:10F8EE00222222222121212120202020201F1F1F01
:10F8FE001F1F1E1E1E1E1E6D696373616D700065D7
:10F90E00746865726E75740069646C65006D61690A
:10F91E006E00FF4641494C004F4B005349474E4144
:10F92E004C4544005349474E414C45440A005452FD
:10F93E004D0052554E0052445900534C5000DE03B8
:10F94E00E203E603EA0300000000000000001C12C0
:10F95E0000000000000000009712000000000000F0
:10F96E00000061130000000000000000E41300001E
:10F97E000000000000006E140000000000000000F7
:10F98E00E9140000000000000000B71500000000A0
:10F99E00000000003A160000000000000000C4162F
:10F9AE0000000000000000008E17000000000000A4
:10F9BE00000018180000000000000000A21800004F
:10F9CE00000000000000FC18000000000000000015
:10F9DE007F190000000000000000FC19000000006C
:10F9EE0000000000CF1A00000000000000004D1BB8
:10F9FE000000000000000000D01B0000000000000E
:10FA0E0000004C1C0000000000000000181D00004B
:10FA1E00000000000000791D000000000000000042
:10FA2E00FC1D0000000000000000721E000000001F
:10FA3E0000000000411F0000000000000000C41F75
:10FA4E0000000000000000004A200000000000003E
:10FA5E000000192100000000000000009C210000A1
:10FA6E000000000000002622000000000000000040
:10FA7E00F4220000000000000000772300007561F2
:10FA8E00727430000000000500000000004F0556A3
:10FA9E0041D5413E4536452E458143EF43724100E7
:10FAAE000000000000000000000000000000000048
:10FABE000000000000000000000000000000000038
:10FACE000000000000000000000000000000000028
:10FADE00000000001627ED26362638263B27162670
:10FAEE009627A0266426F8241228152546282625B2
:10FAFE009A253025D627FF250801000200030000B5
:10FB0E00000000000000000000286E756C6C2900DB
:10FB1E003031323334353637383961626364656675
:10FB2E00003031323334353637383941424344456B
:10FB3E0046002020202020202020202020202020B1
:10FB4E0020203030303030303030303030303030C7
:10FB5E003030004C4544000F01545F5445524D491E
:10FB6E004E414C006C656400626174007061747487
:10FB7E0065726E2575257525752575007061747411
:10FB8E0065726E636C72006F6E2575006F6666250A
:10FB9E007500686225752575257500757361676535
:10FBAE003A0A206C6564207061747465726E203C34
:10FBBE0073706565643A312D31303E203C64757248
:10FBCE006174696F6E3E203C6E723A312D383E2064
:10FBDE005B6172675D0A206C656420706174746588
:10FBEE00726E636C720A206C6564206F6E203C6EC0
:10FBFE00723A302D333E0A206C6564206F666620A3
:10FC0E003C6E723A302D333E0A206C656420686279
:10FC1E00203C70617573653E203C342D6269742002
:10FC2E007061747465726E3E203C647572617469A5
:10FC3E006F6E3E0A004261747465727920566F6C65
:10FC4E00746167653A2025642E2530326420560A89
:10FC5E000D00082008000A00256300252E32783A90
:10FC6E00252E32783A252E32783A252E32783A25BC
:10FC7E002E32783A252E327800252E327820003119
:10FC8E00323334004254537461636B005F554152FA
:10FC9E00547772697465206572726F72210A005F03
:10FCAE005541525472656164206572726F72210AF9
:10FCBE00006672616D696E67206572726F720A00FE
:10FCCE00627566666572206F76657272756E2065F6
:10FCDE0072726F720A007061726974792065727245
:10FCEE006F720A007061636B6574206F7574206F9C
:10FCFE00662073796E6320746F2042542075617292
:10FD0E0074210A00722B00307825580A0073656D35
:10FD1E00610073656D612025703A2025640A00002C
:00000001FF
